:020000040800F2
:100000000020001061B60208416B020851FF000891
:100010003D6B0208396B0208356B020800000000D6
:10002000000000000000000000000000316B02082A
:100030002D6B020800000000256B020879CC000837
:10004000C9B60208C9B60208C9B60208C9B602088C
:10005000C9B60208C9B60208591B0008851C000869
:10006000491C00080D1C0008D11B0008AD2C00081D
:100070009D2C00088D2C00087D2C00086D2C00089C
:10008000592C0008452C0008C9B60208C9B6020858
:10009000D52E0208C9B60208C9B60208951B000889
:1000A000D1C3000821C40008C9B6020831C4000841
:1000B00011C4000801C40008C9B60208C9B6020884
:1000C000C9B60208C9B60208C9B60208C9B602080C
:1000D000C9B60208FDCD000881CD000805CD000895
:1000E0001F1B0008C9B60208C52E0208C9B60208BF
:1000F000E1C30008C9B60208F1C30008C9B6020886
:10010000000000000000000000000000C9B6020866
:10011000C9B60208C9B60208BD1B0108A11B010827
:10012000312C00081D2C0008092C0008F52B0008B4
:10013000E12B0008C9B60208000000000000000022
:10014000C9B60208C9B60208C9B602080000000014
:10015000000000000000000000000000000000009F
:100160000000000000000000C9B60208C9B602087D
:10017000C9B60208000000000000000000000000F6
:0801800000000000C9B60208EE
:100188000A4B30B503F10C0493F900205D78072A77
:10019800C8BF143A811804338D7213F8025C855471
:1001A80013F8012C0A75A342EED130BDF4DE020823
:1001B80003682DE9F041DF691FB13B46BDE8F04116
:1001C8001847002A164611DD04460D460E4400E085
:1001D80023689B68204698470028F9D0236815F8BB
:1001E800011B1B6820469847AE42F1D1BDE8F0815B
:1001F80000232822027043708370C3707047232342
:1002080003702423C37025238371704730B4836837
:1002180013B11C689B882385436840F2E93401E0E8
:10022800002C3FD01D89013C15F0020FA4B2F7D075
:10023800197303F10C0540F2E93101E000293BD0C4
:100248001C89013914F0010F89B2F7D02B78436863
:1002580040F2E93100E0D9B11C89013914F0020FEC
:1002680089B2F8D01A7303F10C0440F2E93200E0C5
:1002780072B11989013A11F0010F92B2F8D02378BE
:10028800836813B11A689B889361012030BC70475A
:100298000F4A9342F4D10F4A538901339BB25381D9
:1002A8005389EDE70A498B42D2D10A4C6189013161
:1002B80089B261816189CBE705498B42C7D105497C
:1002C8004B8901339BB24B814B894368C0E700BF20
:1002D800003001405C680020002870B51EDB09284A
:1002E800044620DD012303EB83035B00B0FBF3F23C
:1002F800092AF8D87BB10E4EB4FBF3F00928CCBF1D
:1003080057223022A6FB03E5024403FB1044EB0806
:1003180001F8012BF0D100230B7070BD2D230B7059
:1003280040420131DBE7303001F8010BF3E700BF51
:10033800CDCCCCCC884230B44FF001042ED301FB95
:1003480004F4B0FBF4F58D42F9D284B1AAB901E006
:10035800B0FBF4F5092DCCBF572230222A4404FB08
:10036800150003F8012BB4FBF1F4002CF0D10022A6
:100378001A7030BC7047B0FBF4F5092DCCBF37229A
:1003880030222A4404FB150003F8012BB4FBF1F4D6
:10039800002CF0D100221A7030BC70470546002AA4
:1003A800EBD1D7E703685A1C0260197070472DE932
:1003B800F047089C2578002B804689460CBF4FF0F3
:1003C800200A4FF0300A661C35B3002A29DD33466F
:1003D80001E0024698B113F8011B501E0029F8D11C
:1003E800971E60B13D46013D51464046C8476B1CCB
:1003F800002BF8DC257827EAE770013055B1041B9B
:1004080029464046C847301916F8015B002DF7D138
:10041800BDE8F087BDE8F087002A04DC2846BDE87F
:10042800F0870020EBE7571EDCE783684268D0EDD1
:10043800037A00EB83010133934281ED040A836060
:1004480004BF0023836000EB830393ED047A036801
:1004580070EE277A9A42C0ED037A77EEC77AC0ED3C
:10046800037A0CDA013307EE103AF8EEC76AB7EEF2
:10047800007A87EEA60A036030EE070A704707EE97
:10048800102AB8EEC77A87EE870A704790ED057A8A
:1004980090ED004AD0ED066AD0ED014AD0ED047A1D
:1004A80090ED035AD0ED025AA4EE007AB0EE406AFD
:1004B800B0EE470AB0EE667AA6EE247A67EEC07A06
:1004C800A0EE457AE6EE257A80ED057AC0ED067A4B
:1004D8007047D0ED057A90ED013AD0ED003AD0EDB5
:1004E800064A90ED024A90ED077A90ED035A90ED96
:1004F800086AD0ED045AC0ED067AF0EE406A27EE9D
:10050800830AC0ED056AA3EEA60A80ED087AA4EE78
:10051800240AA5EE470AA5EEC60A80ED070A704729
:10052800D0ED007A90ED017A30EE670AE7EE007AB6
:10053800B0EE670AC0ED007A704770470A449142EE
:1005480014D030B40139551E41F2210211F8014F7F
:10055800082380EA042004044CBF82EA40004000DB
:10056800013B80B2F7D18D42F0D130BC70474FF4D7
:100578000063838270474FF400638382704750F8AA
:10058800043C012280F84520103803B11847704711
:1005980070B5044682B01430E56D06236A464321DF
:1005A800A847B0B19DF804009DF800609DF80110BF
:1005B8009DF802509DF803209DF8053041EA062178
:1005C80043EA002342EA0522A187E287A4F84030E3
:1005D800012002B070BD70B5044682B00830656A6B
:1005E80006236A463B21A847A8B19DF804009DF858
:1005F80000609DF801109DF802509DF803209DF8B9
:10060800053041EA062143EA002342EA0522E18255
:1006180022836383012002B070BD70B40468037B39
:100628002268022101FA03F31A4213D042690A49E7
:10063800582000FB02124FF6FE7650685289C568B2
:100648000068296831402960C168D24392B20A40E3
:10065800C260636070BC70474862002030B4094BC8
:100668001C7864B1084B002503EBC4041A68998808
:100678005562D06808330143A342D160F6D130BC3B
:10068800704700BF086500200C65002010B40268A0
:10069800047B11680223A340194209D00649406827
:1006A80000240C7001684FF6FE742140016053600D
:1006B8005DF8044B704700BF8A6C002010B50446F3
:1006C800C06CA160036823F001030360A37986B0BE
:1006D80013F00402009141D04FF4805213F002034A
:1006E800019244D102934FF4806362790393D10756
:1006F8004FF000030493059345BF04230493082394
:100708000C236946920748BF049326F0C9FE607916
:10071800E36CA17900F00202002A15BF4FF44032C1
:100728004FF480324FF40034002410F0010F586861
:1007380008BF2246CC074CBF024320EA02025A6097
:100748009A6809074CBF42F0080222F008029A6032
:100758001A6842F001021A6006B010BD13F00203D5
:10076800019207D04FF4005113460291BDE74FF4B0
:100778000053B7E70293B8E72DE9F3410569064648
:100788000F467DBBD0F80080C8F30A0323B30023CB
:10079800D6F8008001931DF077FB042819D1224C6C
:1007A800236943F001032361BBB2A8F800301DF0B0
:1007B8006BFB04282ED108F102030193019B3F0C27
:1007C8001F801DF061FB2369042823F001032361C6
:1007D80025D06FF0010505E01DF056FB042805D073
:1007E8004FF0FF35284602B0BDE8F0810E4C236972
:1007F80043F002032361C4F81480236943F04003E3
:1008080023611DF041FB2369042823F002032361BF
:10081800BDD0E5E7236923F001032361D9E73368F5
:1008280004333360DEE700BF00200240F8B5044619
:100838000D468E180027B54201D12069F8BDE3683E
:10084800591CE160234415F8012B1A720429F2D1CE
:10085800A1682046FFF790FFE7602061EBE770B5DD
:1008680082B004466946143028F0E0F9B0B19DF82A
:1008780005009DF801609DF802109DF803509DF851
:1008880004209DF8063041EA062143EA002342EAA3
:100898000522A187E287A4F84030012002B070BD8C
:1008A80010B490E80600047B40690223A3404B6023
:1008B80013685DF8044B4FF6FE710B4013600CF0A3
:1008C800D7BA03685B6A03B11847704703681B6AA5
:1008D80003B11847704703682DE9F041DF691FB17C
:1008E8003B46BDE8F0411847002A164611DD04468C
:1008F8000D460E4400E023689B6820469847002870
:10090800F9D0236815F8011B1B6820469847AE42AA
:10091800F1D1BDE8F08103689B69184703685B69FA
:1009280018470368DB68184703689B68184703681B
:100938005B68184703681B681847014B1868F9E794
:10094800CC5E0020054B53F8203033B11A689B88E1
:10095800918A0B4218BF1B049361704750650020B1
:1009680003682DE9F04F03F13845644EAD0A0124C0
:10097800755D05F01F066D09022D04FA06F400F0F6
:10098800A280032D00F0A480012D52D08088B0FAF7
:1009980080F4C4F11F04A4B2E50803EB850504F054
:1009A80007042E6AA4000F27A74026EA07062E622E
:1009B8002E6A01F0030702FA04F47A1E3443012A6E
:1009C800C1F3810CC1F300182C62C1F3411135D970
:1009D800C60700F19780850700F1A380440700F15E
:1009E800B180020700F1BF80C60600F1CD80850600
:1009F80000F1DB80440600F1E980020600F1F7808F
:100A0800C60500F10581850500F11381440500F153
:100A18002181020500F12F81C60400F13D81850482
:100A280000F14B81440400F15981020455D4BDE81A
:100A3800F08F334D6E6934436C61A7E7002422467A
:100A48004FF0010E4FF0030904E00132102A04F1BF
:100A58000204ECD00EFA02F636EA0005F5D1D3F816
:100A680008A009FA04F5ED430AEA050AC3F808A044
:100A7800D3F808B00CFA04FA4AEA0B0AC3F808A03B
:100A8800B3F804A01FFA8AFA2AEA06069E80B3F889
:100A980004A008FA02F646EA0A06B6B29E801E6864
:100AA8002E401E60D3F800A007FA04F646EA0A06AC
:100AB8001E60D3F80CA001FA04F605EA0A0A46EA11
:100AC8000A05DD60C1E70E4DAE693443AC615DE7F0
:100AD8000B4DEE693443EC6158E71A6822F0404246
:100AE8001A601A6842EA87771F60DA6822F0404283
:100AF80042EA8171D960BDE8F08F00BF2801030880
:100B0800001002401A6822F003021A601A683A4379
:100B18001A60DA6822F003020A438507DA607FF573
:100B28005DAF1A6822F00C021A601A6842EA87025E
:100B38001A60DA6822F00C0242EA81024407DA609D
:100B48007FF54FAF1A6822F030021A601A6842EA3D
:100B580007121A60DA6822F0300242EA0112DA60FB
:100B680002077FF541AF1A6822F0C0021A601A68BE
:100B780042EA87121A60DA6822F0C00242EA811259
:100B8800C606DA607FF533AF1A6822F440721A603D
:100B98001A6842EA07221A60DA6822F4407242EAC6
:100BA80001228506DA607FF525AF1A6822F44062D3
:100BB8001A601A6842EA87221A60DA6822F44062E8
:100BC80042EA81224406DA607FF517AF1A6822F4F8
:100BD80040521A601A6842EA07321A60DA6822F448
:100BE800405242EA0132DA6002067FF509AF1A681C
:100BF80022F440421A601A6842EA87321A60DA68B8
:100C080022F4404242EA8132C605DA607FF5FBAE43
:100C18001A6822F440321A601A6842EA07421A60D7
:100C2800DA6822F4403242EA01428505DA607FF54B
:100C3800EDAE1A6822F440221A601A6842EA874226
:100C48001A60DA6822F4402242EA81424405DA60F6
:100C58007FF5DFAE1A6822F440121A601A6842EA79
:100C680007521A60DA6822F4401242EA0152DA6046
:100C780002057FF5D1AE1A6822F440021A601A689C
:100C880042EA87521A60DA6822F4400242EA815244
:100C9800C604DA607FF5C3AE1A6822F040721A60A3
:100CA8001A6842EA07621A60DA6822F0407242EA79
:100CB80001628504DA607FF5B5AE1A6822F04062F9
:100CC8001A601A6842EA87621A60DA6822F040629B
:100CD80042EA81624404DA607FF5A7AE1A6822F01E
:100CE80040521A601A6842EA07721A60DA6822F0FB
:100CF800405242EA0172DA6097E6036803F138422B
:100D08002DE9F04F920A584DAA5C02F01F055209CE
:100D18000124022A04FA05F400F08C80032A00F06A
:100D28008E80012A3CD001F003077A1E012AC1F304
:100D3800810CC1F300188088C1F3411135D9C60769
:100D480000F19680850700F1A280440700F1B08089
:100D5800020700F1BE80C60600F1CC80850600F1CE
:100D6800DA80440600F1E880020600F1F680C60544
:100D780000F10481850500F11281440500F120810C
:100D8800020500F12E81C60400F13C81850400F1C2
:100D98004A81440400F15881020455D4BDE8F08F1B
:100DA800324A55692C435461BDE7002422464FF06E
:100DB800010E4FF0030904E00132102A04F1020485
:100DC800ECD00EFA02F636EA0005F5D1D3F808A001
:100DD80009FA04F5ED430AEA050AC3F808A0D3F8AE
:100DE80008B00CFA04FA4AEA0B0AC3F808A0B3F8E8
:100DF80004A01FFA8AFA2AEA06069E80B3F804A01D
:100E080008FA02F646EA0A06B6B29E801E682E4026
:100E18001E60D3F800A007FA04F646EA0A061E6028
:100E2800D3F80CA001FA04F605EA0A0A46EA0A050C
:100E3800DD60C1E70D4A95692C43946173E70B4A5D
:100E4800D5692C43D4616EE71A6822F040421A60D3
:100E58001A6842EA87771F60DA6822F0404242EA5D
:100E68008171D960BDE8F08F2801030800100240A5
:100E78001A6822F003021A601A683A431A60DA689C
:100E880022F003020A438507DA607FF55EAF1A682D
:100E980022F00C021A601A6842EA87021A60DA68BD
:100EA80022F00C0242EA81024407DA607FF550AF73
:100EB8001A6822F030021A601A6842EA07121A60A9
:100EC800DA6822F0300242EA0112DA6002077FF59E
:100ED80042AF1A6822F0C0021A601A6842EA871202
:100EE8001A60DA6822F0C00242EA8112C606DA60A5
:100EF8007FF534AF1A6822F440721A601A6842EA21
:100F080007221A60DA6822F4407242EA0122850652
:100F1800DA607FF526AF1A6822F440621A601A6810
:100F280042EA87221A60DA6822F4406242EA8122A1
:100F38004406DA607FF518AF1A6822F440521A6046
:100F48001A6842EA07321A60DA6822F4405242EA22
:100F58000132DA6002067FF50AAF1A6822F44042CD
:100F68001A601A6842EA87321A60DA6822F4404244
:100F780042EA8132C605DA607FF5FCAE1A6822F4CF
:100F880040321A601A6842EA07421A60DA6822F4A4
:100F9800403242EA01428505DA607FF5EEAE1A6812
:100FA80022F440221A601A6842EA87421A60DA6814
:100FB80022F4402242EA81424405DA607FF5E0AE3D
:100FC8001A6822F440121A601A6842EA07521A6034
:100FD800DA6822F4401242EA0152DA6002057FF52B
:100FE800D2AE1A6822F440021A601A6842EA87529E
:100FF8001A60DA6822F4400242EA8152C604DA60D2
:101008007FF5C4AE1A6822F040721A601A6842EA84
:1010180007621A60DA6822F0407242EA01628504C7
:10102800DA607FF5B6AE1A6822F040621A601A6874
:1010380042EA87621A60DA6822F0406242EA816214
:101048004404DA607FF5A8AE1A6822F040521A60AC
:101058001A6842EA07721A60DA6822F0405242EAD5
:101068000172DA6098E610B50409013C052C17D81E
:101078000C4B33F8142000F00F0042FA00F313F081
:1010880001030DD0012303FA00F0013810402AF0C3
:10109800CFFA054A054B125D104403EBC00010BDA2
:1010A800002010BD1401030820010308306000204F
:1010B8002DE9F04F4A484B4B4B4C4FF090414FF0C5
:1010C800010A4FF002094FF004084FF0080C4FF0E6
:1010D800100E20274026802530F8022B12F0010F31
:1010E80003D01960A3F804A0083312F0020F03D04C
:1010F8001960A3F80490083312F0040F03D01960A4
:10110800A3F80480083312F0080F03D01960A3F87D
:1011180004C0083312F0100F03D01960A3F804E0DC
:10112800083312F0200F02D019609F80083312F0A4
:10113800400F02D019609E80083312F0800F02D051
:1011480019609D80083312F4807F05D04FF4807BAE
:101158001960A3F804B0083312F4007F05D04FF4E7
:10116800007B1960A3F804B0083312F4806F05D02F
:101178004FF4806B1960A3F804B0083312F4006FC1
:1011880005D04FF4006B1960A3F804B0083312F4CB
:10119800805F05D04FF4805B1960A3F804B0083372
:1011A80012F4005F05D04FF4005B1960A3F804B097
:1011B800083312F4804F05D04FF4804B1960A3F820
:1011C80004B00833D20B04D04FF4004219609A805F
:1011D800083301F58061A1427FF47EAFBDE8F08F4E
:1011E800140103083060002000180048002867D068
:1011F80003682DE9F04F03F138445C4EA40A012539
:10120800345D04F01F066409022C05FA06F558D06F
:10121800032C00F0A580012C58D08088B0FA80F407
:10122800C4F11F04A4B2E50803EB850504F0070424
:101238002E6AA4000F27A74026EA07062E622E6A08
:1012480001F00307A2407C1E3243012CC1F3810C3C
:10125800C1F300182A62C1F341113CD9C60700F155
:101268008980850700F19580440700F1A380020773
:1012780000F1B180C60600F1BF80850600F1CD807F
:10128800440600F1DB80020600F1E980C60500F1A2
:10129800F780850500F10581440500F113810205F9
:1012A80000F12181C60400F12F81850400F13D8100
:1012B800440400F14B81020400F15981BDE8F08F2C
:1012C80070472B4CA6693543A561A6E7284C66698B
:1012D80035436561A1E7002422464FF0010E4FF027
:1012E800030904E00132102A04F10204E6D00EFAE0
:1012F80002F636EA0005F5D1D3F808A009FA04F594
:10130800ED430AEA050AC3F808A0D3F808B00CFAB6
:1013180004FA4AEA0B0AC3F808A0B3F804A01FFAB3
:101328008AFA2AEA06069E80B3F804A008FA02F6AA
:1013380046EA0A06B6B29E801E682E401E60D3F8A2
:1013480000A007FA04F646EA0A061E60D3F80CA0C5
:1013580001FA04F605EA0A0A46EA0A05DD60C1E769
:10136800034CE6693543E56157E700BF28010308E8
:10137800001002401A6822F003021A601A683A4301
:101388001A60DA6822F003020A438507DA607FF5FB
:101398006BAF1A6822F00C021A601A6842EA8702D8
:1013A8001A60DA6822F00C0242EA81024407DA6025
:1013B8007FF55DAF1A6822F030021A601A6842EAB7
:1013C80007121A60DA6822F0300242EA0112DA6083
:1013D80002077FF54FAF1A6822F0C0021A601A6838
:1013E80042EA87121A60DA6822F0C00242EA8112E1
:1013F800C606DA607FF541AF1A6822F440721A60B7
:101408001A6842EA07221A60DA6822F4407242EA4D
:1014180001228506DA607FF533AF1A6822F440624C
:101428001A601A6842EA87221A60DA6822F440626F
:1014380042EA81224406DA607FF525AF1A6822F471
:1014480040521A601A6842EA07321A60DA6822F4CF
:10145800405242EA0132DA6002067FF517AF1A6895
:1014680022F440421A601A6842EA87321A60DA683F
:1014780022F4404242EA8132C605DA607FF509AFBC
:101488001A6822F440321A601A6842EA07421A605F
:10149800DA6822F4403242EA01428505DA607FF5D3
:1014A800FBAE1A6822F440221A601A6842EA8742A0
:1014B8001A60DA6822F4402242EA81424405DA607E
:1014C8007FF5EDAE1A6822F440121A601A6842EAF3
:1014D80007521A60DA6822F4401242EA0152DA60CE
:1014E80002057FF5DFAE1A6822F440021A601A6816
:1014F80042EA87521A60DA6822F4400242EA8152CC
:10150800C604DA607FF5D1AE1A6822F040721A601C
:101518001A6842EA07621A60DA6822F0407242EA00
:1015280001628504DA607FF5C3AE1A6822F0406272
:101538001A601A6842EA87621A60DA6822F0406222
:1015480042EA81624404DA607FF5B5AE1A6822F097
:1015580040521A601A6842EA07721A60DA6822F082
:10156800405242EA0172DA6002047FF5A7AE1A68B7
:1015780022F040421A601A6842EA87771F60DA68E8
:1015880022F0404242EA8171D960BDE8F08F00281C
:1015980052D0036803F138422DE9F04F920A514DB9
:1015A800AA5C02F01F0552090124022A04FA05F474
:1015B80043D0032A00F09080012A43D001F00307AA
:1015C8007A1E012AC1F3810CC1F300188088C1F387
:1015D80041113CD9C60700F18980850700F1958043
:1015E800440700F1A380020700F1B180C60600F1AC
:1015F800BF80850600F1CD80440600F1DB8002063D
:1016080000F1E980C60500F1F780850500F1058144
:10161800440500F11381020500F12181C60400F19F
:101628002F81850400F13D81440400F14B810204BF
:1016380000F15981BDE8F08F70472B4A95692C431A
:101648009461BBE7284A55692C435461B6E70024E6
:1016580022464FF0010E4FF0030904E00132102A30
:1016680004F10204E6D00EFA02F636EA0005F5D1D6
:10167800D3F808A009FA04F5ED430AEA050AC3F805
:1016880008A0D3F808B00CFA04FA4AEA0B0AC3F81F
:1016980008A0B3F804A01FFA8AFA2AEA06069E8070
:1016A800B3F804A008FA02F646EA0A06B6B29E8023
:1016B8001E682E401E60D3F800A007FA04F646EA1A
:1016C8000A061E60D3F80CA001FA04F605EA0A0A15
:1016D80046EA0A05DD60C1E7034AD5692C43D461AF
:1016E8006CE700BF28010308001002401A6822F0C6
:1016F80003021A601A683A431A60DA6822F0030291
:101708000A438507DA607FF56BAF1A6822F00C028E
:101718001A601A6842EA87021A60DA6822F00C0234
:1017280042EA81024407DA607FF55DAF1A6822F069
:1017380030021A601A6842EA07121A60DA6822F060
:10174800300242EA0112DA6002077FF54FAF1A68E9
:1017580022F0C0021A601A6842EA87121A60DA6830
:1017680022F0C00242EA8112C606DA607FF541AF74
:101778001A6822F440721A601A6842EA07221A604C
:10178800DA6822F4407242EA01228506DA607FF5BF
:1017980033AF1A6822F440621A601A6842EA872254
:1017A8001A60DA6822F4406242EA81224406DA606A
:1017B8007FF525AF1A6822F440521A601A6842EA87
:1017C80007321A60DA6822F4405242EA0132DA60DB
:1017D80002067FF517AF1A6822F440421A601A68A9
:1017E80042EA87321A60DA6822F4404242EA8132D9
:1017F800C605DA607FF509AF1A6822F440321A602C
:101808001A6842EA07421A60DA6822F4403242EA69
:1018180001428505DA607FF5FBAE1A6822F44022A2
:101828001A601A6842EA87421A60DA6822F440228B
:1018380042EA81424405DA607FF5EDAE1A6822F487
:1018480040121A601A6842EA07521A60DA6822F4EB
:10185800401242EA0152DA6002057FF5DFAE1A68EB
:1018680022F440021A601A6842EA87521A60DA685B
:1018780022F4400242EA8152C604DA607FF5D1AE12
:101888001A6822F040721A601A6842EA07621A60FF
:10189800DA6822F0407242EA01628504DA607FF574
:1018A800C3AE1A6822F040621A601A6842EA876278
:1018B8001A60DA6822F0406242EA81624404DA601F
:1018C8007FF5B5AE1A6822F040521A601A6842EAEB
:1018D80007721A60DA6822F0405242EA0172DA604E
:1018E80002047FF5A7AE1A6822F040421A601A680F
:1018F80042EA87771F60DA6822F0404242EA817143
:10190800D960BDE8F08F10B1036882881A857047E6
:1019180010B1036882889A61704738B100298388BA
:10192800026814BF002110218B409361704710B4E6
:101938000A4B0B4A1C7801238340234052F82000AD
:1019480029B9B3FA83F149095DF8044BE5E7191C95
:1019580018BF01215DF8044BDFE700BF4D6500208B
:101968005065002030B1036882881B8A1A4214BF70
:1019780001200020704738B5044690F85900002827
:101988005AD104F11405236E80226B21284698470A
:1019980064200BF0CFF8236E072268212846984769
:1019A80064200BF0C7F8236E00226B212846984765
:1019B80064200BF0BFF8236E01226B21284698475C
:1019C8000F200BF0B7F894F85320236E042A34BF85
:1019D80018221A221B21284698470F200BF0AAF834
:1019E800236E18221C21284698470F200BF0A2F8D6
:1019F800236E94F852201A21284698470F200BF09E
:101A080099F8236E94F854201921284698476420A1
:101A18000BF090F8236E10223721284698470F20A4
:101A28000BF088F82846236E0122382198470F20AA
:101A3800BDE838400BF07EB8FFF715FB0546FFF709
:101A480091FF014600289CD1D5B12023E871AB71E4
:101A58002846FFF79CFD21460F4B41F8103F2846CA
:101A680027F07CF8AB88B3FA83F3C3F11F035A1C41
:101A780087D001229A4009490B6813430B6080E71D
:101A88002946FFF784FD2146034B41F8103F2846BD
:101A980027F064F80122EEE78705000800040140FA
:101AA80010B504460120A269138823F040031B04E3
:101AB8001B0C138013889BB223F0380343F03003C8
:101AC800138013889BB243F0400313800AF0D8FFB9
:101AD8002046FFF750FF102204F114006A21FEF798
:101AE80095FB64200BF026F8A269138823F04003C5
:101AF8001B041B0C1380138823F038031B041B0CD6
:101B0800138013889BB243F0400313800120BDE883
:101B180010400AF0B5BF2DE9F0410B4E34687369E7
:101B28001C400FD0DFF824800127B4FA84F3C3F1F6
:101B38001F0307FA03F558F8230003689847AC43D6
:101B48007561F2D1BDE8F081000401408C68002085
:101B58002DE9F0410B4E346873691C400FD0DFF853
:101B680028800127B4FA84F3C3F11F0307FA03F5A9
:101B780058F8230003689847AC437561F2D1BDE873
:101B8800F08100BF000401408C6800202DE9F0417D
:101B98000B4E346873691C400FD0DFF8288001278A
:101BA800B4FA84F3C3F11F0307FA03F558F82300C6
:101BB80003689847AC437561F2D1BDE8F08100BF76
:101BC800000401408C6800202DE9F0410B4E346878
:101BD80073691C400FD0DFF828800127B4FA84F31A
:101BE800C3F11F0307FA03F558F823000368984761
:101BF800AC437561F2D1BDE8F08100BF000401403B
:101C08008C6800202DE9F0410B4E346873691C4044
:101C18000FD0DFF828800127B4FA84F3C3F11F033B
:101C280007FA03F558F8230003689847AC43756131
:101C3800F2D1BDE8F08100BF000401408C680020AB
:101C48002DE9F0410B4E346873691C400FD0DFF862
:101C580028800127B4FA84F3C3F11F0307FA03F5B8
:101C680058F8230003689847AC437561F2D1BDE882
:101C7800F08100BF000401408C6800202DE9F0418C
:101C88000B4E346873691C400FD0DFF82880012799
:101C9800B4FA84F3C3F11F0307FA03F558F82300D5
:101CA80003689847AC437561F2D1BDE8F08100BF85
:101CB800000401408C680020084A094808B5936967
:101CC80043F001039361002140222CF05AF8054BA0
:101CD8004FF0FF321A60C3F8032008BD001002401D
:101CE8008C680020CC6800202DE9F0410446184695
:101CF8000D461646984628F0F1FF2768E6722844F4
:101D0800A07229467D69434632462046AC46BDE866
:101D1800F0416047036810B504461B68984723687C
:101D280020469B689847A37B0133A37310BDF0B48A
:101D380084894FF6FF764FF47A740BB300292ED0BE
:101D48000F78013101E0B44217D00589013CAD0795
:101D5800A4B2F8D507734FF47A7402E0BCB2B44267
:101D68000BD00589ED0704F1FF37F7D5057BEDB2F8
:101D78000AB115700132013BDFE70A4B984202D0E5
:101D88000120F0BC7047084A538901339BB2538144
:101D9800508980B2003018BF0120F0BC7047FF277F
:101DA800D3E700BF003001405C68002070B50646EC
:101DB800806810B104688088208541F080017068CF
:101DC80040F2E93400E0F4B10589013C15F0020F56
:101DD800A4B2F8D0017300F10C0540F2E93100E03B
:101DE800D9B10489013914F0010F89B2F8D02978E2
:101DF80070680021FFF79BFFB36813B11A689B88CE
:101E08009361012070BD0A498842F2D1094C618969
:101E1800013189B261816189EBE705498842E7D1DF
:101E280004484189013189B2418141897068E0E7FC
:101E3800003001405C680020427A02B9704710B552
:101E480004460368406804F10A0198470023637256
:101E580010BD437A5A1C0344D2B242729972037A73
:101E6800934200D802B9704710B504460368406829
:101E780004F10A0198470023637210BD30B40B4D7A
:101E8800002305F10C0101E0272B0BD011F81320DA
:101E980082424FEA430403F10103F5D12C44607BED
:101EA80030BC7047002030BC704700BFF4DE020829
:101EB80070B5448806460D46C4F30B04224600213B
:101EC80028462BF05EFF3369094A934209D3094A31
:101ED800934206D2224628461946BDE8704029F0AA
:101EE800D1BC23B121462846BDE87040184770BDD3
:101EF8002C3903081C3A0308064B07498B4202D3C6
:101F08000023184670471A88C2F30B029042F8D093
:101F18001433F3E7083503082C390308024A136819
:101F280023EA00001060704714320020F8B5174DFE
:101F38002B78A32B28D16B78BE2B25D102222946DA
:101F48004FF6FF70FEF7FAFA114FAC1C22884AB11F
:101F5800A618BE4218D2052A16D92146FEF7EEFA6F
:101F68003446F3E721460222FEF7E8FA0222A118D6
:101F7800FEF7E4FA0634074B641B1C8041F60F5346
:101F8800C31A58425841F8BD0020F8BD00F00308B4
:101F980000000408B02E00202DE9F04FDFF864910E
:101FA8004F4F8BB00326A7EB09071822002104A87E
:101FB8002BF0E7FE4B4BCDF8109005971A691206E7
:101FC80004D5494A5A6002F188325A6001228DF8D4
:101FD80024203422DA60454B454C1B88ADF800308C
:101FE8000222694604A8FEF721FC022269464FF640
:101FF800FF70FEF7A3FADFF810A180464FF0000B40
:10200800544536D30AAC002524F8245D0222214623
:1020180004A8FEF70BFC022221464046FEF78EFA82
:1020280040BAC043ADF80800022202A904A8FEF78E
:10203800FDFB079860B106ABC0F1040229461844BD
:102048002BF09FFE069904A8FEF796FB07950890CB
:102058009DF82430089A23B122490B6943F0800384
:102068000B61013E2DD0002A9FD1FFF75FFF50B3CF
:1020780032E065888DF80DB0C5F30B05AB1DADF8E2
:1020880008302388C3F30B02ADF80A201B0B062285
:1020980002A904A88DF80C30FEF7C8FB062202A995
:1020A8004046FEF74BFA616880462A4604A8FEF7C8
:1020B800BDFB616840462A46FEF740FA1434804664
:1020C8009EE7002AD1D005201FF058FE094B0A4A86
:1020D8001A600A4B0A4ADA600BB0BDE8F08F00BFFD
:1020E8000000040800200240230167454EDF020873
:1020F80008350308FC9F0020EFBEADDE00ED00E0D0
:102108000400FA0500F003082C3903080378202B93
:10211800024600F10100F9D0092BF7D02D2B2CD065
:102128002B2B03BF5378B7EE000A0246B7EE000A1E
:10213800A3F13001C8B209289FED467A10D8F2EE13
:10214800046A07EE901AF8EEE77A12F8013FE7EE14
:10215800267AA3F13001C8B20928B0EE677AF0D91F
:102168002E2B4CD003F0DF03452B0BD0F7EE007A73
:1021780067EE276A20EE260A70475378BFEE000AFA
:102188000246D5E710B451782D2959D02B290ABF1A
:102198009178501C901C0024A1F13003092B53D8CE
:1021A800002303EB830301EB430310F8011FA1F1A4
:1021B8003002092AA3F13003F3D9B3F59A7F28BF77
:1021C8004FF49A73072B42D9DFED236A1A46F7EECC
:1021D800007A083A072A67EEA67AFAD803F00703C6
:1021E8002BB1F2EE046A013B67EEA67AFBD124B369
:1021F800C7EE276A5DF8044B20EE260A704753782D
:10220800A3F13001C8B2092802F10102AAD8F2EEFE
:10221800046AF0EE665A07EE901AF8EEE77A12F8BA
:10222800013F87EEA66AA3F13001C8B2092866EE1D
:10223800A56A37EE067AEED994E767EE276AD9E7FA
:10224800901C91780124A7E7F7EE007ACFE7F7EE24
:10225800007AC5E70000000020BCBE4CB5EEC00AFD
:10226800DFED317AF1EE10FACCBF30EE270A30EE0E
:10227800670ADFED2E7A20EE270A30B5FDEEC07A28
:1022880087B017EE904A054684EAE470002303A954
:10229800A0EBE4700193009302931BF0F5FF002C70
:1022A800ACBF20232D2303A88DF8003028F016FD9D
:1022B800012803A924D002282DD0032805BF3023E4
:1022C800684668468DF801302BF081FD684628F095
:1022D80005FD0338C4B22246694628462BF0D5FDD1
:1022E80000232B55284628F0F9FC2E22431C2A549B
:1022F8000DEB0401E8182BF087FD284607B030BD28
:10230800302368468DF801308DF802308DF803309F
:102318002BF05DFDDAE7302368468DF801308DF843
:1023280002302BF054FDD1E76F12033A00007A44D3
:102338002DE9F041064615460846B6FBF2F43CB9CD
:1023480005FB1464124B1B5D00F8013BBDE8F081EE
:10235800B4FBF2F767B90E4B05FB174705FB14648E
:10236800DA5D00F8012B1B5D00F8013BBDE8F08148
:10237800B7FBF2F8B8F1000F02D04046FFF7D8FFDC
:1023880005FB1878024B13F8082000F8012BE3E747
:102398007403030830B402681146531C036011F833
:1023A800024B0160D31C517803609378151D0560BA
:1023B8001B0443EA0123D078234343EA006030BC7E
:1023C80070470368591C1A46016012F8021B026024
:1023D800587841EA0020704703685A1C0260187850
:1023E800704738B504460068154629F04BFA22684C
:1023F8002A44226038BD036810B40A0A5C1C0460D1
:102408001A7003685A1C026019705DF8044B704713
:1024180003685A1C026010B4197003680A0A5C1C2D
:1024280004601A7003680A0C5C1C04601A70036864
:10243800090E5A1C026019705DF8044B7047036856
:102448005A1C026019700368090A5A1C0260197044
:1024580070472DE9F047002488B080460F461E4695
:10246800A14605AD531C0393117839B3252933D1FF
:10247800931CCDF810900393507830284ED04FF02D
:10248800000AA0F13003DBB2092B42D96C2819D01D
:10249800642800F0938024D825281CD063D95828B4
:1024A80076D063281BD131784046B847039A531C2D
:1024B80003931178043601340029D7D1204608B097
:1024C800BDE8F087039B5A1C03921B78642B7CD0D1
:1024D8002AD8252B54D1252140460134B847039AE0
:1024E800C0E7732833D044D975284FD106F1040EBC
:1024F80030682B4600220A217646FDF71BFF049A16
:102508000095534639464046FDF751FF039A044467
:10251800A8E704AA03A91BF093FEB7E7D31C03930B
:1025280090784FF0010AACE7732B10D05BD9752B6C
:102538003AD0782B96D1A3F15802B2FA82F23068D9
:1025480052092B4610210436FDF7F4FED7E733680D
:10255800049A0093394600234046FDF728FF0436C5
:102568000444039A7EE70028B9D1204608B0BDE8A4
:10257800F0876E28B3D1039A336804361C6071E77C
:102588002AD9582BD7D0632B8DD06BE77828A6D1C2
:10259800A0F15802B2FA82F2306852092B46102193
:1025A800FDF7C8FE0436AAE706F1040E30682B468C
:1025B80000220A217646FDF7BDFEA0E7331D3068EC
:1025C80029461E46FDF788FE99E7331D30682946DF
:1025D8001E46FDF781FE92E7002B7FF443AF2046AD
:1025E80008B0BDE8F0876E2BC6D03BE70EB400B547
:1025F80084B005AB019053F8042B0649039301A856
:10260800FFF727FF019B00221A7004B05DF804EB66
:1026180003B07047AD0300080FB430B583B006AB04
:102628000A490B4853F8042B096800680193FFF71F
:1026380010FF084C05462068FEF770F90028FAD00C
:10264800284603B0BDE8304004B070474C2C002049
:10265800502C0020CC5E0020DFED2B7AB4EEE70A88
:10266800F1EE10FA4ADDDFED296A9FED297A01E0E3
:10267800B0EE670AB4EEC70AF1EE10FA70EE667AA9
:10268800F6DC9FED247AF4EEC77AF1EE10FA38D52D
:10269800DFED1E6A9FED207A01E0F0EE407AF4EE5D
:1026A800C77AF1EE10FA37EEA60AF6D4DFED1B7AF8
:1026B800B4EEE70AF1EE10FA14DDDFED137A37EE27
:1026C800C00A60EE006A9FED166A9FED167ADFED8C
:1026D800167AA6EE867A20EE266AE6EE877AA6EEC7
:1026E800270A7047DFED117AB4EEE70AF1EE10FA27
:1026F80044BFDFED087A37EEC00AE2E7F0EE407A31
:10270800BFE7B0EE670AD1E7DB0F4940DB0FC940EE
:10271800E4CB1641DB0F49C0E4CB16C1DB0FC93F40
:1027280092E741B99730083C15A82ABEDB0FC9BF0C
:1027380009B909E0194690FBF1F301FB13030846B8
:10274800002BF7D1084670470146FBE710B507EEA6
:10275800901A2DED028BB8EE678ADFED217A28EE0C
:10276800008A044628EE278AB0EE480A29F04AFA79
:10277800F0EE408AB0EE480A29F0A6F9F7EE007AA2
:102788009FED187AF0EE675AE8EE875A0023A361A6
:10279800B0EE676AC7EEA56A63612362E361A8EEDB
:1027A800C76ABDEC028B77EEC07AB6EE007AF8EE17
:1027B800005A27EE877A20EE250A27EE267A26EE9B
:1027C800266A67EEA67A20EE260A84ED046AC4ED2E
:1027D800017A84ED007A84ED027A84ED030A10BD53
:1027E80027D4D236F304353F10B44C09012250F8EF
:1027F800243001F01F0102FA01F10B4340F82430A4
:102808005DF8044B70474B0901F01F0150F8232075
:10281800012303FA01F1114214BF18460020704742
:10282800F0B55B4B5B4A97B01968914200AF00F076
:10283800A3805949594A00234FF47000C1F8880011
:102848003B607B60136843F48033136003E03B68AC
:10285800B3F5A04F09D0136803F400337B603B68DD
:1028680001333B607B68002BF1D04C4B1B6813F4A1
:10287800003318BF01237B607B68012B52D0464C84
:10288800464B474AE260474A596A11605A6A42F021
:1028980080725A625A6942F4FC025A610025032286
:1028A80007F10801012341F6FF764FF09040FD60E3
:1028B800BE603A73BB7324F04FFE4FF6FF7307F107
:1028C80008013948BB6024F047FE07F10801374882
:1028D800374E24F041FE07F10801364824F03CFE4B
:1028E80007F10801344824F037FE07F1080133489E
:1028F80024F032FE07F1080024F0E4FBBB683049FD
:10290800304AA1FB031330499B0CF0204FF0070E0F
:102918005C370B60566084F823009560C2F800E0CD
:10292800BD46F0BD294A1D4B122111605A685A60F4
:102938005A685A605A6842F480625A605A6822F4A7
:102948007C125A605A6842F4E8125A601A6842F0D7
:1029580080721A601A689201FCD559680F4A21F0F2
:1029680003015960596841F002015960536803F046
:102978000C03082BFAD182E700221A6062B6144BC6
:102988001B6883F30888134B1B689847FEE700BF52
:10299800FC9F0020EFBEADDE00ED00E0001002401D
:1029A8000005FA056C4200200004004800080048B1
:1029B8003F190100000C00480010004800140048AE
:1029C80083DE1B4310E000E0886500200020024001
:1029D80000D8FF1F04D8FF1F70B50F4C0F4DC0EB78
:1029E800C00004EB8004686926693043686182B0DE
:1029F8009209667BA1600025012101A863618DF819
:102A080004608DF805208DF806508DF8071024F025
:102A180083FA02B070BD00BFF80B0020001002401E
:102A2800074BC0EBC00030B403EB8000054C0569D0
:102A380063692B4363610176427630BC704700BFFF
:102A4800F80B0020001002402DE9F04F5E4C54F8BE
:102A5800204083B0002C71D0666D984691465B4B40
:102A68007268E264A160236004F15A014FF4807334
:102A780004F5AD726161A261E36023610746307EAF
:102A880025F03CFDF068A8B1514B00215A689042EE
:102A980003F11C0300F0928001310C29F6D10020CB
:102AA8007A1CD2B20C21FFF7BBFFE36CF2682263F9
:102AB8002433A364B068D8B1454B00215A689042CA
:102AC80003F11C0378D001310C29F7D100257A1CB9
:102AD800D2B20B212846FFF7A3FF2346F27E3D49D9
:102AE8002846FFF779FFE36CB268626328336364B2
:102AF80094F85900FEF7B7FA054694F85800FEF71F
:102B0800B2FA18F0080F824696F819B01AD0CDB16B
:102B180018F0110F4FF00B0307F1010714BF4E21F6
:102B28003E21EF715A46AB712846FEF75FFB18F05D
:102B3800010F45D0236B5BB3636B4BB3204603B0E7
:102B4800BDE8F08F18F0010F0CBF4FF02E084FF0C2
:102B58004E0819F0020F09D045B10B227B1CAA714F
:102B6800EB7128465A464146FEF740FB19F0010F23
:102B7800E0D0BAF1000FDDD001370C238AF80770D6
:102B88005A4641468AF806305046FEF72FFBD1E7F1
:102B9800337FB27E8DF804209B090021012201A811
:102BA8008DF805308DF806108DF8072024F0B4F95B
:102BB800204603B0BDE8F08FCDB288E7C8B26FE712
:102BC8002846FEF7A0FEB5E7582C002050DF020883
:102BD800F80B0020A90800080348D0F83C3113B1CD
:102BE80000F59A7018477047F80B00200348D0F892
:102BF800203113B100F58C7018477047F80B00208E
:102C08000348D0F804310BB1FC301847704700BFB7
:102C1800F80B00200348D0F8E8300BB1E030184733
:102C2800704700BFF80B00200348D0F8CC300BB138
:102C3800C4301847704700BFF80B00200348D0F88D
:102C4800B0300BB1A8301847704700BFF80B002010
:102C58000348D0F894300BB18C301847704700BF48
:102C6800F80B00200248836F0BB17030184770478B
:102C7800F80B00200248C36D0BB154301847704759
:102C8800F80B00200248036C0BB138301847704726
:102C9800F80B00200248436A0BB11C3018477047F4
:102CA800F80B00200248836803B11847704700BF3B
:102CB800F80B00201749184B184A194810B4D1F8D6
:102CC800884044F47004C1F888401C6844F001044A
:102CD8001C605C6822405A601A6822F0847222F4F0
:102CE80080321A601A6822F480221A605A6822F424
:102CF800FE025A60DA6A22F00F02DA621A6B0024C6
:102D080010404FF0006218639C608A605DF8044BC5
:102D1800704700BF00ED00E0001002400CC07FF8D3
:102D2800CCFC00FF2DE9F04F2DED028B93B08346CC
:102D380022F05EFBB54B1D7825B113B0BDEC028BBC
:102D4800BDE8F08FB24B1B685C05F6D5B14FB24EAB
:102D58003B68002B56D0B14C3168D4F810218A1A40
:102D68007C2A4FD994F81421DFF8FC829FEDAC8AB5
:102D7800C4F81011013284F814214FF0240A5E209F
:102D8800984750463B689847A64BF8EC016A9B8ADF
:102D980007EE103AF8EEE66AB8EEC77A0AF1010AC9
:102DA800C6EE877A5FFA8AFA67EE887AFDEEE77AE6
:102DB800CDED027ABDF908905FFA89F022F086FA23
:102DC800C9F3072022F082FABAF1270F3B68D6D15F
:102DD8005E2098473B6830209847002022F076FA1A
:102DE800002022F073FA3B685E20984794F814316B
:102DF80013F0030800F08481580701F03682282B6D
:102E080001F03283884B1B78002B72D0834C874AA1
:102E1800D4F81831ABEB0303934200F27B8794F8A4
:102E28002091B9F1000F35D1DFF84082D8F80000C1
:102E3800FDF77DFDC0B201280FD902287C4F41F073
:102E4800A5833B78002B41F02A86D4F82431ABEBDC
:102E58000303B3F57A6F81F09D87D4F82831002BEE
:102E680047D094F82031C3B9724B1B689B78012175
:102E78001E3B00228B4284F8201184F8342141F251
:102E88002E87D8F800000221043022F097F994F830
:102E98002C3111E0D4F828315BB3D4F8303140F646
:102EA800B732ABEB0303934223D994F82C31002BB0
:102EB80001F0C382DFF8B481013BDBB284F82C3126
:102EC800002B00F08287D4F8287194F8342117F881
:102ED800011B94F83531D8F80000C4F828710A4469
:102EE800013384F8342184F83531FDF723FDC4F823
:102EF80030B1514BD6F800801B7843B14F4F38683A
:102F080028B14F4B1B78013B012B40F26E874D4B8C
:102F18001B7863B14C4F3B684BB1404CD6F80090DE
:102F2800D4F84C31A9EB0303632B00F21C81DFF8C2
:102F3800408198F80030022B01F05E823C4F97F8F0
:102F48007430032B00F02B87404B1B7873B1404D36
:102F58002B685BB1314C09F047FDD4F85831029029
:102F680044F61F62C31A934200F25881394B1B780A
:102F7800002B7FD1384B1B7843B1284CD4F8A832AA
:102F880003F5C333A0339B4580F07286334B1B781F
:102F9800002B3FF4D2AE214E314C324D06F2C927F8
:102FA8002068FDF7C4FC00283FF4C7AE2068FDF791
:102FB800B8FC2B7880465A1E33B120682A70FDF77A
:102FC800B6FC0028F2D1B8E603223946781E2AF06A
:102FD800BEFE96F8C83296F8C92286F8CB8283F4EA
:102FE8007F4383F0FF039B1A1FFA88F89BB2B8EB64
:102FF800132FD5D196F8CA22DBB29A42D0D1781EC7
:1030080019F0A6FC2B7818442870C9E7D66C002064
:1030180030550020B45B002084650020DC1D0020B2
:1030280000007A44BC330020465C00203F0D0300BA
:1030380000000020B05B0020485C0020FC59002004
:10304800505C0020585C0020204B0020605C002071
:10305800645C0020A45C0020B55C00206A5C002051
:10306800705C0020745C0020F4330020AC5B00200E
:10307800F25800205B4C2278A2B15B4B9B7A53B18B
:1030880009F0B2FC594B1B68C31AA3F57A73B3F560
:10309800FA6F07D82278564B56491868FDF71BFC7B
:1030A80000232370544CD4F8A03203F5C333A03363
:1030B8009B45FFF45FAF514DC4F8A0B22B78002BAD
:1030C80041F030834E4D2B78002B41F01D824D4945
:1030D80094F8A4228D5CE90701F1E784AA0701F1BD
:1030E800A1846B0701F19983474A94F8A4321178B7
:1030F800013393FBF1F201FB123384F8A43239E770
:10310800D4F8102141F288339A4201F216823B68C2
:103118005E2098473B68142098473C4B3C4AB3F9DB
:10312800043082FB03124FEAE378C8EBA2080FFAD7
:1031380088F85FFA88F022F0C9F8C8F3072022F06F
:10314800C5F83B685E2098473B681C2098470020DC
:1031580022F0BCF8002022F0B9F83B685E209847BE
:1031680094F8143148E6DFF8A4A0DFF8A4804120E1
:1031780021F0D2FFBAF9023088FB0320DB17C3EB3A
:10318800A00080B221F0AEFFBAF9003088FB03201E
:10319800DB17C3EBA00080B221F0A4FFBAF904301A
:1031A80088FB0320DB17C3EBA00080B221F09AFF55
:1031B800184B38681978FDF7BDFB94F8503113F0B7
:1031C800010801F0F481144AC4F84C910133DBB2D0
:1031D800A2FB0312D20802EB8202A3EB420384F89B
:1031E8005031A4E6385C00204042002034390020E9
:1031F800A85C0020F85B0020DC1D0020AC5C0020EF
:10320800AD5C0020B05C0020B45C0020245000209D
:1032180067666666EC4E0020CDCCCCCC94F85E3167
:10322800002B41F06C81DB4B1A6802F00803002B7D
:1032380048F603414AF60B404BF60F4349F6074759
:1032480004BF03460F4612F0040F4FF0190118BFD0
:103258001F46920684F85E1103D547F4804747F06D
:103268002007CD4B5A79C7F30909002A41F0BF85D9
:103278009B79002B41F0AA86984664204FF0FF3ACC
:103288004FF0000C0A970B97ADF834C0CDF83AC050
:10329800CDF83EC0CDF842C0CDF83090ADF83680BC
:1032A800ADF838A08DF846000AAF0FCFDFF800E37D
:1032B80084F805C0AEE80F0097E80F00AEE80700F5
:1032C8002EF8023B71464FF0010C1B0CFE271F2005
:1032D800C82201F81E39A770A27184F807C0E070EF
:1032E80094F86E01207180F0F10383EA0313DAB2D7
:1032F800130983F0E70343EA022383EAC2031BB2FC
:1033080083EA0312D2B2C3F3072383EA121343EA10
:10331800022383EAC2031BB283F0C80282EA0212C4
:10332800D2B2C3F3072383EA121343EA022383EAE0
:10333800C2031BB283EA0C0787EA0717FFB2C3F37D
:10334800072282EA171242EA072200EB0C0382EAFC
:10335800C7070EEB0C0084F86E31278011F8013B8B
:103368007B4083EA0313DBB21A0982EA172242EA96
:10337800032282EAC3031BB29FB281422780EDD1A8
:1033880083F07C0383EA0313DBB24FEA131E8EEA51
:10339800172E8EEA032E8EEAC30E0FFA8EFE1FFA40
:1033A8008EFADFF810C2A4F800A05FFA8EFE4FEA8A
:1033B8001A2A84F828A084F827E00CF5CB7804F1C1
:1033C8002209DCF80000DCF80410DCF80820DCF83E
:1033D8000C3047460FC70CF1100CCC45B846F0D15D
:1033E800DCF8000038606D4F9CF8043088F8043031
:1033F80007F1270884F8BDE184F8BEA117F8011F7A
:103408002868FDF797FAB845F8D194F85F31002B92
:1034180041F070806249326809780A2084F85F01B7
:10342800002901F0F0815F4F01293888069041F2A8
:10343800C1850229B7F802E001F0F484B888059044
:10344800032901F0CE85F8880490042901F0DC8571
:103458000529388901F0D3850629B7F80A9001F0C3
:10346800CA850729B7F80C8001F0C285FB89039348
:1034780094F86E110A920B4683F0300282EA021227
:10348800D2B217094849079387F07A0747EA022713
:103498000988237187EAC202444FC1EB012187FBE7
:1034A800013A069B4FF0000C63F30F0C059B6EF37B
:1034B8001F4C4FF0000E63F30F0E049BCDF82CC089
:1034C80012B28A440027C91763F31F4EC1EB6A2A58
:1034D800039BCDF830E082EA021160F30F07002069
:1034E800C9B268F30F00C2F3072269F31F4782EAE3
:1034F800111263F31F404FF000090D978DF83DA09E
:103508000E908DF83C9042EA01220DF1280C82EAD7
:10351800C107BCE80F003FB287F0C80888EA08185E
:10352800DFF88CE084F805905FFA88F8C7F307277E
:10353800AEE80F0087EA181747EA08239CE803005B
:1035480083EAC8031BB283F023024EF8040B82EA15
:103558000212D2B2C3F30723079F83EA12137046FD
:1035680043EA022383EAC20207F1010C20F8141986
:103578004FF023081621FE27C82384F86EC1228045
:1035880084F807800EF1020EA770E170A37111464E
:1035980012E000BF043600204C6C0020731F00208E
:1035A800D4380020AC6C0020446C00200308208034
:1035B800E41D0020DE1D002010F8013B4B4083EA8B
:1035C8000313DBB21A0982EA112242EA032282EAD1
:1035D800C3031BB299B270452180EDD183F0F40387
:1035E80083EA0313DBB24FEA131E8EEA112E8EEA2A
:1035F800032E8EEAC30E0FFA8EFE1FFA8EF8E64FE0
:10360800A4F800804FEA182C5FFA8EFE84F81EE0BA
:1036180084F81FC07968BA683868FB6807F5CB7802
:10362800A8E80F0038697969BA6904F29717A8E819
:10363800070004F2B51884F8B5C184F8B4E117F8A6
:10364800011F2868FDF776F9B845F8D194F866C1E6
:10365800BCF1000F40F04887D04B94F86E71B3F975
:103668000010B3F90220B3F904309FEDCD6ADFF8FA
:1036780040E384F805C007EE103A33680A9387F0F0
:103688006A0383EA031306EE901AD9B20B0983F092
:10369800D50343EA012383EAC1031BB283EA03117A
:1036A8005242C9B207EE902AC3F3072383EA1113E3
:1036B80043EA0123F8EEE77AF8EEE66AB8EEC77A4D
:1036C80083EAC1031BB267EE867A66EE866A27EE46
:1036D800067A002083F0C808CDED0C7ACDED0B6A90
:1036E8008DED0D7A0E900F90109088EA08160DF166
:1036F8002809F6B2C3F30728B9E80F0088EA1618B4
:1037080048EA062888EAC6080FFA88F8AEE80F00E3
:1037180088F01E0699E8070086EA0616F6B2C8F38E
:10372800072383EA161343EA06238EE8070083EA91
:10373800C6061C20C8214FF005084FF01E0CFE23BA
:103748007A1CE070A17184F8668184F807C0A370C0
:10375800AEF1100127710EF10C00268084F86E215D
:1037680011F8013B734083EA0313DBB21A0982EABA
:10377800162242EA032282EAC3031BB29EB28142A6
:103788002680EDD183F0270383EA0313DBB24FEAE7
:10379800131E8EEA162E8EEA032E8EEAC30E0FFA39
:1037A8008EFE1FFA8EFC7C4FA4F800C05FFA8EFED6
:1037B8004FEA1C2C84F825C084F824E007F5CB7860
:1037C80004F1220938687968BA68FB6846460FC66A
:1037D80010374F45B046F5D1724E3B88A8F80030F7
:1037E80006F1240784F8BAE184F8BBC116F8011F72
:1037F8002868FDF79FF8B742F8D194F867A1BAF1A5
:10380800000F40F06B8694F86E81644B664AB3F9FA
:103818000410B2F90620654EDFF898E1644F84F889
:1038280005A088F0220080EA0010C0B2030983F0E6
:10383800590343EA002383EAC0031BB2B2F5FA6FC7
:1038480083EA0310C0B2A8BF4FF4FA62C3F3072398
:10385800B2F57A7F83EA101343EA0023B8BF4FF426
:103868007A7283EAC000A2F57A72642303FB02F23B
:103878008EFB023ED31786FB0162C9174FF0000C7E
:10388800C3EBAE13C1EBA201CDF828C006B2CDF848
:103898002CC0CDF830C0CDF834C0ADF83A30ADF812
:1038A80038100DF1280CBCE80F0086F0C80E8EEA1F
:1038B8000E1E5FFA8EFEC6F3072686EA1E1646EA35
:1038C8000E260FC786EACE0636B286F04A0383EA8A
:1038D8000313DBB2C6F3072181EA13113A46DCF879
:1038E80000E042F810E941EA032108F1010681EA03
:1038F800C30305204A214FF0FE0C84F86E614FF097
:10390800C80E142684F8670184F8048023800437DD
:10391800E17184F802C0E67084F806E0184612F8EF
:10392800011B414081EA0111C9B20B0983EA102346
:1039380043EA012383EAC10109B288B2BA4220806E
:10394800EDD181F0140181EA0111C9B24FEA111ECB
:103958008EEA102E8EEA012E8EEAC10E0FFA8EFE26
:103968001FFA8EF60C4F26804FEA16295FFA8EFE54
:1039780084F81D9084F81CE079683868BA68FB6898
:10398800B7F8188007F5CB7CACE80F00386979697F
:10399800ACE8030010E000BFDE1D0020245000202A
:1039A80088C3E43A731F0020AC6C00206766666623
:1039B800E41D0020D34D621004F29716ACF8008085
:1039C80084F8B391B04684F8B2E104F2B31918F858
:1039D800011F2868FCF7AEFFC145F8D1C44BC54AA2
:1039E8001B781278013B12F00100DBB214BFC02132
:1039F8004021172B03D8C04A134493F830A0BF4B7B
:103A08001A8893071ABF002341F01001012312F40A
:103A1800027F18BF022312F0100F18BF062312F0FE
:103A2800200F18BF1023002841F08C814FF0030CA1
:103A380094F86E910A9389F0460383EA0313DAB285
:103A4800130983F0920343EA022383EAC2031BB2F9
:103A580083EA0310C0B2C3F3072282EA101242EAD3
:103A6800002282EAC00212B282F0C80E8EEA0E1E4E
:103A78005FFA8EFEC2F30722002382EA1E12032099
:103A88008DF82CA08DF82FC08DF82D3042EA0E2C21
:103A98008DF82E108DF830000AAA07CA8CEACE0ECF
:103AA8000FFA8EFEDFF868A2E3718EEA0E1CAAE810
:103AB80003005FFA8CFCCEF3072E8EEA1C1E4EEA3A
:103AC8000C2181EACC0C94F808E08AF800200FFA5F
:103AD8008CFC8EEA0C0E8EEA0E1E5FFA8EFECCF37C
:103AE800072282EA1E1242EA0E22607AA17A94F82C
:103AF8000BC0637182EACE0212B2504080EA001E07
:103B08005FFA8EFEC2F3072080EA1E1040EA0E20FC
:103B180080EACE0000B2414081EA0111C9B2C0F387
:103B2800072282EA111242EA012282EAC10212B293
:103B38008CEA020C8CEA0C1C5FFA8CFCC2F307229C
:103B480082EA1C1242EA0C2294F80CE0607BA17B0A
:103B580094F8108084F8049082EACC0212B28EEABB
:103B6800020E8EEA0E1E5FFA8EFEC2F3072282EA6A
:103B78001E1242EA0E2282EACE0212B2504080EAB7
:103B88000010C0B2C2F3072282EA101242EA0022F1
:103B980082EAC00212B2514081EA0111C9B2C2F3ED
:103BA800072282EA111242EA012282EAC102E17B7B
:103BB80013B281EA030282EA0212D2B2C3F30723E4
:103BC80083EA121343EA022383EAC2031BB288EA98
:103BD800030282EA0212D2B2C3F3072383EA121362
:103BE80043EA022383EAC2031BB283F0320282EA69
:103BF8000212D2B2C3F3072383EA121343EA022361
:103C080083EAC2031BB29AB24FF0FE0C4FF0090EC2
:103C1800C82009F10101DBB284F802C084F803E08E
:103C28004FEA122CA07184F86E11228084F812C019
:103C3800637438687968BA68B7F80C900AF5C47E76
:103C4800AEE807000AF5CC7A8EF80280AEF800904C
:103C580084F8A8C184F8A73116F8011F2868FCF772
:103C680069FEB245F8D1029BC4F85831FFF77EB916
:103C780094F8AC32204AC4F8A8B202EB8302926CE2
:103C880042B312AD04F2B3231D4E45F8203D002186
:103C980004F2C52331800B9380211523A52784F8CE
:103CA800B232284684F8B11284F8B0729047284698
:103CB8003188FEF7C4FB0A9D124804F52C716D1A71
:103CC800152DA8BF15252A4627F0DCFD0E4A94F8C5
:103CD800AC3215700D4A013382FB0312A2EBE3727A
:103CE80002EB42029B1A84F8AC32FFF74FB900BFCF
:103CF800003600205B5F002078DF0208D46C0020CB
:103D0800EC590020BC370020D137002056555555B6
:103D1800E41D0020D34AD44B92F80BE03168D4F864
:103D28001C211B88D148891A4FF47A72DFB202FB32
:103D38000EF21B0A8777077591424FF00007C37789
:103D480043758770077180F01284C94BC9491A6896
:103D58009B68C4F818B181FB02E7D21781FB03E125
:103D6800C2EBA702DB17C3EBA10311124FEA232C06
:103D78004FF0F40E02770127417780F82030302188
:103D88007522782380F821C080F81AE0C77680F879
:103D9800221080F8232080F82430FFF740B8DFF89D
:103DA800F492D9F80000FCF7B9FD00283FF4CCA83C
:103DB800D9F800000121FCF7AEFD0222002387F8A4
:103DC800742088F80030FFF7BFB894F8341194F8DD
:103DD8003531D8F800004A1C013384F8342184F8BE
:103DE8003531FCF7A7FDFFF782B8A34CDFF8A8929E
:103DF8004FF0000A0AE01B2B00F014830D2B00F093
:103E080012824FF0010389F801303868FCF78FFD02
:103E1800002838D03868FCF784FD83B27E2B3268DE
:103E28002AD099F801100029EFD194F83621002AF8
:103E3800E1D07D2B00F00C8294F844E1BEF1000F34
:103E480004D080F02003DBB284F84411511CC9B2BD
:103E58002244092984F8361182F8383100F0EC81BF
:103E68000829D2D8B4F84221134403EB132303F0F2
:103E7800FF03A4F84231C8E784F836A184F837A1D3
:103E880089F801A0C1E794F8453133B194F8393184
:103E980084F84501302B00F0498794F83721774B97
:103EA800DFF8F8C1DFF8F8E1DFF8F8A101271046DC
:103EB80000283FF42CA83268A2EB0802012A00F27D
:103EC800AD8194F84691B9F1000F40F0C28294F8A0
:103ED800471133F8112012B984F84771E8E7013126
:103EE800B2F5826F84F8471100F002811FD9B2F54C
:103EF800E26F00F09A8034D9B2F5046F00F0A48024
:103F0800B2F5116F00F04781B2F5E46FD0D11046D9
:103F18005B4A176C918A642303FB07F393FBF1F167
:103F280021F032F9002384F83731FEF7F0BFB2F5FB
:103F3800007F00F0B9802CD8B2F5807F00F0458171
:103F4800B2F5887FB4D1DCF800205207B0D5002143
:103F58004FF4887021F018F9002384F83731FEF700
:103F6800D6BFB2F5C06F00F0B380B2F5E06F9FD155
:103F7800434A906B918A642303FB00F34FF4E0609B
:103F880093FBF1F121F000F9002384F83731FEF7B3
:103F9800BEBFB2F5047F00F02781B2F5806F87D1EC
:103FA80094F848310133DBB2032B00F2588142F216
:103FB800107184F8483101FB03F1324B1B88002B48
:103FC80040F04B810131304B1B78DF072F4B1B88AA
:103FD80048BF0431D80748BF0A319A0748BF14318F
:103FE8001F0648BF2831D80548BF28315A0748BF9F
:103FF80064311F0748BFC831980548BF01F5C8712B
:104008009A0648BF01F57A71DF0648BF01F5FA61E3
:10401800580648BF01F57A614FF4806021F0B4F882
:10402800002384F83731FEF772BF1046144AD76B65
:10403800918A642303FB07F393FBF1F121F0A4F8C1
:1040480084F83791FEF763BF114BB3F9041001EB05
:1040580081011046490021F097F884F83791FEF75E
:1040680056BF00BF443E00203C3E0020785C002044
:10407800F059002067666666DC1D002078DF0208BC
:10408800BC330020806C00205B5F0020D46C0020D3
:104098002450002078590020000000200436002019
:1040A8004C6C0020523E00209EF8061000293FF478
:1040B800FFAEC44BC4491B68104681FB0321DB17C4
:1040C800C3EBA10121F060F884F83791FEF71FBF18
:1040D8009EF80620002A3FF4EBAEBA4B4FF4C060BE
:1040E800996821F051F8002384F83731FEF70FBFA3
:1040F800DCF8002012F020097FF4DAAEB34A116828
:10410800090600F1F585B24A127B002A3FF4D0AEC9
:1041180094F84911032900F29486DFE801F0322867
:104128001902AC4B1B6859799A79DB7901F1407116
:1041380001EB022101EB0341002384F849314FF4DC
:10414800826021F021F8002384F83731FEF7DFBEC2
:10415800A14B1A68137A507992781B0403EB002359
:1041680013444A1C84F8492103EB0161E7E79A4BA1
:104178001A68D379107952781B0403EB002313448F
:10418800EFE7954B1A689379D07812781B0403EB04
:1041980000231344E5E79EF80520002A3FF488AE83
:1041A8009AF8001000293FF483AE8C4B1B8803EB70
:1041B80083035B004FF4116093FBF1F120F0E4FFFF
:1041C800002384F83731FEF7A2BEDCF8002051073F
:1041D8007FF56EAE00214FF4807020F0D5FF0023EC
:1041E80084F83731FEF793BE9EF80520002A3FF485
:1041F8005FAE9AF8001000293FF45AAE744B5B7B0F
:10420800002B00F09B85754B1B8893FBF1F101EBAC
:10421800810149004FF4047020F0B6FF002384F8B0
:104228003731FEF774BE4FF0010184F8361184F877
:104238003831A4F84221E8E5B4F84221C2F1FF027E
:1042480093427FF4DEAD4FF0010384F84531D8E5A1
:104258004FF0010384F84431D7E50231B3E6012376
:1042680084F8483142F21071A7E63B685E2098470F
:104278003B68022098475A4B534AB3F9503082FBA7
:1042880003124FEAE378C8EBA2080FFA88F85FFA3E
:1042980088F021F01BF8C8F3072021F017F83B68D5
:1042A8005E2098473B68032098474E4B1B78D907F8
:1042B80040F1318112F008FF4B4B9FED4C7AD3ED62
:1042C800037A67EE877AFCEEE77ACDED027ABDF8DD
:1042D8000830002800F02285D8B24FEA132820F0D1
:1042E800F5FF404620F0F2FFDFF8088198F8053026
:1042F800002B40F0C4820AA93D4820F0ADFF3B687E
:104308005E2098473B6813209847BDF928805FFADC
:1043180088F020F0DBFFC8F3072020F0D7FF3B68C8
:104328005E2098473B681B209847BDF92A805FFAB2
:1043380088F020F0CBFFC8F3072020F0C7FF3B68C8
:104348005E2098473B68232098474E2020F0BEFF08
:10435800002020F0BBFF0AA9254820F07DFF3B681C
:104368005E2098473B6812209847BDF928805FFA7D
:1043780088F020F0ABFFC8F3072020F0A7FF3B68C8
:104388005E2098473B681A209847BDF92A805FFA53
:1043980088F020F09BFFC8F3072020F097FF3B68C8
:1043A8005E2098473B6822209847452020F08EFFE2
:1043B800002020F08BFF3B685E20984794F814316A
:1043C800FEF71DBDF059002067666666305500206F
:1043D800443E002040300020943000203C3E002025
:1043E800D86500205B5F0020543E0020CDCC4C3EB9
:1043F800809698004C6C002008F0F6FAB54B1B68C4
:10440800C01A40F6B833984200F2C680DFF804A319
:104418009AF804303A2B00F09283002388F8003091
:10442800FEF792BD3868FCF782FA00287FF4E9AC01
:104438004FF0010384F83731E7E4C4F8283184F8F1
:104448002031DFF8D48220F0EDFE94F82C31FEF70D
:1044580033BDA149062018F005FB002384F8460166
:1044680084F83731FEF753BD4FF000093B6884F8F4
:1044780014915E203468DFF8A48298473B681720BF
:104488009847484620F022FF944BA3FB04239B0B3C
:10449800A8FB03125209C2EB0212A3EB8203D8B2A3
:1044A80020F014FF3B685E2098473B681820984727
:1044B8008B4BA3FB04239B09A8FB03125209C2EBF5
:1044C8000212A3EB8203D8B220F000FF484620F086
:1044D800FDFE3B685E209847FEF794BC0AF1FF3A60
:1044E80084F867A1FFF7BFBB0CF1FF3C84F866C1F5
:1044F800FFF783B9013B84F85F31FFF7A7B8013BA9
:1045080084F85E31FEF781BF76493A2018F0AAFA9E
:104518002870FEF72FBDDFF80882734BB8F80890B3
:10452800A3FB09394FEA99095FFA89F020F0CEFE1A
:104538004FEA192020F0CAFED8E63B685E2098476B
:104548003B6810209847404620F0C0FE404620F0C7
:10455800BDFE3B685E2098473B682120984740464F
:1045680020F0B4FE404620F0B1FEFEF7D0BD5F4B10
:1045780032681B78C4F81C21013B012B3FF6E5ABE0
:104588001022022382700371FFF7DFBB20F03AFE8E
:1045980001233B70FEF761BC554AB2F85231002145
:1045A8000133A2F8523188F80010FEF7CDBC514B08
:1045B8001B88DA0515D4D80600F13084990600F175
:1045C8003C845A0600F14884180700F15284D90740
:1045D80000F1EC8413F0020F0CBF4FF004084FF009
:1045E8000C08454B454A1B78D27803F001030AB101
:1045F80043F002035320029320F08EFD404A1288B4
:1046080002EB820202EB8202900080B220F06AFD87
:10461800002020F067FD3B4A3B4912883868C2EB0E
:10462800C212520081FB023111444FEAE27ACAEB0E
:10463800612A5FFA8AFA5146FCF77CF9334B3868ED
:104648001A78029B48EA0308304B8AEA020A0021DA
:1046580083F800A0FCF76EF941463868FCF76AF960
:104668002A4B2A4A1B78386888EA0303DBB21946C2
:104678001370FCF75FF994F85031002B7EF4A3AD6A
:104688004F2020F049FD1AF0B5FA1AF0B3FA1AF0E3
:10469800B1FA01213868FCF74DF91D4A1B4B92F815
:1046A80000801B78194A386808F0010883F0010374
:1046B80041461370FCF73EF9144B144A1B783868CE
:1046C80088EA030319461370FCF734F994F850315B
:1046D800FEF779BDF85800208951020873B2E74502
:1046E800D34D621079530208CDCCCCCC476C002056
:1046F800DC1D0020D46C00205B5F00205C6C002077
:104708003C3E0020446C002003082080EC4E002032
:1047180094330020E0580020AC5B0020898888880A
:104728004C6C0020AE4EAF4B00930024A6F13F0125
:10473800AD4BAE4A089106F8404CAD4909960AA817
:10474800FDF754FF089E731C08933470089B2922B8
:10475800591C08911A70089BEA22591C08911A7072
:10476800089BC822591C08910AA81A7026F0B6FAA4
:10477800471C0AA93A46089827F084F8089AD319DA
:1047880001330893D455089B5A1C08921C70089B47
:104798005A1C08921C70089B5A1C08921C70089B93
:1047A8005A1C08921C70089B5A1C08921C70089B83
:1047B8005A1C08921C70089B5A1C08921C70089B73
:1047C8005A1C08921C70089B5A1C08921C70089B63
:1047D8005A1C08921C70089B5A1C08921C70089B53
:1047E800FF22591C08911A70089B0122991812A8D7
:1047F80008911A7050F8283D9B1B337020F088FDF3
:104808002C70FEF7B7BB8846894608460491059187
:104818008E4606910391FEF72BBE764A704B1268BE
:104828000B93A3F1400500202121D70003F8400C89
:10483800A97040F1D08270490326704B1B88580537
:1048480000F1C682DA0700F1F58203F002036C4A30
:10485800002B1CBF032611466A4F3246384627F004
:1048680011F8F31912A80133B91E40F8203D0022AF
:104878005B1AF2556B7020F04BFDFEF735BC624BAE
:1048880093F800A0BAF1000F3FF435AD5F4AB4F8D1
:1048980016E111883B6802924FEA0E1E64201FFA47
:1048A8008EFE00FB01A14FEA4A00B1FBF0F14EEA8F
:1048B800012E1FFA8EFEC1F303215E204EEA010984
:1048C80098473B68062098475FFA89F020F0FEFC7D
:1048D8004FEA192020F0FAFCB4F81631029A4C4934
:1048E800B2F800904A7A01339BB2012A93FBFAF09E
:1048F8000AFB1033A4F8163100F049836E234548AB
:104908004A7B03FB09F380FB03014FEAE379C9EB18
:10491800A1092AB13C4B1FFA89F91B7899FBF3F9D5
:104928003B68DFF8FCA05E2098471FFA89F93B68CE
:104938003A209847AAFB093A4FEA5A1A1FFA8AF30B
:10494800D8B2029320F0C2FC029B180A20F0BEFCE9
:104958003B685E2098473B683B209847642303FBED
:104968001A939BB22C48053380FB0320DB17C3EB5B
:10497800A000C0B220F0AAFC002020F0A7FC3B68F1
:10498800DFF898A0DFF890905E2098473B682820D1
:104998009847DAF8003089FB0329DB17C3EBA9092C
:1049A8005FFA89F020F092FCC9F3072020F08EFC12
:1049B8003B685E2098473B6804209847B8F8083061
:1049C800002B40F04D82DAF8083083F310085FFAC4
:1049D80088F020F07BFCC8F3072020F077FC8AE4FD
:1049E800F85B002087300020B8030308C0030308E1
:1049F800CC0303088C3300209C030308D46C0020EC
:104A0800B4030308BB5B0020523E00203C3E00205C
:104A1800443E0020310CC33067666666F0590020BA
:104A28001F85EB51CC4ACD4B0B9212AEA2F13D0043
:104A380046F8200D1988CA4FA2F1400300204FF014
:104A48000A0E02F8400C082283F801E030469A70FA
:104A5800FDF7D1FC3B68C349DA1781FB0313C2EBAE
:104A6800A30399B23046FDF7C6FC0DF0F9FCBF6808
:104A78000A9B3A0C591C0A911A700A9B3A0A591C4B
:104A88000A911A700A9B5A1C0A921F700A9B5A1C98
:104A98000A921870304620F03BFCFEF722BBC4F89F
:104AA80024B187F80090FEF7D8B9AF4F9FEDAF8AD1
:104AB800B7F90220A8480B9007EE902AF8EEE77A9B
:104AC80012AE67EE887AA0F13D01FDEEE77A46F86E
:104AD800201D00F8403C0823CDED027A00F83F3C49
:104AE8001E23BDF8081000F83E3C3046FDF783FC55
:104AF800B7F9003007EE903AF8EEE77A304667EEFD
:104B0800887AFDEEE77ACDED027ABDF80810FDF758
:104B180072FCB7F9043007EE903AF8EEE77A3046BF
:104B280067EE887AFDEEE77ACDED027ABDF80810D7
:104B3800FDF761FC304620F0EBFBFEF7CFBA9AF8A0
:104B48000240C4B1013CE4B201345444514600224D
:104B580011F8013B534083EA0313DBB2120ADF006A
:104B680042EA03228C4287EA131382EA0302EFD156
:104B7800002A7FF452AC794A7D4F794B12887D4CDC
:104B8800FA61DFF808921A68FA629B68B4F8522151
:104B9800F8660021FB64D9F80000F963FA6506F0AD
:104BA8009FFD029000287EF4CAA90221D9F80000CE
:104BB800FBF7B1FE94F854319AF803200392642B62
:104BC8004FF0040287F8742040F0578194F855316B
:104BD800072B04BF9DF8083084F8553194F85531F7
:104BE800069307EB031ADAF804100291084626F038
:104BF80075F8DAF8081005915FFA80FA084626F089
:104C08006DF8C0B204900AEB0002069B5A4802995C
:104C180002900832C27123F00F028646827204980D
:104C280003F00F0300EBCA008EF80D3052468EF8E1
:104C38000E000EF10F0026F025FE504B049A059940
:104C48000AF10900184426F01DFE0298C37903F101
:104C5800010ACBB1013B5FFA83FC0CF1080CDFF8C9
:104C680030E184440023073010F8011B59408B00C1
:104C7800CA0883EA410302F018024B404EFA02F2D6
:104C880053408445DBB2EFD13C4A03980AF802301E
:104C980019F07EFF94F855310022013384F855311C
:104CA80084F85421029BDDF808A09B785BB11AF8C0
:104CB8000510D9F80000FBF73DFE01359AF80230DF
:104CC800EDB2AB42F3D894F854310322013384F89F
:104CD800543187F8742088F80020FFF762B8022161
:104CE800D8F80000FBF717FE94F82C31FEF7E4B86B
:104CF8001023042218460AA98DF82A908DF82B90C3
:104D08008DF82C908DF82D908DF828308DF829206D
:104D180020F01AFA84F83791FEF7F9B8184A1268A1
:104D2800D2067FF5D9AA8046FFF7D9BA1549881F58
:104D380020F0E4F884F84601FFF7AFB8074B19886C
:104D4800FFF765BA104AD278002A0CBF4FF0040C5E
:104D58004FF0050CFEF76CBEF85B00203C3E0020CF
:104D6800F0590020676666662450002058A08B41E1
:104D780000000020DC1D0020F84A0020FE4A002028
:104D8800305500201C1F00205C6C00207859002042
:104D98000007090E0123D8F800003B70FBF7C1FD9E
:104DA8000746D8F80000FBF7BCFD7F067EF455A83F
:104DB8008E287EF452A894F82031002B7EF46AA83D
:104DC800944BC4F828312D2384F82C31FEF74CB8C5
:104DD8000326914940E5914B914A1B68914903F498
:104DE800800383420ABF11460326042625E58E491F
:104DF8009A790B8803EB830303EB83034FEA830859
:104E08001FFA88F8002A00F0DE80884B1B680FFA2A
:104E180083FA0DF025FB40B2FEF732BA4FF03408A2
:104E2800FFF7DFBB9846994618460493059303930A
:104E3800FEF71EBB7E4904260EE54FF02408FFF757
:104E4800D0BB4B1CDBB2042B84F849314FEA01611B
:104E58007FF475A9FFF770B94FF01008FFF7C1BBD1
:104E68000DF0FEFA20F032FA002020F02FFAFFF7BA
:104E780042BA4FF02008FFF7B4BB97F875A06D4908
:104E880004951AF00F0F04BF0AF1010A5FFA8AFAB3
:104E9800BAF1070F28BF4FF0010A4FEA0A1C07EBC7
:104EA8000C03187C644B02930A18002392F8241010
:104EB800614A93725FFA8CF31A46604B964607EB89
:104EC8000C024EEA000001291870D26803F10100B3
:104ED8000CD90239C9B28D1C1D44034603F8012BB5
:104EE800AB424FEA1222F9D101310844BC4422F006
:104EF80060030AF1010A9CF811205FFA8AFA134349
:104F0800BAF1080F037000F1010366D04FEA0A1CDA
:104F180007EB0C01494A087C464901449A1A91F862
:104F2800241055180EF1100E132D5FFA8EFEC6DDF3
:104F3800049D0298DFF80CE1D1B28B1DDBB243F07F
:104F48004002C27103F1010CCBB14B1DDBB2083337
:104F5800C31804930EF10100002310F8011B5940F7
:104F68008B0083EA4103CA084B40354902F0180216
:104F780041FA02F25340049A8242DBB2EDD103981F
:104F88000CF80E3087F875A019F002FE8AE63B6827
:104F98005E2098473B68392098475FFA89F020F0EF
:104FA80095F94FEA192020F091F9E8E44FF0080844
:104FB800FFF717BB984699461846049305939E46F3
:104FC8000393FEF755BA4FF0FF3320E7174B90468F
:104FD800B3F900A06420FEF753B9184A049D9A1A41
:104FE800A7E798469946184604930393FEF740BAF4
:104FF8000393FEF73DBA98460393FEF739BA9846ED
:1050080099460393FEF734BA98469946184603938F
:10501800FEF72EBA785C0020A8030308305500205C
:10502800A00303089C0303083C3E0020F05900201D
:10503800AC03030878DF0208F84A0020054B00207B
:105048000007090EFE4A00202DE9F04F2DED0C8BCC
:105058003C4B1B7895B0012B089001F070863A4CB8
:1050680094F80021002A41F0C180072B374D01F048
:105078006186002305936B6834489847002800F040
:105088006981B5F8B470002285F85520002F40F0EA
:105098004387B5F93E00AA6AB5F93C60696AB5F973
:1050A8004030DFF8B4B0821AE86A6A63711A1B1AD2
:1050B8002963274895F85610AB6316F02FFBDBF8E9
:1050C8000030990040F1F080D5ED0D5AD5ED0C7AFD
:1050D800204A94ED656AD4ED666A94ED677AD4F84F
:1050E800A0311268B8EEE58AD5ED0E5AF8EEE77AE7
:1050F800F8EEE58A013377EE867A38EE268A78EE7E
:10510800878A9342C4ED657A84ED668AC4ED678A1E
:10511800C4F8A03101F0D0830A4B1F78142F02F095
:1051280013870023D4F8A8610693062E00F2AF80F7
:10513800DFE816F0DA1537156C149F1614004B15B6
:10514800D01400BF2C3E0020A8200020D8650020E5
:10515800086600208039002030550020D84B1A7886
:10516800D4F8ACE1DFF8D0C39FEDD67A4FEACE0091
:105178000CEB000383ED007A002A7DD0D249B0EE13
:10518800476AF0EE476A0023F1EC017A013367EED3
:10519800A77A05EE903AB4EEE77AF1EE10FAF8EE57
:1051A800E55AB8BFB0EE677A934276EEA76AA7EEE3
:1051B800A56AE9D1F5EEC06A0CEB0003F1EE10FA2E
:1051C80083ED007A58DDC6EE265AC04BC04A1288D5
:1051D800F7EE007A75EEE75AD3ED007A65EEA77A16
:1051E800FDEEE77A17EE903A812B43F3058593425B
:1051F800A8BF134607EE903AF8EEE77AB54B00EBF6
:105208000E0103EB810393ED057AD3ED003A93ED9C
:10521800066A93ED014AD3ED046AD3ED034A93ED90
:10522800025AA3EEA77AA4EE276A66EEC76AA7EE2B
:10523800646ABDEEC77AE5EE276A17EE101A81296F
:1052480083ED056AC3ED066A43F3D3848A42A8BF97
:105258000A4607EE902AF8EEE77AFCEEE77ACDEDFB
:10526800077ABDF81C300CEB00029380BEF1000FEA
:1052780002D1132F04F02081152F42F01C846044C2
:10528800DFF8B882838828F81E30D4F8A861924BDA
:10529800013683FB06239A19F317C3EBA203C3EB6A
:1052A800C303F61AC4F8A8618C4B1B78002B01F0D5
:1052B800A3808B4EDFF88892DFF880A206F5BC78D1
:1052C8000027884BD5ED087A1B78172B01F08E83C1
:1052D80096ED007AB8EEC78A082B28EE278A07D100
:1052E800B0EE480A069326F041FC069B2AF8170000
:1052F800DBF8002092000BD5002F04F02084B0EEDC
:10530800480AD5F8143208F170009847B0EE408A80
:10531800B0EE480AD5F83431A8F170009847D5F8AE
:10532800A431404698476F4B1B78032BB0EE408A58
:1053380001F05683D6F8F800D5F8B830B0EE480A30
:1053480098470137032F08F12408A9EC010A06F150
:105358000406B6D1634B93F80090B9F1070F00F03B
:10536800988694F8B831002B40F0A0865E4B5B79A4
:10537800002B40F0CB8501235A4A84F8B8311278C3
:10538800072A02F0258000230B93584B94ED709A5E
:1053980093ED007A564BD4ED6FCAD3F800A0554B65
:1053A8000693F7EE007A37EEC9CA534B09932CEEF1
:1053B80007CA524B0A93B4EEE7CA514B079300252C
:1053C800F1EE10FA4F4BDFF87C91DFF87CB1DFED9E
:1053D8004E8A9FED4EAADFED3BBADFED4D9A9FED69
:1053E8004DBADFED4DAADFF864814C4F059388BFB5
:1053F800B0EE67CA2E464A4B99ED008A2B44D3ED8E
:10540800007AF5EE407AF1EE10FA17D0454B2B44AE
:10541800D3ED006A38EE667AB0EEC76AF4EEC67A63
:10542800F1EE10FA08D5B5EEC07AF1EE10FACCBF5D
:1054380037EEA68A36EEE78A83ED008A069B1A883D
:10544800930700F08580022E00F082809AF82E10D3
:10545800354B07EE901A2B4493ED007A4B42F8EE49
:10546800E76A07EE903A26EE877AF8EEE77AB4EE26
:10547800E77AF1EE10FA0AD407EE901AF8EE677A96
:10548800F4EEC77AF1EE10FA88BFF0EE477A274BB0
:10549800274903EB460331F91600B3F90C30C01A5B
:1054A80007EE100AB8EEC77AD007E7EE687A40F13F
:1054B8000586204B93ED008A27EE888A48E000BFD6
:1054C8008639002000000000A8200020883900202C
:1054D80084390020BC3B0020932449927D39002068
:1054E800086600202C3E00200C550020F0530020B8
:1054F80094300020D46C0020780000205B5F0020EE
:105508002055002098330020CDCCCC3DAE47813FBC
:105518000000C84200003443610BB63BA4330020AE
:10552800E45300206C22002014220020C4350020FF
:1055380024500020CC530020A43B0020303E002003
:1055480024550020AC210020DC520020B03300207C
:10555800079B94F8D0212B44D3ED01DA38EE6DDAAD
:10556800002A3DD0D24BD4F8D42108991B688A1A56
:105578009A4235DD9AF84830022B01F09D87022EB9
:1055880004F05A82CB4B1B68990740F11C87CA4B21
:10559800CA49DFF890E331F916C09EED008ADFF8BA
:1055A80088E3C7ED00BA03EB460028EE288AB0F975
:1055B8000C00A0EB0C0007EE900AF8EEE77ADEF894
:1055C800000027EE888A904238EE6DDAC1F2268113
:1055D800F7EE007AB4EEE79AF1EE10FA01F1F580F1
:1055E800B74B2B4493ED000A059B2CEE800A022E44
:1055F80020EE0D0AA3EC010A059304F0AA81099B89
:105608009BED007AD3ED007AAE4BD7ED006A93EDAF
:10561800006AAD4B67EE277A2B4427EE8C7AD3EDE0
:10562800007A67EE277AF0EE665AE7EE8D5AB1EE09
:10563800467AB4EEE57AF1EE10FA08DCB4EEE56AE3
:10564800F1EE10FA8CBFB0EE657AB0EE467A94EDC2
:10565800706AF7EE007AB4EEE76AF1EE10FAACBFC2
:105668000123002343B1F0EEE66AF0EEC77AF4EEC8
:10567800E67AF1EE10FA01D587ED007A022E04F0F1
:105688004281924A924B52F826001B68B0EE6D0A8E
:105698009847904A904B52F826001B6898479AF80A
:1056A800373023B1069B1B88002B00F06B85B0EECA
:1056B8006B8A8A4B9BED007A38EE400A2B4493EDB7
:1056C800008A83ED000A9AF8483030EE480AC0EEA6
:1056D800077A2BB30A9B1B78DB0721D5B7EE007A34
:1056E800B4EEC79AF1EE10FA04DB94F8D031002B2F
:1056F80000F05587D4F8D431089AD31A6C4A126846
:105708009A420DDD764B93ED007AB0EECDDAB4EE29
:10571800C7DAF1EE10FA41F19D80002384F8D03108
:10572800704B94F8E0212B4493ED007A2CEE877AA5
:1057380067EE277AC8ED007A32B9059BC7ED00BA43
:1057480043ED01BAC8ED00BA0136032E09F1040988
:1057580008F1040807F1040705F104057FF44BAECE
:10576800614B1B78072B01F03583012B01F01D8657
:10577800002794F8E831002B40F0EF855B4A5C4B3A
:1057880010681B6810F4805A93F82C3040F05E863D
:10579800584A594992ED006A498B584A84ED7E6A05
:1057A80092ED007A564A84ED7F7A07EE901AF8EE69
:1057B800E76AD2ED037A534A84ED7C6A37EE467A7B
:1057C80077EEE67AD2ED006A84ED7B7A012284F8DE
:1057D8000022C7EEA65A4C494C4A91ED005A4C4952
:1057E8009FED4C6A91ED004A4B49DFED4C6AD1EDD3
:1057F800004A92ED007A35EE045AF7EE007AF4EE9C
:10580800E75A35EE245AF1EE10FA88BFF0EE675ADF
:1058180025EE065AF4EEE65AB1EE476AF1EE10FAB2
:10582800B4EEC65AB8BFF0EE665AF1EE10FAC4EDFF
:10583800815A01F1CE80B4EEC75AF1EE10FA88BF52
:10584800B0EE475A304ADFED336AD2ED017A304A7A
:1058580092ED014A304A77EE847AD2ED014A77EE2A
:10586800A47A67EEA67AB4EEE76AF1EE10FA08DCDD
:10587800B4EEE77AF1EE10FA8CBFB0EE676AB0EEDC
:10588800476A214ADFED236AD2ED027A204AD2ED37
:10589800024A234A77EEA47A92ED007A67EEA67A56
:1058A800B1EE473AF4EEC37AF1EE10FA47D43DE090
:1058B800F853002004360020C4350020245000206E
:1058C800A053002014540020AC530020E4520020C0
:1058D800E05200203853002034530020802200205A
:1058E80004540020B85300202C3E002030550020DE
:1058F800943000203C3400204042002094350020A1
:10590800543E0020D454002098330020185400201E
:10591800A43300206F12833AB03300200000000047
:105928001C540020CC530020F4530020F4EEC77A16
:10593800F1EE10FA8CBFB0EE473AB0EE673AF04A93
:1059480052780AB9B1EE433A002B41F06483F7EE7E
:10595800003AEC4D2A78002A02F04686EA4BDFED41
:10596800EB7AD3ED024AD3ED016A93ED037A66EE42
:10597800244AE5EE264AE3EE074A63EEA44AF4EE2B
:10598800E74AF1EE10FAB4BFB0EE674AB0EE644AE7
:1059980098BFF0EE647A012ACDED0C4A02F04986F0
:1059A80093ED067AD3ED052AD3ED076A26EE077A3A
:1059B800A5EE227AA3EE267A23EE877AB4EEE77A6A
:1059C800F1EE10FAB4EEC47A8CBFF0EE676AF0EE2E
:1059D800476AF1EE10FA88BFF0EE676AB4BFF0EEDE
:1059E800447AF0EE477A022A8DED0D7A00F0DE80D7
:1059F80093ED0A7AD3ED092A93ED0B4A26EE077A3E
:105A0800A5EE227AA3EE047A23EE877AB4EEE67A3C
:105A1800F1EE10FAB4EEE77A8CBFB0EE664AB0EE5B
:105A2800474AF1EE10FA98BFF0EE446AA8BFF0EECC
:105A3800477A032A8DED0E7A00F0B88093ED0E7A3E
:105A4800D3ED0D2A93ED0F4A26EE077AA5EE227ABA
:105A5800A3EE047A23EE877AB4EEE67AF1EE10FA32
:105A6800B4EEE77A8CBFB0EE664AB0EE474AF1EE84
:105A780010FA98BFF0EE446AA8BFF0EE477A042AFD
:105A88008DED0F7A00F0928093ED124AD3ED112A32
:105A980093ED137A26EE044AA5EE224AA3EE074AAE
:105AA80023EE844AB4EEE64AF1EE10FAB4EEE74A81
:105AB8008CBFB0EE667AB0EE447AF1EE10FA98BF79
:105AC800F0EE476AA8BFF0EE447A052A8DED104A39
:105AD8006CD093ED164AD3ED152A93ED177A26EE7E
:105AE800044AA5EE224AA3EE074A23EE844AB4EEFE
:105AF800E64AF1EE10FAB4EEE74A8CBFB0EE667AE9
:105B0800B0EE447AF1EE10FA98BFF0EE476AA8BFFB
:105B1800F0EE447A062A8DED114A47D093ED1A4AE1
:105B2800D3ED192A93ED1B7A26EE044AA5EE224AF4
:105B3800A3EE074A23EE844AB4EEE64AF1EE10FAE1
:105B4800B4EEE74A8CBFB0EE667AB0EE447AF1EE76
:105B580010FA98BFF0EE476AA8BFF0EE447A072A19
:105B68008DED124A22D093ED1E7AD3ED1D2A93EDC6
:105B78001F4A26EE077AA5EE227AA4EE037A27EECC
:105B8800237AB4EEE67AF1EE10FAB4EEE77A8CBF37
:105B9800B0EE666AB0EE476AF1EE10FA8DED137A50
:105BA80098BFF0EE466AA8BFF0EE477A77EEE67A3D
:105BB800F7EE006AF4EEE67AF1EE10FAC4ED707AC8
:105BC80043F35F8486EEA77A022ADDED0D7A67EE4D
:105BD800244A67EE877ACDED0C4ACDED0D7A2DD0AB
:105BE800DDED0E7A67EE877A032ACDED0E7A25D0A1
:105BF800DDED0F7A67EE877A042ACDED0F7A1DD096
:105C0800DDED107A67EE877A052ACDED107A15D08A
:105C1800DDED117A67EE877A062ACDED117A0DD07F
:105C2800DDED127A67EE877A072ACDED127A05D074
:105C3800DDED137A27EE877A8DED137A344B1E68E3
:105C480016F0805601F09480F6EE005AC4ED815AA1
:105C5800002A02F0BE842F4BD4ED7F4A93F80380CC
:105C680094F900320A99D4ED7E6A91F800E0DFF8E1
:105C7800B0C02949DFF8AC90B1F906109CED007A64
:105C8800059106EE103AFDEEE44A244B99F800908F
:105C9800B3F81AB094ED7B5AD4ED7C7A14EE903AAE
:105CA800FDEEE64A00F0100C00F480000EF0010E44
:105CB800B8EEC66A14EE901A0690B8F1000F41F0DB
:105CC800ED81DFF84480BCF1000F41F0988098ED39
:105CD800007ADDED0C6ADFF850C025EE877AA6EE73
:105CE800267AF0EE676AE5EE076ABDEEE67A17EE09
:105CF800106A17EE100A9E42A8BF184616E000BFA9
:105D080000360020DA3D0020445400200000000046
:105D18008C3300205C6C0020AC6C002040420020DA
:105D2800205400204462002014340020B142C8BF2F
:105D3800084607EE100AB8EEC77A012A8CED007AF9
:105D480000F0DC8098ED047ADDED0D6A25EE877AA7
:105D5800A6EE267AF0EE676AE5EE076ABDEEE67A09
:105D680017EE106A17EE100A9E42A8BF1846B142F5
:105D7800C8BF084607EE100AB8EEC77A022A8CEDAB
:105D8800017A00F0BB8098ED087ADDED0E6A25EE09
:105D9800877AA6EE267AF0EE676AE5EE076ABDEE28
:105DA800E67A17EE106A17EE100A9E42A8BF184648
:105DB800B142C8BF084607EE100AB8EEC77A032AF0
:105DC8008CED027A00F09A8098ED0C7ADDED0F6A7E
:105DD80025EE877AA6EE267AF0EE676AE7EE056A80
:105DE800BDEEE67A17EE106A17EE100A9E42A8BFBB
:105DF8001846B142C8BF084607EE100AB8EEC77A7F
:105E0800042A8CED037A79D098ED107ADDED106ACA
:105E180025EE877AA6EE867AF0EE676AE7EE056ADF
:105E2800BDEEE67A17EE106A17EE100A9E42A8BF7A
:105E38001846B142C8BF084607EE100AB8EEC77A3E
:105E4800052A8CED047A59D098ED147ADDED116AA3
:105E580025EE877AA6EE867AF0EE676AE7EE056A9F
:105E6800BDEEE67A17EE106A17EE100A9E42A8BF3A
:105E78001846B142C8BF084607EE100AB8EEC77AFE
:105E8800062A8CED057A39D098ED187ADDED126A7C
:105E980025EE877AA6EE867AF0EE676AE7EE056A5F
:105EA800BDEEE67A17EE106A17EE100A9E42A8BFFA
:105EB8001846B142C8BF084607EE100AB8EEC77ABE
:105EC800072A8CED067A19D098ED1C7ADDED136A55
:105ED80065EE875AE6EE265AE5EE257AFDEEE77A74
:105EE80017EE900A8342A8BF03468142C8BF0B46FB
:105EF80007EE903AF8EEE77ACCED077ABEF1000F9C
:105F080040F03882002A40F0308233E2AB4B1B78F5
:105F1800013BDBB2FFF730BAA94B07934FF47A760F
:105F28001B68B6FBF3F3C3EB4316A649DFF8B88248
:105F380091F801A0A449B8F9060091F8009003EB84
:105F48008603DE00B6B2B74202F0E680D5F88810C4
:105F5800B5F93CE0EB6E4A1C07EE90EA7344012A5F
:105F6800C5F88820EB66F8EEE77A02F0E080D5ED18
:105F78001E5AD5ED206A07EE102A37EEE56AB8EE0C
:105F8800C75A012F86EE057A37EE257A77EEC77A5B
:105F980085ED1F7AE7EE866A85ED1E7AF0EE667A61
:105FA800C5ED216AC5ED206A02F07E84D5F89C1003
:105FB800B5F93EE02B6F4A1C07EE90EA7344012ABC
:105FC800C5F89C202B67F8EEE77A02F0C980D5ED7A
:105FD800235AD5ED256A07EE102A37EEE56AB8EEA2
:105FE800C75A012F86EE057A37EE257A77EEC77AFB
:105FF80085ED247AE7EE866A85ED237AF0EE667AF7
:10600800C5ED266AC5ED256A02F08284D5F8B01080
:10601800B5F940E06B6F4A1C07EE90EA7344012A19
:10602800C5F8B0206B67F8EEE77A02F0B280D5EDDC
:10603800285AD5ED2A6A07EE102A37EEE56AB8EE37
:10604800C75A012F86EE057A37EE257A77EEC77A9A
:1060580085ED297AE6EE276A85ED287AF0EE667AEC
:10606800C5ED2B6AC5ED2A6A02F04684A8F8060039
:10607800B5F8B430544A013B92F80090A5F8B43012
:1060880007990023B9F1070F4B608B60CB607FF451
:1060980068A906F0A9FC059BDFF84C81C01A94F8A2
:1060A800B831A8F80000002B3FF460A9013B84F840
:1060B800B83115B0BDEC0C8BBDE8F08F94ED5E7A6D
:1060C800B1F90000D4ED5F6AB1F902E03F4AF4EE9D
:1060D800C76A80EAE0738EEAEE71A3EBE073F1EE33
:1060E80010FAA1EBEE71B8BFF0EE476A8B42B8BF69
:1060F8000B4607EE103A1378B8EEC77A27EE287ADF
:10610800002B40F01D82324B93ED006AB4EECA6A50
:10611800F1EE10FA41F1DE80F7EE005A75EEC65A3C
:106128003BEE477A65EEAA5A2A4BA7EE256A93ED0D
:10613800007A26EE076AB5EEC06AF1EE10FA40F270
:106148001386C9EE865AB7EE007AB0EE476AA6EE15
:10615800E56AF0EE466AF4EEC76AF1EE10FA88BF17
:10616800F0EE476AF5EEC06AF1EE10FAB8BFF0EE4D
:106178006B6A194B93ED007A67EE877AA7EEA68AC9
:10618800FFF7E6B9154B164A2B4493ED007AD2ED8A
:10619800007A144B67EE277AF7EE006AF4EEE67A97
:1061A800F1EE10FA93ED007A88BFF0EE667A67EEAA
:1061B800877A27EE888AFFF77CBA00BFB8350020B7
:1061C800205500200C5500202C3E0020D8530020DC
:1061D800E0530020D4530020D05300202022002078
:1061E800C8530020C4530020303E0020072B02F083
:1061F8001B820026DFF83CB3B64DDBF800305905AA
:1062080001F16D80B44B1B78002B40F0F381B34F44
:1062180094F8123123B1B24A1288920742F09A8157
:1062280094F81821002A41F06480BB7F002B00F00D
:10623800F383022B02F01880032B01F0C082A94BD4
:106248005B88F97F0231C9B2002A01F0FE87002B72
:1062580001F0FB87A4480068B3FBF0F30FFA83F959
:10626800A4F84891002903F0148107EE909AF8EEFB
:10627800E77AF7EE006A86EEA77A9C4B0129D4EDFF
:10628800576AD3ED007A77EEE67A67EE877AC4ED3F
:10629800537A21D0D3ED017AD4ED586A77EEE67AB5
:1062A800022967EE877AC4ED547A15D0D3ED027AC5
:1062B800D4ED596A77EEE67A032967EE877AC4ED5A
:1062C800557A09D0D3ED037AD4ED5A6A77EEE67A97
:1062D80067EE877AC4ED567A85480078092803F076
:1062E8001081B9F1000F40F39E8391B394ED577A72
:1062F800D4ED537A77EE877A0129C4ED577AC3ED46
:10630800007A21D094ED587AD4ED547A77EE877AD2
:106318000229C4ED587AC3ED017A15D094ED597A63
:10632800D4ED557A77EE877A0329C4ED597AC3ED0F
:10633800027A09D0D4ED5A7A94ED567A77EE877AB4
:10634800C4ED5A7AC3ED037A01390229B8BF022194
:10635800C9B2002A18BF022166E30A9B654D1B7863
:10636800DE0700F163812A7822B19200624963480E
:1063780025F088FA624B1B68002B40F02E83614B96
:106388001B789BB1287870B1DFF87081DFF8A8918D
:106398000026F0B2D9F80030B8EC010A98472878FE
:1063A80001368642F5DB584B1B689847504B1B78E3
:1063B800072B00F0E284012384F8003115B0BDEC0E
:1063C8000C8BBDE8F08F514BC7ED00BA1B689342A8
:1063D800BFF6FEA84E4B1A88002384F8D031002A55
:1063E80041F090864B4A4C4B1178186881F00101B6
:1063F800FBF793FAFFF7F4B8484EDFF8409106F53B
:10640800F47806F51577F6EC017A95ED080AD5F8D3
:106418001432F8EEE77A404627EE800A9847A8F14A
:10642800E000D5F834319847A8F17000D5F8A431C8
:106438009847D6F8F400D5F8B830984708F12408FA
:106448004745A9EC010ADED1FEF784BF0A9A127803
:10645800D50703D4214A128BA4F8F421304A2349E2
:10646800128891ED037A07EE902AF8EEE77AB4EEF7
:10647800E77AF1EE10FA41F283802A49098807EE9B
:10648800901AF8EEE77AB4EEE77AF1EE10FAC0F275
:10649800E9872549254AD1ED006A92ED006A244929
:1064A800C4ED7E6ABCEEC75A76EE665A15EE102A1F
:1064B800C4ED7C6AC4ED7B5A84ED7F6AA4F8F421AC
:1064C8000122D1ED006A84F8002277EE677AFFF79F
:1064D80080B900BFD8650020E000002040420020BD
:1064E800D46C0020D4380020E8350020543E002029
:1064F8002C3E0020DA3D00202454002014340020D3
:10650800905100204C65002040620020F453002088
:106518005C6500205E65002060650020086600203C
:10652800D8540020DA540020C454002094350020A8
:10653800E054002030550020386200202455002007
:10654800CC4B93ED005AB5EEC05AF1EE10FA40F379
:106558000B84C94BD3ED004AF5EEC04AF1EE10FAB0
:1065680040F3028434EEC77A66EEE95A87EE246A6D
:10657800C5EE856AB7EE007AB4EEC76AF1EE10FA96
:1065880088BFB0EE476AB5EEC06AF1EE10FA76EE53
:10659800876AB8BFB0EE6B6A66EE266ADBE5B74A73
:1065A80092ED007AF0EEE76AF4EEC76AF1EE10FABF
:1065B8007FF7A0A8B24A92ED007AF0EECD6AF4EE29
:1065C800C76AF1EE10FA7FF795A8AE4A99ED007AFE
:1065D800D2ED006AB0EEC77AB4EEE67AF1EE10FAC0
:1065E8007FF588A801220899C4F8D41184F8D0212D
:1065F800FFF784B8A44BA54FB3F906207B8B9A42CA
:106608003FF706AEA24B1B78012B01F00986192B28
:1066180001F006860E2B3FF4FBAD082B3FF4F8ADD6
:106628009C4B00229A60C4F80C21F1E52B78002BD2
:106638003FF4A0AED4ED5F3A94ED5E6AD4ED7C7A77
:10664800954A94ED7B7AD2ED005A94ED5C4AD4EDEC
:106658005B4ADFF85C82DFF85CC2F4EEC63AF3EE20
:10666800046AF1EE10FA37EEA65A00F1F98798EDB0
:10667800026A26EE446AF0EE674AE6EE074AF4EE4E
:10668800C54A34EEE66AF1EE10FA48BFB0EE656A24
:10669800012B8CED006A3FF46DAE98ED066A26EE8C
:1066A800446AF0EE674AE6EE074AB4EEE45A34EE7E
:1066B800E66AF1EE10FA88BFB0EE656A022B8CED3F
:1066C800016A3FF457AE98ED0A6A26EE446AF0EE86
:1066D800674AE6EE074AF4EEC54A34EEE66AF1EE9A
:1066E80010FA48BFB0EE656A032B8CED026A3FF4DE
:1066F80041AE98ED0E6A26EE446AF0EE674AE6EE81
:10670800074AB4EEE45A34EEE66AF1EE10FAC8BF6E
:10671800B0EE656A042B8CED036A3FF42BAE98ED5E
:10672800126A26EE446AF0EE674AE6EE074AB4EECD
:10673800E45A34EEE66AF1EE10FAC8BFB0EE656AC4
:10674800052B8CED046A3FF415AE98ED166A26EE1B
:10675800446AF0EE674AE6EE074AF4EEC54A74EE7C
:10676800E66AF1EE10FAB8BFF0EE656A062BCCEDDA
:10677800056A3FF4FFADD8ED1A6A66EEC46AF0EE1A
:10678800674AE6EE874AB3EE046AB4EEE45A74EE5A
:10679800C66AF1EE10FAC8BFF0EE656A072BCCEDB9
:1067A800066A3FF4E7ADD8ED1E6A26EEC44AE4EE69
:1067B800077AF4EEC57A77EEC67AF1EE10FA48BF9A
:1067C800F0EE657ACCED077AD4E50799334BD1ED35
:1067D800017A93ED007AF0EEE77AF4EEC77AF1EEFB
:1067E80010FA7EF5FDAED1ED027AF0EEE77AB4EE5E
:1067F800E77AF1EE10FA7EF7F3AED1ED037AF0EE18
:10680800E77AB4EEE77AF1EE10FA7EF7E9AE244BB8
:106818001B689A077FF5DEAD2249234BB3F90C209C
:10682800B1F900E02148AEEB020E00688EEAEE7284
:10683800A2EBEE728242BEF6D3AEB3F90E30B1F9D6
:106848000220D21A82EAE273A3EBE27398427EF73F
:10685800C7AEBFE50B4B99ED007AD3ED006AB0EEF9
:10686800C77AB4EEE67AF1EE10FA7EF759AFFEF782
:1068780054BF00BFD4530020DC530020085400202C
:10688800045400200C540020AC6C0020404200202E
:1068980000360020543E00202054002000540020E0
:1068A8000436002024500020C4350020FC5300206A
:1068B800445400201434002007EE103A524BDFF8FD
:1068C80054811B78C4F8A071B8EEC77AF7EE006A55
:1068D800132B86EE879AB8F90400B4F8A47195EDE5
:1068E800080A01F07783494B494A93ED001A93ED62
:1068F800053A93ED122A93ED176AD3ED091A93ED31
:106908000E4AD3ED015AD3ED063A93ED0A7A93ED88
:106918000F5AD3ED132AD3ED186AD3ED044AD3EDF9
:10692800030A67EE897A69EE288A29EE088AA1EEB9
:10693800273A02EB87060021A2EE286AC4F89411D0
:10694800C4F89811A1EE884AE5EEA73AA7EE085ACE
:1069580093ED167AD3ED0D5A93ED021AD3ED0C1A76
:1069680086ED003AE2EEA86A64EEC34A27EE467A5C
:1069780093ED0B2AD3ED152A86ED204AE0EEC33AB3
:1069880065EEC45A93ED143AC3ED053AE1EE274A91
:10699800F0EE477AA1EEC45AE2EE085AE2EEC66A71
:1069A800E3EE287AC3ED064A83ED0E5AC3ED0F5A7B
:1069B80086ED406AC3ED176AC3ED187AC4F89C11D6
:1069C8007B1C03F01F03A4F8A431A8F80400FEF709
:1069D800A3BBB0EE465AFEF735BF18F0DDFECEE495
:1069E80025F0C4F82AF81700FEF7A4BC96ED007A43
:1069F80005EB4702B8EEC78A928F2AF8172028EECF
:106A0800278AFEF775BC00BF2C3E0020283C0020DA
:106A1800A4390020303E0020A4F848319946002AC5
:106A280000F07281D84B0221D84ADFEDD96A10688C
:106A3800D84A90F802C092F800E0027807EE902A4F
:106A4800F8EEE77AB0EE007A67EEA67AF4EEC77A47
:106A5800F1EE10FA40F3108337EEC77ADFEDCE6A15
:106A6800B0EE676AA7EE266AB0EE467A9FEDCB6A6B
:106A7800D3ED006A66EE866AB0EEE66AC4ED5B6A3C
:106A880084ED5E6ABCF1000F13D005EE90CAB8EE33
:106A9800E55ADFEDBF5A66EEA64A25EE255AF7EE0F
:106AA800005A75EEC55A64EE864AE4EE855A66EEDB
:106AB800A56ADFEDBB5A427927EE257A27EE267ABA
:106AC800CAB1DFEDB36ADFEDB75A26EE266A06EEE5
:106AD800902AF8EEE66A26EE266AB4EEE56AF1EE4A
:106AE80010FA00F37485F7EE005A35EEC66AC5EE63
:106AF800866A27EE267ABEF10C0F9FEDAB8ADFED92
:106B0800AB6A00F01585B4EEC87AF1EE10FA98BFBA
:106B1800B0EE478AB4EEE68AF1EE10FAB8BFB0EEEE
:106B2800668A84ED418A002900F0E280B0EE007A9E
:106B3800F4EEC77AF1EE10FA05DD37EEC77ADFED2D
:106B4800966AE7EE267A93ED017ADFED946A27EEEE
:106B5800267AB0EEC76A84ED5C7A84ED5F6ABCF190
:106B6800000F13D006EE90CADFED895AF8EEE66AF8
:106B780027EE075A66EEA56AF7EE005A75EEE65A52
:106B880025EE065AE5EE265A27EE257ADFED846AC9
:106B9800827967EEA67A67EE877AAAB107EE102A9D
:106BA800B8EEC77ADFED7A5ADFED7E6A27EE067A0D
:106BB80027EE257AB4EEE67AF1EE10FA40F30B856B
:106BC800DFED7B6A67EEA67ABEF10C0F00F08F84CA
:106BD800DFED756A9FED757AF4EEE67AF1EE10FA5C
:106BE80088BFF0EE667AF4EEC77AF1EE10FAB8BF15
:106BF800F0EE477A0129C4ED427A79DD4278DFED7B
:106C0800646A07EE902AF8EEE77AB0EE007A67EE4B
:106C1800A67A427AF4EEC77AF1EE10FA05DD37EE7D
:106C2800C77ADFED5D6AE7EE267A93ED027ADFED4B
:106C38005B6A27EE267AB0EEC76A84ED5D7A84ED4A
:106C4800606A9AB106EE902ADFED515AF8EEE66ACC
:106C580027EE075A66EEA56AF7EE005A75EEE65A71
:106C680025EE065AE6EE855A27EE257ADFED4C6AC0
:106C7800C37967EEA67A67EE877A0BB307EE103A08
:106C8800B8EEC77ADFED425ADFED466A27EE067A9C
:106C980027EE257AB4EEE67AF1EE10FA0CDCB5EEC2
:106CA800C07AF1EE10FA01F1C282B7EE006A36EE50
:106CB800477AC6EE076A01E0DFED3D6A67EEA67A1D
:106CC800BEF10C0F00F00984DFED376A9FED377ACB
:106CD800F4EEE67AF1EE10FA88BFF0EE667AF4EE9A
:106CE800C77AF1EE10FAB8BFF0EE477AC4ED437AEE
:106CF800BEF1090F00F0D58397F82170002F40F0FE
:106D08006C83002384F818312A4B1B7823B92A4F47
:106D1800BB78002B41F0AF82089809F0ADF91D4B04
:106D28001B78072B00F021840022072B84F8002110
:106D38007EF49FA905F058FE0590FEF79CB91F4BFD
:106D48001F4C1A681F4BDFF8888094F80001D2693D
:106D58001B88A8F80020A8F8023000287FF449AA68
:106D68000590194DFEF787B9DFED186AFFF701BAEC
:106D780041023EF569AFFEF76BBF05F035FE144BD7
:106D8800C01BD880FFF717BB543E002040300020BE
:106D98000AD7233C2C3E0020D7A368416F12033B3F
:106DA80000004843A4707D3F00C0F94400C0F9C406
:106DB8000000C842D66C0020E2310020C85E0020E6
:106DC800A8200020B22E0020D86500200000000076
:106DD800303E002005F008FEA94B0B9A1B78DFF81F
:106DE800B482801A012BA8F8020000F0E082072B79
:106DF8007EF4BEAC05F0F8FD0746FEF7BABCBEF15E
:106E0800000F41F0438498ED007ADDED0C6ADFF85D
:106E180088C225EE877AA6EE867AF0EE676AE7EEF4
:106E2800056ABDEEE67A17EE106A17EE100A9E4262
:106E3800A8BF1846B142C8BF084607EE100AB8EE08
:106E4800C77A012A8CED007A3FF48FAA98ED047A6C
:106E5800DDED0D6A25EE877AA6EE867AF0EE676A92
:106E6800E7EE056ABDEEE67A17EE106A17EE100A2D
:106E78009E42A8BF1846B142C8BF084607EE100A8E
:106E8800B8EEC77A022A8CED017A3FF46EAA98ED23
:106E9800087ADDED0E6A25EE877AA6EE867AF0EEA0
:106EA800676AE7EE056ABDEEE67A17EE106A17EE36
:106EB800100A9E42A8BF1846B142C8BF084607EE4E
:106EC800100AB8EEC77A032A8CED027A3FF44DAA6D
:106ED80098ED0C7ADDED0F6A25EE877AA6EE867AB4
:106EE800F0EE676AE7EE056ABDEEE67A17EE106A1D
:106EF80017EE100A9E42A8BF1846B142C8BF0846FE
:106F080007EE100AB8EEC77A042A8CED037A3FF42C
:106F18002CAA98ED107ADDED106A25EE877AA6EE98
:106F2800867AF0EE676AE7EE056ABDEEE67A17EE56
:106F3800106A17EE100A9E42A8BF1846B142C8BF91
:106F4800084607EE100AB8EEC77A052A8CED047ACF
:106F58003FF40BAA98ED147ADDED116A25EE877AD5
:106F6800A6EE867AF0EE676AE7EE056ABDEEE67A87
:106F780017EE106A17EE100A9E42A8BF1846B142D3
:106F8800C8BF084607EE100AB8EEC77A062A8CED85
:106F9800057A3FF4EAA998ED187ADDED126A25EE34
:106FA800877AA6EE867AF0EE676AE7EE056ABDEEA6
:106FB800E67A17EE106A17EE100A9E42A8BF184626
:106FC800B142C8BF084607EE100AB8EEC77A072ACA
:106FD8008CED067A3FF4C9A998ED1C7ADDED136AA9
:106FE80065EE875AE6EE265AE5EE257AFDEEE77A53
:106FF80017EE900A8342A8BF03468142C8BF0B46DA
:1070080007EE903AF8EEE77ACCED077A002A7FF49B
:10701800ACA9FFF7AFB91B4B5A79002A3EF497ACDD
:10702800194A1278002A3EF492AC1B78DFED174A11
:1070380007EE903A164BB8EE677A1B8807EE902A4F
:1070480006EE903AF8EEE77AF8EE666A67EE277A87
:10705800B7EE007AC7EEA63AF4EEE43AF1EE10FA8B
:1070680088BFF0EE643AF4EEC73AF1EE10FAB8BF12
:10707800F0EE473AFEF76DBCB0EE677AF6E400BF73
:107088002C3E00204C6C0020523E0020713DAA3F4F
:107098003C3E0020303E002014340020BCF1000F9C
:1070A80000F09783BEF1000F41F07087DFF8A485E8
:1070B800B9F1000F41F0C885D8ED006ADDED0C4A42
:1070C800DFF894C565EEA66ABDEEC77A17EE101A0A
:1070D800B0EE667AA4EE867AF0EE676AE7EE056AA5
:1070E800BDEEE67A17EE106A17EE100A9E42A8BFA8
:1070F8001846B142C8BF084607EE100AB8EEC77A6C
:10710800012A8CED007A3FF430A998ED047ADDED80
:107118000D6A25EE877AA6EE867AF0EE676AE7EEC4
:10712800056ABDEEE67A17EE106A17EE100A9E425F
:10713800A8BF18468E42B8BF084607EE100AB8EE38
:10714800C77A022A8CED017A3FF40FA998ED087AE4
:10715800DDED0E6A25EE877AA6EE867AF0EE676A8E
:10716800E7EE056ABDEEE67A17EE106A17EE100A2A
:107178009E42A8BF18468E42B8BF084607EE100ABE
:10718800B8EEC77A032A8CED027A3FF4EEA898EDA0
:107198000C7ADDED0F6A25EE877AA6EE867AF0EE98
:1071A800676AE7EE056ABDEEE67A17EE106A17EE33
:1071B800100A9E42A8BF18468E42B8BF084607EE7E
:1071C800100AB8EEC77A042A8CED037A3FF4CDA8EA
:1071D80098ED107ADDED106A25EE877AA6EE867AAC
:1071E800F0EE676AE7EE056ABDEEE67A17EE106A1A
:1071F80017EE100A9E42A8BF18468E42B8BF08462E
:1072080007EE100AB8EEC77A052A8CED047A3FF427
:10721800ACA898ED147ADDED116A25EE877AA6EE12
:10722800867AF0EE676AE7EE056ABDEEE67A17EE53
:10723800106A17EE100A9E42A8BF18468E42B8BFC1
:10724800084607EE100AB8EEC77A062A8CED057ACA
:107258003FF48BA898ED187ADDED126A25EE877A4F
:10726800A6EE867AF0EE676AE7EE056ABDEEE67A84
:1072780017EE106A17EE100A9E42A8BF18468E42F3
:10728800B8BF084607EE100AB8EEC77A072A8CED91
:10729800067A3FF46AA898ED1C7ADDED136A65EE6C
:1072A800875AE6EE265AE5EE257AFDEEE77A17EEDE
:1072B800900A8342A8BF03468142D8BF194607EE09
:1072C800901AF8EEE77ACCED077A002A7FF44DA8F9
:1072D800FFF750B8C74B93ED006AFEF72CBFAB68B9
:1072E800002B3EF48FAF05F1500128469847FEF772
:1072F80089BFC14BC149D3F8EC30086844F6206116
:107308008B42A8BF0B46B3F57A7FB8BF4FF47A73A8
:1073180099B2C006A4F81A11DBF8003041F1BF8217
:10732800DB0400F16B83B64BD3F800C0BCF932E044
:10733800B44BB548D3ED037AD4F81C31A0FB010156
:107348008809642191FBF0F11429BDEEE77A04EB7A
:107358004308A8BF142101338B42C4F81C3117EE2F
:10736800109AA4BF0023C4F81C3104EB4303A8F807
:107378002091B3F9203107EE103AB8EEC77A77EECC
:10738800C77AFDEEE77ACDED057ABDF9141081EAEA
:10739800E173A3EBE173734502F364809B4B1946D9
:1073A8004FF07E530B60FEF740BFDFF8B08205F068
:1073B8001BFB974AD4F8E4311268C4F8E401C31AF5
:1073C8009A1A0746A8F80430A8F80620FEF7D1B99B
:1073D80005F00AFB0B90FDF7D8BF1E218748FBF785
:1073E80012FA00283FF48DAC8A4B1B885A063FF5E9
:1073F80088AC94F88431BB4242F0A980834BD4ED29
:10740800627A93ED010AD4ED435A9FED836ADFED6A
:10741800836A27EEE57A68EE277AA8EE007AE5EE29
:10742800807AB4EEC67AF1EE10FA88BFB0EE467AEA
:10743800B4EEE67AF1EE10FAF4EEC67AB8BFB0EE22
:10744800667AF1EE10FA88BFF0EE467AF4EEE67A44
:10745800F1EE10FAB8BFF0EE667A84ED417AC4ED29
:10746800437A4EE4B4F8F411914240F282856C49B3
:107478006C4AD1ED007A92ED007A6B49C4ED7E7AC0
:1074880077EE676AC4ED7C7A0122C4ED7B6A84EDED
:107498007F7AD1ED006ADFED657A84F80022FEF785
:1074A80098B9FDEEC87ADFF8B48117EE903AA8F8DB
:1074B8000490A8F806301FE45D4B1B88002B40F0B1
:1074C80077855C4A5C4B11781868FAF726FAD4F885
:1074D800D421089B9A1AFEF752B8BDEEE77ADFF876
:1074E8007C8117EE103AA8F80430FFF7EDBB9FED4A
:1074F8004A7ADFED4A6ADFF86481F4EEC77AF1EE82
:1075080010FA98BFB0EE677AFDEEE77AB4EEE67A45
:10751800F1EE10FA17EE902AB8BFB0EE667A01299C
:1075280084ED427AA8F802203FF768ABFFF7E4BB86
:10753800B4EEC87AF1EE10FA98BFB0EE478ABDEE05
:10754800C77AB4EEE68ADFF81481F1EE10FA17EE86
:10755800102AB8BFB0EE668A84ED418AA8F80020E8
:1075680000297FF4E3AAFFF7C7BB05F03DFADFF86F
:10757800EC80324B801B1B78A8F80400FFF7D4BBC3
:107588002F4A3049D2ED006A2F4A91ED006A1278ED
:10759800C4ED7E6A84ED7F6A002A40F0E68476EEC8
:1075A800C65AF0EE466ABCEEC76A2849C4ED7B5A53
:1075B80016EE102AC4ED7C6AA4F8F421FF22D1ED5E
:1075C800006A84F8002277EEC77AFEF702B9DFED89
:1075D800206AFFF78EBAB5EEC07AF1EE10FA00F124
:1075E8002A86B7EE006A36EE477AC6EE076AFFF7D4
:1075F800E9BA00BFD4530020200800208C330020B3
:1076080094300020543E0020D34D621078000020B2
:10761800E8350020D46C002000C0F94400C0F9C44B
:10762800C454002094350020E054002000000000DD
:107638005C6500205E650020606500202C3E00200F
:107648003C340020C854002044620020DC54002050
:107658000000C8424454002014340020303E00206A
:1076680098ED016A26EE646AB0EE674AA6EE074A0C
:10767800B4EEC45A34EE666AF1EE10FAC8BFB0EE42
:10768800656A012B8CED006A3EF474AE98ED056ACC
:1076980026EE646AB0EE674AA6EE074AB4EEC45A0C
:1076A80034EE666AF1EE10FAC8BFB0EE656A022BD6
:1076B8008CED016A3EF45EAE98ED096A26EE646AC6
:1076C800B0EE674AA6EE074AB4EEC45A34EE666ACC
:1076D800F1EE10FAC8BFB0EE656A032B8CED026AB2
:1076E8003EF448AE98ED0D6A26EE646AB0EE674A3D
:1076F800A6EE074AB4EEC45A34EE666AF1EE10FA02
:10770800C8BFB0EE656A042B8CED036A3EF432AE56
:1077180098ED116A26EE646AB0EE674AA6EE074A4B
:10772800B4EEC45A34EE666AF1EE10FAC8BFB0EE91
:10773800656A052B8CED046A3EF41CAE98ED156A5B
:1077480026EE646AB0EE674AA6EE074AB4EEC45A5B
:1077580074EE666AF1EE10FAC8BFF0EE656A062BA1
:10776800CCED056A3EF406AED8ED196A66EEE46A19
:10777800B0EE674AA6EE874AB3EE046AB4EEC45A7E
:1077880074EE466AF1EE10FAC8BFF0EE656A072B90
:10779800CCED066A3EF4EEADD8ED1D6A66EEE44A1D
:1077A800E4EE877AF4EEC57A77EEC67AF1EE10FA4F
:1077B800B8BFF0EE657ACCED077AFEF7DBBD97F837
:1077C8002030C3EB431103EB8103DB009BB2FEF7D0
:1077D80038BDDFF80485B9F1000F41F0CB80D8ED52
:1077E800006ADDED0C4ADFF8F4C465EEA66ABDEE6A
:1077F800C77A17EE101AB0EE667AA4EE867AF0EE23
:10780800676AE7EE056ABDEEE67A17EE106A17EECC
:10781800100A9E42A8BF1846B142C8BF084607EEE4
:10782800100AB8EEC77A012A8CED007A3EF466ABEE
:1078380098ED047ADDED0D6A25EE877AA6EE867A54
:10784800F0EE676AE7EE056ABDEEE67A17EE106AB3
:1078580017EE100A9E42A8BF18468E42B8BF0846C7
:1078680007EE100AB8EEC77A022A8CED017A3EF4C8
:1078780045AB98ED087ADDED0E6A25EE877AA6EE1F
:10788800867AF0EE676AE7EE056ABDEEE67A17EEED
:10789800106A17EE100A9E42A8BF18468E42B8BF5B
:1078A800084607EE100AB8EEC77A032A8CED027A6A
:1078B8003EF424AB98ED0C7ADDED0F6A25EE877A5D
:1078C800A6EE867AF0EE676AE7EE056ABDEEE67A1E
:1078D80017EE106A17EE100A9E42A8BF18468E428D
:1078E800B8BF084607EE100AB8EEC77A042A8CED2E
:1078F800037A3EF403AB98ED107ADDED106A25EEBD
:10790800877AA6EE867AF0EE676AE7EE056ABDEE3C
:10791800E67A17EE106A17EE100A9E42A8BF1846BC
:107928008E42B8BF084607EE100AB8EEC77A052A95
:107938008CED047A3EF4E2AA98ED147ADDED116A32
:1079480025EE877AA6EE867AF0EE676AE7EE056A94
:10795800BDEEE67A17EE106A17EE100A9E42A8BF2F
:1079680018468E42B8BF084607EE100AB8EEC77A26
:10797800062A8CED057A3EF4C1AA98ED187ADDED59
:10798800126A25EE877AA6EE867AF0EE676AE7EE47
:10799800056ABDEEE67A17EE106A17EE100A9E42E7
:1079A800A8BF18468E42B8BF084607EE100AB8EEC0
:1079B800C77A072A8CED067A3EF4A0AA98ED1C7ABD
:1079C800DDED136A65EE875AE6EE265AE5EE257A6E
:1079D800FDEEE77A17EE900A8342A8BF034681427C
:1079E800D8BF194607EE901AF8EEE77ACCED077A79
:1079F800BEF1000F7EF4BEACFEF784BAAA4BD3F8F2
:107A080000C0BCF832E04FEA5E0E91E4DFF8D09295
:107A1800D4ED017A94ED006AB9F80000D9F8143071
:107A280077EEA77AF0EE006AB0EE677AA6EE267ACD
:107A3800013804EBC002D6EE267A083A1033F6EE87
:107A4800003A27EE237A67EEA37A84ED207AC4ED14
:107A5800217A964CA64604F1800192ED027A92EDC5
:107A6800036ADEED036ADEED027A53ED014A13ED97
:107A7800025A37EE674A76EEC65A77EE277AE4EE70
:107A8800845A0138A2F10802E5EE047A0EF1080ED4
:107A980003F1080336EE267A01F10801E4EE877A4D
:107AA800E5EE475A67EEA37A25EEA37AC1ED007A90
:107AB80081ED017AD1D1142F7DF4E9AB04F094FF64
:107AC800069BDFF82082C01AA8F80200D4F8A86143
:107AD800FDF7DDBBD4F8AC81B4F8A4A1744BCAF1AE
:107AE80020095FFA89F90AEB481E03EB8E0E5FEA5C
:107AF800990301F00185013318016E496E4A0EEBB6
:107B0800000C0EF1100313ED024A13ED035A13EDA6
:107B1800016A13ED047A51ED024A51ED035A51ED11
:107B2800016A51ED047A64EE244A65EE255A66EE40
:107B3800266A67EE277A10339C4542ED024A42EDE9
:107B4800035A42ED016A42ED047A01F1100102F193
:107B58001002D8D15949A0F11002964401EB020C49
:107B6800224419F0030309D0BEEC017AFCEC017A37
:107B780067EE277A013BE2EC017AF5D1BAF1000F02
:107B880041F0A581142F7DF482AB04F02DFF069BF4
:107B9800DFF85081D4F8A861C01AA8F80200FDF7F0
:107BA80076BBDFF83C914148D9F80820B9F80C10A9
:107BB80023F034F8424B1F78142F01F07385D4F862
:107BC800A8610136C4F8A86122E7D4F8AC913D4B0E
:107BD8003D4ADFED3E7AD2ED008A3D4A4FEAC901BF
:107BE8000B44F8EE688A9B8809EE103A643BC82B70
:107BF800A8BFC82368EEA78AF8EE497A782BB8BFE1
:107C0800782368EEA78A07EE903A4944B0EE680AEE
:107C180002EB8108B8EEE78A23F0F4FFB8EEC99AC0
:107C2800F0EE409AB0EE680A23F04EFF38EE097A7B
:107C380079EE487A28EE098A67EE877AB7EE006A05
:107C480088EE277A142FF8EE007A77EE076A60EE4E
:107C5800277A89EEA67A77EE065A36EE477AC6EE86
:107C6800256A67EEA67A27EE267AC8ED006A88EDBF
:107C7800047AC8ED026AC8ED017AC8ED037A01F00A
:107C88006385144B0E4A09F1010983FB0938A8EBF7
:107C9800E97808EB48080136A9EB08081778C4F812
:107CA800A861C4F8AC8117E794300020A820002010
:107CB800A4390020343B0020B8200020243B0020B9
:107CC8002C3E0020A43B00202055002027D4D2368B
:107CD800F0670020565555554454002014340020B0
:107CE8008C390020303E0020DFF80494B9F800E019
:107CF800D9F804C04FEA5E084FEA880204EB8E0602
:107D08005FEADE0E04EB020300F0A08010320EF1F1
:107D1800010EEB4803EB0E1E324410330CF1100732
:107D280006F1100151ED032A51ED043A10ED043A21
:107D380010ED032A51ED026A11ED016A10ED020AF5
:107D480010ED018A12ED044A12ED035A53ED044A6C
:107D580053ED035A13ED027A53ED017A52ED020AFC
:107D680012ED011A73EE238A72EE221A40ED048A8C
:107D780040ED031A70EE268A78EE061A40ED028A64
:107D880040ED011A74EE848A75EE851A43ED048A73
:107D980043ED031A77EE208A77EE811A43ED028AC3
:107DA80043ED011A73EE633A75EE655A17ED035AFF
:107DB80032EE623A74EE644A65EE631A17ED044ACD
:107DC80023EE052A64EE652AE3EE041A10339E4575
:107DD80024EE843AA3EE842A00F1100007F110077C
:107DE800A5EE853A01F1100102F11002E4EE852AB0
:107DF80041ED071A01ED082A02ED073A42ED082A7B
:107E080057ED055A17ED065A70EE666A38EE466A5F
:107E180030EEC77A71EE677A26EE253A65EEE63AD5
:107E280025EE674A67EE054AE6EE053AA6EE853A7C
:107E3800A7EE254AE7EEA54A01ED063A41ED053AD7
:107E480002ED064A42ED054A7FF46CAF1FFA88F846
:107E5800624641469B4820F037FF4146D9F8042046
:107E6800304620F031FF984B1B78142B7FF42EAE50
:107E780024E6DFF8809299F80020900801F0CB847E
:107E8800DFF874C200F101084FEA48180CEB080E3D
:107E98000CF12003ACF1700113ED076A53ED056A8C
:107EA80013ED037A53ED017A53ED025A13ED084AA4
:107EB80053ED064A13ED045A26EE066A66EEA66AE4
:107EC80027EE077A67EEA77AA4EE046A20339E4568
:107ED800E4EEA46A01F11001A5EE057AE5EEA57AB3
:107EE800F1EEC65AB1EEE66AF1EEC76AB1EEE77A8C
:107EF80041ED085A01ED076A41ED066A01ED057A80
:107F0800CAD1A8F12008C44404EB001012F00303FE
:107F180018BF0CF1080C0FD05CED017A1CED027A49
:107F280067EEA77A013BE7EE077A0CF1080CB1EE91
:107F3800E77AA0EC017AEFD1142F01F0138401360F
:107F4800C4F8A861FDF70CB904F04EFD5E4B06902D
:107F58001F78142F05BFDFF8A481D4F8A861D4F8DE
:107F6800A861A8F80060FDF7E0B876EE665AFFF75A
:107F78001ABB564A5649D2ED007A564A91ED007A14
:107F88001278C4ED7E7A84ED7F7A002A01F064824B
:107F980077EE676A5049C4ED7C7AC4ED7B6AFF22AC
:107FA800D1ED006ADFED4D7A84F80022FDF711BCAF
:107FB8004B494B69002B3DF4E2AA4A484A4B0088DA
:107FC80093FBF0F00B684FF0010E186081F811E098
:107FD800FDF7D5BA454EDFF8289196ED004A96EDA3
:107FE800057AD6ED014A96ED066AD6ED046A96ED55
:107FF800035AD6ED025A67EE897A09EB8703A4EE95
:10800800277AA4EEA76A66EEC76AA5EE476AE5EE88
:10801800A76A20EE070A86ED056AC6ED066A83EDB3
:10802800007A29EE088A23F0A1FD69EE288AD6EDA8
:108038000E5AD6ED176A96ED091AD6ED121A96ED74
:108048000F5A96ED187A96ED0A2AD6ED132A96ED70
:108058000D6AD6ED167A96ED0C3AD6ED0B3A96EDFA
:10806800154AD6ED144AE1EE085A002209EB8703B7
:10807800E8EEA16A00B2C4F89421A2EE085AC4F846
:108088009821C4F89C21A8EEA27A26EE656A67EECC
:10809800E67AA3EE655AA3EE886AA6EEC47AE8EEFD
:1080A800A47A86ED0E5AC3ED205A86ED0F6AC3ED09
:1080B800406A86ED177AC6ED187AFEF781BC00BFD4
:1080C800B8200020A82000202C3E00203C340020AE
:1080D800C854002044620020DC5400200000000046
:1080E800646500207C65002020A10700283C002052
:1080F8008C3900208639002028210020303E0020BD
:10810800A4390020C6494A69002A3DF469AA0A68C8
:1081180013604B74FDF764BAB5F93C306A6207EE38
:10812800903A0122F8EEE77AEB66C5F8882000233A
:10813800012FC5ED1F7AC5ED1E7AC5F8803001F014
:10814800B781B7427DF432AFB5F93E302B6707EE01
:10815800903A00220123F8EEE77AAA62C5F89C302B
:108168000023012FC5ED247AC5ED237AC5F8943094
:1081780001F09A81B7427DF449AFB5F940306B6799
:1081880007EE903A00220123F8EEE77AEA62C5F892
:10819800B0300023012FC5ED297AC5ED287AC5F83E
:1081A800A8307DF463AF9FED9F8AB9F1030F46D0E5
:1081B800BAF1000F09D007EE90AAF8EEE77AF4EECC
:1081C800C87AF1EE10FA01F17183974A6B6F126861
:1081D80094F8B011A8F8060003EB560393FBF6F6E3
:1081E8000023EE6293621363D36231B18F4B1B8815
:1081F80023F40063002B7DF43BAF8D4B1B6813F415
:10820800003341F049818B491A46C85C012803F1C3
:108218000C0300F0F5840132152AF6D1FDF728BFCA
:10822800854B9B7B002B3EF4FBA9FDF7F1BFF7EED6
:10823800006AFEF743BDF7EE006AFEF7C3BCB0EE76
:10824800480A23F093FC00B2B2E7B4F8489109F168
:10825800FF390FFA89F9B9F1000FA4F848917EF7B0
:10826800DEAB764BFEF741B8B4F81A3103F57A73F2
:108278009BB2FDF7E6BFDFF8E88198F80020013AE5
:108288000A2A1DD8DFE812F0A1005A0104013E01B4
:108298001C001C00EE008F006A0054000B00684AA6
:1082A800684952680968C8328A4203D322F0A6F99D
:1082B80030B1BB78032B01F02D83012388F80030FF
:1082C800FB78002B3EF428AD5F4B1B78D80740F1B4
:1082D8008580DFF87091D4F89021D9F800309A425F
:1082E80000F2888098F80030012B3EF415AD94F820
:1082F8008C21002A3EF410AD0B2B0DD801229A4098
:1083080040F6030112EA01070DD112F4C06F03D041
:10831800093B012B41F2E783494BD9F800205A6009
:108328000B2388F80030002384F88C31FEF7F4BC66
:10833800464B1B78002B01F025821A200EF098FE80
:10834800002841F01F8294F88C31002B41F01A82EA
:10835800092388F8003010F01FFFB1E71A200EF04B
:1083680087FE0028F7D03A4B1B88002BF3D1394BF6
:108378004520D3F8009022F063F90E2022F060F92E
:10838800484622F003FADDF82090484622F0FEF92C
:10839800314A324B12681A6048460A2388F800307E
:1083A80010F046FCD7E722F00BF910F02FFF002859
:1083B80086D022F023F9002882D0274A274B12685A
:1083C8001A600A2388F800307AE71F4B1B78DB070E
:1083D80001F18F82FB78002B3EF49EAC19F032FA43
:1083E80000283FF476AF174B1B6803F59C530833FE
:1083F800C4F8903198F80030012B7EF48DAC94F8D5
:108408008C31002B7EF488ACBB78032B01F0798388
:1084180011F0C0FC012384F88C31FEF77DBC00BF4D
:108428006465002000000000C85E0020806C002009
:10843800D42E0020B8F10208605F0020543E0020CE
:1084480098350020846500205B5F002058360020A6
:10845800746D0020706D0020846D00207C6D0020FC
:10846800DF31002022F0ACF87B4B002105208DE89D
:108478000300A3F108020291532011F0C1FB002868
:108488007FF41EAF754A0823106088F8003017E79C
:10849800DFF8C89122F094F8714AD9F804301268CC
:1084A80064339342BFF40CAF402022F06FF80028E9
:1084B8007FF406AFD9F80030DFF8CCB169494FF046
:1084C800400A0FE0059122F0BBF80599D9F8003071
:1084D8000A680133013ABAF1010A0A60C9F80030A2
:1084E80001F02A821BF803301846002BEAD100233A
:1084F8004FF0FF32C9F800300423C9F8042088F887
:108508000030DDE622F05CF8574A0292A2F10C0333
:10851800252101930091A2F10A035021163A49201E
:1085280011F06EFB00287FF4CBAE4C4B4FF0FF31BF
:1085380007221860596088F80020C1E6484B474A6E
:108548001B68536047490023136003220B6088F8B7
:108558000020B5E6454ADFED467A92ED080A059314
:10856800B4EEE70AF1EE10FA40F2AD8423F094FB82
:10857800D4ED457A20EE270A23F0F8FAB0F5617FAA
:10858800059B00F33A8607EE900AF8EEE76ADFEDFE
:10859800397A66EEA76A07EE903AB8EEE77AFDEE0A
:1085A800E67A17EE903A2033402B41F2F0809FEDA7
:1085B800320A23F0DBFA00B207EE900AB8EEE77A47
:1085C8002E4BD3ED037A77EE877AC3ED037AFDF766
:1085D80027BE0A9B93F800E00EF0010EBEF1000FD3
:1085E8007DF4C8AEFDF78EBC254BDFED267A1E68FC
:1085F800C4ED707A16F0805640F01A8310F48006A5
:1086080000F0AE810026B6EE007A67EE877AF4EEC7
:10861800E75AF1EE10FA48BFF0EE675A40F10883C6
:10862800C4ED815AFDF714BB04F0DEF90646FDF7E8
:10863800E1BD74EE677AB7EE007AF4EEC77AF1EE30
:1086480010FAC4ED707A40F31C8784EEA77A8DED9A
:108658000C7AFDF7F3BA00BFE4E102089835002070
:1086680084650020646D002036E0020878520020FE
:108678008FC2753CD06D393A00000000543E00208E
:108688008C33002000000080D0DF0208BAF1000F10
:1086980000F0CD8598ED007ADDED0C6ADFF8E8C8CA
:1086A80025EE877AA6EE867AF0EE676AE7EE056A27
:1086B800BDEEE67A17EE106A17EE100A9E42A8BFC2
:1086C8001846B142C8BF084607EE100AB8EEC77A86
:1086D800012A8CED007A3DF44DAE98ED047ADDED7B
:1086E8000D6A25EE877AA6EE867AF0EE676AE7EEDF
:1086F800056ABDEEE67A17EE106A17EE100A9E427A
:10870800A8BF1846B142C8BF084607EE100AB8EE1F
:10871800C77A022A8CED017A3DF42CAE98ED087ADE
:10872800DDED0E6A25EE877AA6EE867AF0EE676AA8
:10873800E7EE056ABDEEE67A17EE106A17EE100A44
:108748009E42A8BF1846B142C8BF084607EE100AA5
:10875800B8EEC77A032A8CED027A3DF40BAE98ED99
:108768000C7ADDED0F6A25EE877AA6EE867AF0EEB2
:10877800676AE7EE056ABDEEE67A17EE106A17EE4D
:10878800100A9E42A8BF1846B142C8BF084607EE65
:10879800100AB8EEC77A042A8CED037A3DF4EAADE4
:1087A80098ED107ADDED106A25EE877AA6EE867AC6
:1087B800F0EE676AE7EE056ABDEEE67A17EE106A34
:1087C80017EE100A9E42A8BF1846B142C8BF084615
:1087D80007EE100AB8EEC77A052A8CED047A3DF444
:1087E800C9AD98ED147ADDED116A25EE877AA6EE0B
:1087F800867AF0EE676AE7EE056ABDEEE67A17EE6E
:10880800106A17EE100A9E42A8BF1846B142C8BFA8
:10881800084607EE100AB8EEC77A062A8CED057AE4
:108828003DF4A8AD98ED187ADDED126A25EE877A49
:10883800A6EE867AF0EE676AE7EE056ABDEEE67A9E
:1088480017EE106A17EE100A9E42A8BF1846B142EA
:10885800C8BF084607EE100AB8EEC77A072A8CED9B
:10886800067A3DF487AD98ED1C7ADDED136A65EE66
:10887800875AE6EE265AE5EE257AFDEEE77A17EEF8
:10888800902A9342A8BF13468A42A8BF194607EE0A
:10889800901AF8EEE77ACCED077AFDF76BBDD800B1
:1088A8003EF53EADFDF7C1BC012A40F3018607EE57
:1088B800101AB8EEC77AC7EE876AB1EEE68AB9F140
:1088C800030F13D0BAF1000F09D007EE90AAF8EE03
:1088D800E77AF4EEC87AF1EE10FA00F1E787EB6E6A
:1088E80003EB560393FBF6F36B622AE4B0EE480AF7
:1088F80023F03CF900B2E5E7012A7FF754AC07EE14
:10890800101AB8EEC77AC7EE876AB1EEE68A4CE469
:10891800012A40F3C98507EE101AB8EEC77AC7EEE8
:10892800876AB1EEE68AB9F1030F13D0BAF1000FE6
:1089380009D007EE90AAF8EEE77AF4EEC87AF1EEDD
:1089480010FA00F1B3872B6F03EB560393FBF6F392
:10895800AB620FE4B0EE480A23F008F900B2E5E78D
:10896800B6EE007AF4EEC75AF1EE10FA3FF74BAEC6
:10897800FDF76EB9D8ED004A9DED0C4ADFF808C640
:1089880065EEA44AFDEEC73AE4EE064AB0EE674A41
:10899800A4EE854A13EE901AF4EEC46AF1EE10FACA
:1089A800F0EE444A88BFF0EE474AFDEEE44A14EE82
:1089B800900A14EE906A9842A8BF1E468142C8BF2A
:1089C8000E4604EE906AF8EEE44A012ACCED004A1D
:1089D8003DF494AAD8ED044A9DED0D4A65EEA44AEB
:1089E800E4EE064AB0EE674AA4EE854AF4EEC46A9D
:1089F800F1EE10FAF0EE444A88BFF0EE474AFDEE79
:108A0800E44A14EE900A14EE906A9842A8BF1E46F3
:108A18008842B8BF0E4604EE906AF8EEE44A022A8D
:108A2800CCED014A3DF46AAAD8ED084A9DED0E4AFC
:108A380065EEA44AE4EE064AB0EE674AA4EE854A1B
:108A4800F4EEC46AF1EE10FAF0EE444A88BFF0EE94
:108A5800474AFDEEE44A14EE900A14EE906A9842F2
:108A6800A8BF1E468842B8BF0E4604EE906AF8EECC
:108A7800E44A032ACCED024A3DF440AAD8ED0C4A58
:108A88009DED0F4A65EEA44AE4EE064AB0EE674A49
:108A9800A4EE854AF4EEC46AF1EE10FAF0EE444A08
:108AA80088BFF0EE474AFDEEE44A14EE900A14EE51
:108AB800906A9842A8BF1E468842B8BF0E4604EE88
:108AC800906AF8EEE44A042ACCED034A3DF416AA6B
:108AD800D8ED104A9DED104A65EEA44AE4EE064A28
:108AE800B0EE674AA4EE854AF4EEC46AF1EE10FAD5
:108AF800F0EE444A88BFF0EE474AFDEEE44A14EE31
:108B0800900A14EE906A9842A8BF1E468842B8BFE1
:108B18000E4604EE906AF8EEE44A052ACCED044AC3
:108B28003DF4ECA9D8ED144A9DED114A65EEA44A2E
:108B3800E4EE064AB0EE674AA4EE854AF4EEC46A4B
:108B4800F1EE10FAF0EE444A88BFF0EE474AFDEE27
:108B5800E44A14EE900A14EE906A9842A8BF1E46A2
:108B68008842B8BF0E4604EE906AF8EEE44A062A38
:108B7800CCED054A3DF4C2A9D8ED184A9DED124A3C
:108B880065EEA44AE4EE064AB0EE674AA4EE854ACA
:108B9800F4EEC46AF1EE10FAF0EE444A88BFF0EE43
:108BA800474AFDEEE44A14EE900A14EE906A9842A1
:108BB800A8BF1E468842B8BF0E4604EE906AF8EE7B
:108BC800E44A072ACCED064A3DF498A9D8ED1C4A98
:108BD8009DED134A65EEA45AE6EE045AE5EE257AB1
:108BE800F4EEE76AF1EE10FAC8BFF0EE477AFEF746
:108BF800EFBE8223FCF737BBDFEDE07AFCF7FEBA65
:108C0800D4F8B46153003EB1981801EB800076782F
:108C18004078B042BDF42CAA134401EB8301002331
:108C2800C4F8B411A4F80832C4F80C32FDF720BA1D
:108C3800B7EE007A77EE677AF4EEE75AF1EE10FABB
:108C480088BFF0EE675AEBE4D8ED004A9DED0C4A78
:108C5800DFF834C365EEA44AFDEEC73AE4EE064AEF
:108C6800B0EE674AA4EE854A13EE901AF4EEC46A91
:108C7800F1EE10FAF0EE444A88BFF0EE474AFDEEF6
:108C8800E44A14EE900A14EE906A9842A8BF1E4671
:108C98008142C8BF0E4604EE906AF8EEE44A012A03
:108CA800CCED004A3DF461ABD8ED044A9DED0D4A88
:108CB80065EEA44AE4EE064AB0EE674AA4EE854A99
:108CC800F4EEC46AF1EE10FAF0EE444A88BFF0EE12
:108CD800474AFDEEE44A14EE900A14EE906A984270
:108CE800A8BF1E468842B8BF0E4604EE906AF8EE4A
:108CF800E44A022ACCED014A3DF437ABD8ED084AE4
:108D08009DED0E4A65EEA44AE4EE064AB0EE674AC7
:108D1800A4EE854AF4EEC46AF1EE10FAF0EE444A85
:108D280088BFF0EE474AFDEEE44A14EE900A14EECE
:108D3800906A9842A8BF1E468842B8BF0E4604EE05
:108D4800906AF8EEE44A032ACCED024A3DF40DABF2
:108D5800D8ED0C4A9DED0F4A65EEA44AE4EE064AAA
:108D6800B0EE674AA4EE854AF4EEC46AF1EE10FA52
:108D7800F0EE444A88BFF0EE474AFDEEE44A14EEAE
:108D8800900A14EE906A9842A8BF1E468842B8BF5F
:108D98000E4604EE906AF8EEE44A042ACCED034A43
:108DA8003DF4E3AAD8ED104A9DED104A65EEA44AB9
:108DB800E4EE064AB0EE674AA4EE854AF4EEC46AC9
:108DC800F1EE10FAF0EE444A88BFF0EE474AFDEEA5
:108DD800E44A14EE900A14EE906A9842A8BF1E4620
:108DE8008842B8BF0E4604EE906AF8EEE44A052AB7
:108DF800CCED044A3DF4B9AAD8ED144A9DED114AC8
:108E080065EEA44AE4EE064AB0EE674AA4EE854A47
:108E1800F4EEC46AF1EE10FAF0EE444A88BFF0EEC0
:108E2800474AFDEEE44A14EE900A14EE906A98421E
:108E3800A8BF1E468842B8BF0E4604EE906AF8EEF8
:108E4800E44A062ACCED054A3DF48FAAD8ED184A23
:108E58009DED124A65EEA44AE4EE064AB0EE674A72
:108E6800A4EE854AF4EEC46AF1EE10FAF0EE444A34
:108E780088BFF0EE474AFDEEE44A14EE900A14EE7D
:108E8800906A9842A8BF1E468842B8BF0E4604EEB4
:108E9800906AF8EEE44A072ACCED064A3DF465AA42
:108EA800D8ED1C4A9DED134A65EEA45AE6EE045A25
:108EB800E5EE257AF4EEE76AF1EE10FAC8BFF0EEB7
:108EC800477AFEF7F2B99FED2E7AFFF779BB2D4B63
:108ED8004FEA890E5FEA9A0901EB0E0C03EBC818FA
:108EE800A64400F0FF8409F101094FEA091908EBCB
:108EF800090008F110030CF110010EF1100213ED36
:108F0800024A13ED035A13ED016A13ED047A51ED89
:108F1800024A51ED035A51ED016A51ED047A64EEAB
:108F2800244A65EE255A66EE266A67EE277A1033DC
:108F3800984242ED024A42ED035A42ED016A42ED7F
:108F4800047A01F1100102F11002D8D1A9F1100937
:108F5800C8440CEB0901CE441AF0030A3EF412AEE1
:108F6800B8EC017AF1EC017A67EE277ABAF1010AD6
:108F7800EEEC017AF4D1FEF705BE00BF0000024313
:108F880000000000A439002014340020BAF1000FBA
:108F980000F09483DFF854869DED0C4AD8ED004A22
:108FA80065EEA44AE4EE064AB0EE674AA4EE854AA6
:108FB800F0EE444AB9F1000F06D0F4EE446AF1EE3F
:108FC80010FAC8BFF0EE474ABDEEC77A17EE101A7E
:108FD800BDEEE47A04EE901A17EE100A814200F30F
:108FE80071849842A8BF184607EE100AB8EEC77AEF
:108FF800DFF8FCC5012A8CED007A3DF4BBA998ED99
:10900800047A9DED0D4A25EE877AA4EE067AB0EE35
:10901800674AA7EE054AB0EE447AB9F1000F00F0AE
:109028003A84F4EEC46AF1EE10FA40F33484084648
:109038009842A8BF184607EE100AB8EEC77A022A67
:109048008CED017A3DF496A998ED087A9DED0E4ACB
:1090580025EE877AA4EE067AB0EE674AA7EE054AAF
:10906800B0EE447AB9F1000F00F00A84F4EEC46A55
:10907800F1EE10FA40F3048408469842A8BF184657
:1090880007EE100AB8EEC77A032A8CED027A3DF48F
:1090980071A998ED0C7A9DED0F4A25EE877AA4EE1A
:1090A800067AB0EE674AA7EE054AB0EE447AB9F1FF
:1090B800000F00F0DB83F4EEC46AF1EE10FA40F31F
:1090C800D58308469842A8BF184607EE100AB8EE9E
:1090D800C77A042A8CED037A3DF44CA998ED107AEE
:1090E8009DED104A25EE877AA4EE067AB0EE674A1F
:1090F800A7EE054AB0EE447AB9F1000F00F0AC8350
:10910800F4EEC46AF1EE10FA40F3A68308469842DA
:10911800A8BF184607EE100AB8EEC77A052A8CEDE4
:10912800047A3DF427A998ED147A9DED114A25EEAD
:10913800877AA4EE067AB0EE674AA7EE054AB0EE43
:10914800447AB9F1000F00F07D83F4EEC46AF1EEC1
:1091580010FA40F3778308469842A8BF184607EEEE
:10916800100AB8EEC77A062A8CED057A3DF402A9F2
:1091780098ED187A9DED124A25EE877AA4EE067AC4
:10918800B0EE674AA7EE054AB0EE447AB9F1000F8F
:1091980000F04E83F4EEC46AF1EE10FA40F348830F
:1091A80008469842A8BF184607EE100AB8EEC77AD4
:1091B800072A8CED067A3DF4DDA898ED1C7A9DED22
:1091C800134A65EE875AE4EE065AE5EE857AB9F158
:1091D800000F00F02583F4EEE67AF1EE10FA40F184
:1091E8001F830A469A42A8BF1A4604EE902AF8EE50
:1091F800E44ACCED074AFDF7BDB807EE903ADFED3B
:10920800EC6AB8EEE77A66EEA65A9FEDEA5A9FED49
:10921800EA6ADFEDEA7AA5EE856A26EEA55AE5EE5A
:10922800867AE5EE276A26EE870AFFF7C2B9D8EDF7
:10923800006ADDED0C4A65EEA66AE4EE866AF0EE99
:10924800674AE6EE854AFDEEE46A16EE90EA714555
:1092580000F325829E45A8BF9E4606EE90EAF8EEEA
:10926800E66A002E00F03484DFF884C3012ACCEDCE
:10927800006A3DF47FA8D8ED046ADDED0D4A65EE7D
:10928800A66AE4EE866AF0EE674AE6EE854AFDEEE7
:10929800E46A16EE90EA714500F31F819E45A8BF67
:1092A8009E4606EE90EAF8EEE66A002E00F03C8450
:1092B800022ACCED016A3DF45DA8D8ED086ADDED1F
:1092C8000E4A65EEA66AE4EE866AF0EE674AE6EEB6
:1092D800854AFDEEE46A16EE90EA714500F30981CD
:1092E8009E45A8BF9E4606EE90EAF8EEE66A002E76
:1092F80000F00F84032ACCED026A3DF43BA8D8EDB8
:109308000C6ADDED0F4A65EEA66AE4EE866AF0EEB9
:10931800674AE6EE854AFDEEE46A16EE90EA714584
:1093280000F3E4809E45A8BF9E4606EE90EAF8EE5C
:10933800E66A002E00F0B883042ACCED036A3DF4F7
:1093480019A8D8ED106ADDED104A65EEA66AE4EEBC
:10935800866AF0EE674AE6EE854AFDEEE46A16EEA6
:1093680090EA714500F3BF809E45A8BF9E4606EE71
:1093780090EAF8EEE66A002E00F08C83052ACCED20
:10938800046A3CF4F7AFD8ED146ADDED114A65EED6
:10939800A66AE4EE866AF0EE674AE6EE854AFDEED6
:1093A800E46A16EE90EA714500F39A809E45A8BFDC
:1093B8009E4606EE90EAF8EEE66A002E00F07E83FE
:1093C800062ACCED056A3CF4D5AFD8ED186ADDED78
:1093D800124A65EEA66AE4EE866AF0EE674AE6EEA1
:1093E800854AFDEEE46A16EE90EA714572DC9E4508
:1093F800A8BF9E4606EE90EAF8EEE66A002E00F058
:10940800BF83072ACCED066A3CF4B4AFD8ED1C6ADA
:10941800DDED134A65EEA65AE4EE865AE5EE257AA6
:10942800FDEEE77A17EE902A914203DC9A42A8BF34
:109438001A46114607EE901AF8EEE77A002E7FF4E6
:109448002AAA069B002B7FF426AA059B5B45B8BF7A
:10945800F0EE477AFFF71FBA77EEC76AF0EE477A61
:10946800FEF798BDBCF834309FED557A07EE903A78
:10947800F8EEE77A534B67EE877AC3ED007AFCF78C
:10948800D4BE514B1E6816F080567FF4BCA8FFF777
:10949800B5B84E4BFCF720BF4D4B1B78032B00F0A3
:1094A80024820023FEF7AFBE9FED4A8AFFF73BBA3E
:1094B8009FED488AFFF703BA9FED470ADFF834812A
:1094C80025EE800A22F052FBD4F8A861A8F806001D
:1094D800FBF7DDBE06EE901A8EE706EE901AE2E67E
:1094E80006EE901A67E706EE901A42E706EE901A23
:1094F8001DE706EE901AF8E63849394A8C46FEF719
:1095080030BB93ED000A05930791069222F02EFBDB
:10951800DFF8E4E0DFF8E4C0DEF8ECE0DFF8D48060
:10952800069AA8F800008CFB0E3C4FEAEE7ECEEBC4
:10953800AC1E07EE90EAF8EEE77A059B0799FDEE78
:10954800E77A17EE900AA8F80200FCF7CABE07EE01
:10955800907AF8EEE78ADFED237A9FED2C0A84F8FB
:10956800847168EEA78A38EE800AFDEEC07A17EE9D
:10957800903A2033402B40F29F819FED160A114B01
:10958800FDEEE87A83ED010A17EE903A2033402B7E
:1095980000F29581DFED1E7AF4EEE78AF1EE10FA1B
:1095A80040F3D481DFED176ADFED0F7A3AE000BFB0
:1095B80084F9223F92E741B99730083C15A82ABEA2
:1095C8006F12833A780000208C330020543E00202C
:1095D800476C0020000000000000C842243B002027
:1095E800A820002035FA8E3CE4CB164144540020D4
:1095F80014340020303E002020080020D34D621093
:10960800DB0F49C0DB0FC940E4CB16C1DB0FC93FF4
:10961800DB0F494092E741B99730083C15A82ABEAC
:10962800F0EE478AF4EEE78AF1EE10FA38EEE67AC1
:10963800F6DC5FED0D7AB4EEE77AF1EE10FA40F160
:1096480082811FED106A5FED106A01E0B0EE677A63
:10965800B4EEE67AF1EE10FA77EE067AF6D41FED5C
:10966800157AF4EEC77AF1EE10FA40F32F811FED68
:10967800187A77EE677A27EEA76A5FED1A5A5FEDD8
:109688001A6A1FED1A7AE6EE256A67EE865AA6EE82
:10969800267AE5EE877AC4ED627AFDF7B4BE06EE67
:1096A800901ADCE503F0A0F9CB4BDFF874831F7840
:1096B800069BC01AA8F80200FEF781BAFDEEC74A59
:1096C8000DF1300E9A46DFF85CC3DFF85C8314EEC8
:1096D800901A0EEB82024B4606E07245E8EC014A0E
:1096E8000CF1100C3CF446AEDCED004ABEEC014A2D
:1096F80065EEA44AE6EE044AB0EE674AA5EE244AAF
:10970800F0EE444A33B1F4EE446AF1EE10FAC8BF01
:10971800F0EE474AFDEEE44A14EE909A494504EE0D
:10972800901A04DCD145A8BFD14604EE909AF8EE11
:10973800E44A002ED1D106980028CED10598584584
:10974800B8BFF0EE474AC8E703F04EF9069BDFF8CA
:10975800D082D4F8AC91D4F8A861C01AA8F8020055
:10976800FEF78FBA03F040F99B4BDFF8B4821F78FD
:10977800069B99F80020D4F8A861C01AA8F804003C
:10978800FEF7DDBB08980FF053FAFEF7E4BDDFEDF6
:10979800937AF4EEE76AF1EE10FA40F3EE81DFED2A
:1097A800905A9FED906A01E0F0EE676AF4EEC66A9F
:1097B800F1EE10FA76EEE57AF6DCDFED8B6AF4EE80
:1097C800E67AF1EE10FA40F1D581DFED855A9FED8A
:1097D800876A01E0F0EE667AF4EEC67AF1EE10FAE6
:1097E80077EEA56AF6D4DFED827AF4EEE76AF1EE59
:1097F80010FA04DDDFED797A77EEE66A03E5DFED4E
:109808007D7AF4EEE76AF1EE10FA44BFDFED767A7E
:1098180077EEE66AF7E4784800F1800CFEF776BB4D
:10982800FDEEE77A17EE902A8A42FFF6E0ACD9E41B
:10983800BDEEC77A17EE100A8842BFF6B2AC07EE43
:10984800101AB3E4BDEEC77A17EE100A8842BFF6C5
:1098580083AC07EE101A84E4BDEEC77A17EE100A3F
:109868008842BFF654AC07EE101A55E4BDEEC77A2D
:1098780017EE100A8842BFF625AC07EE101A26E448
:10988800BDEEC77A17EE100A8842BFF6F6AB07EEB0
:10989800101AFFF7F7BBBDEEC77A17EE100A884219
:1098A800BFF6C6AB07EE101AFFF7C7BBA8F806004D
:1098B800A5F8B460FCF7E4BBF8F7CEFE5FE6DFED91
:1098C8004F7AE8E607EE101AFFF790BB9FED497A4A
:1098D800F4EEC77AF1EE10FA44BF9FED437A77EEC3
:1098E800677AC8E66146FFF737BB21F041F8FCF715
:1098F800BFBB802014F078FF08B107F0C9F910F059
:1099080049FAFEF7DDBC94F8E031002B7BF428AF70
:10991800FBF713BFDFF81491D9F8000007F096F9A8
:10992800374B1B780022022BC9F800207EF4C5AC07
:1099380007F0F0FBFEF7C1BC1BF80330002B7EF4E8
:10994800BFACFEF7D4BDF0EE477A88E6B0EE687A91
:109958006FE62C4A2C4B10681B689847099BDBED77
:10996800007A93ED007A294BD7ED006A83ED020A5D
:10997800274B67EE277A2B4427EE8C7AD3ED007AB3
:10998800244B67EE277AF0EE665AEDEE275A93EDF0
:10999800006AB1EE467AB4EEE57AF1EE10FA08DC28
:1099A800B4EEE56AF1EE10FA8CBFB0EE657AB0EE6F
:1099B800467A194B1B78012B02D0192B7BF447AE42
:1099C800DFED167AB4EEE7DAF1EE10FACCBF012338
:1099D8000023FBF747BE00BF2C3E0020DB0F4940A9
:1099E800DB0FC940E4CB1641DB0F49C0E4CB16C1FD
:1099F800DB0FC93FDB0FC9BFA82000200000000013
:109A0800E4350020885300209C5300209833002020
:109A1800AC5300201454002020500020000096422F
:109A2800303E00204454002014340020686D00208B
:109A380000C0F84400C0F8C45FED037AF4EEE7DA3A
:109A4800F1EE10FA20DC5FED057AF4EEE7DAF1EEDC
:109A580010FA19D44F4BD3ED007AB1EE677AB4EE11
:109A6800C7DAF1EE10FA12D4B4EEE7DAF1EE10FA32
:109A780088BFB0EE67DA484BC7ED00BA1B6893425F
:109A8800BBF6A6ADFCF7C3BE9FED44DAF3E7B0EE34
:109A980047DAF0E7069800287FF470AC0598584537
:109AA800B8BFF0EE476A69E4069800287FF444AC32
:109AB80005985845B8BFF0EE476A3DE40698002877
:109AC8007FF47EAC05985845B8BFF0EE476A77E456
:109AD800069800287FF4C8AB05985845B8BFF0EE43
:109AE800476AFFF7C1BB452020F0AAFDFF2020F000
:109AF800A7FD2B4820F090FD384620F0A1FDFEF789
:109B08000BBC802014F070FE00287DF405A9FEF738
:109B18007FBC069800287FF4EDAB05985845B8BF80
:109B2800F0EE476AFFF7E6BB069800287FF4C0AB63
:109B380005985845B8BFF0EE476AFFF7B9BB132B35
:109B480005D1B0EE480A22F011F8AAF80000B0EEEC
:109B5800480AD5F8143213489847134B1B78132B2F
:109B6800B0EE408A7BF4D4AB22F000F8AAF80200E9
:109B7800FBF7CEBBF0EE676A35E6F0EE667A1CE6D8
:109B8800069800287FF43DAC05985845B8BFF0EE1C
:109B9800476A36E410540020F45300200000000007
:109BA80038040308F06700202C3E00202DE9F04F10
:109BB800B0F908500D81EDB2442D8BB00C46164615
:109BC80000F00D8207462FD9812D00F04B8200F25C
:109BD8008180542D00F0AE8040F298816E2D00F007
:109BE800CC81802D40F0B280B54B1D780B3D15F02F
:109BF800FF0512D0B34F00220A2621683B88481C73
:109C080020600E702168FF2B02F10102A8BFFF231C
:109C1800481CAA4220600B70EFDB01252B46284622
:109C280063810BB0BDE8F08F052D00F0C6811ED80A
:109C3800022D77D040F23181032D00F09281042D5E
:109C480040F084802A46A0492046F8F7CAFB002144
:109C58002046F8F7F4FB22680021531C01252360F5
:109C680028462B46117063810BB0BDE8F08F242D78
:109C780056D040F2CA80282D00F0B981382D65D120
:109C88000A68924B0125511C216015702268052134
:109C980050192060117022680A2150192060117033
:109CA8002268002150192060117022681978501913
:109CB800206011702268597850192060117022684C
:109CC8009978531923602B461170284663810BB08D
:109CD800BDE8F08FA02D11D040F2B580B82D00F06E
:109CE800BF81FE2D32D17A4D05F1080635F8021BE9
:109CF8002046F8F7A4FBB542F8D18EE7754B084625
:109D08001968F8F785FB744B20461968F8F780FB4B
:109D1800724B196820460125F8F77AFB2B467EE737
:109D28006F4BF6E704226F4920460125F8F759FBE7
:109D38002B46CAE70B6800215A1C2260197022685A
:109D48000125531923602B461170BEE7214628468A
:109D580005F056F900287FF460AF742D00F0F48008
:109D6800772D0CD13B687A689A421BBF5A1C3A601F
:109D7800014619785C4A20461CF07CFD4DE7F52D1C
:109D880000F0C9817A683E68292DA2EB060300F02D
:109D98006C8240F24982392D01F0FE81532D40F04A
:109DA8007D82721C3A603178032900F2C4844A1E0D
:109DB8004E4D4F48D2B202EB420205EB420201700F
:109DC800557800293FF429AF013BDBB2AB4240F0A4
:109DD800B284821C00231360536013725DB1013595
:109DE8003B682844013A01333B6013F8011C02F830
:109DF800011F8242F7D13F4B1B78002B3FF40DAF78
:109E080001251FF041FA2B465FE7202D9ED10B68F4
:109E1800394D591C6A7821601A7023682A78591CB0
:109E280021601A702368AA78591C21601A70298940
:109E38002046F8F704FB23686A79591C21601A70D8
:109E48002268A97909E7822D80D10B682B4A2C4D0D
:109E58001178294A581C2060197011892046F8F792
:109E6800EEFA284B22681B88FF2B02F10101A8BFDC
:109E7800FF2321601370A96881F3100189B220467D
:109E8800F8F7DDFA296801F30F0189B22046F8F7DF
:109E9800D6FA1D4B22681978DFE6012D7FF456AFFC
:109EA8000B680022591C21601A7023685A1C226012
:109EB8001D7022682421531C23602B46117004E76F
:109EC800DA3D0020D8240020873000207D30002093
:109ED800303E0020ACF7FF1FB0F7FF1FB4F7FF1F9D
:109EE8001432002018050308555B0208F8E202083E
:109EF800D4680020982C00204C6C0020523E002092
:109F0800F05900203C3E0020476C0020522D7FF481
:109F18001DAF0A68AE4E531C0321236006F10C07DF
:109F280011703346062001212268551C25601170E6
:109F380022689F4202F101012160107000F0CC807C
:109F48009979D8790633EFE73B687A689A421BBF5C
:109F58005A1C3A60014619789E4A20461CF08AFC31
:109F68005BE60B685A1C0A601D700B680222591CBC
:109F780021601A70226800216FE6974B0A681B88D7
:109F8800964DFF2BA8BFFF23511C21601370A968B1
:109F980081F3100189B22046F8F751FA904B204618
:109FA8001988F8F74CFA296801F30F0189B220469D
:109FB8000125F8F744FA2B4687E60B228949204603
:109FC800F8F70FFA082288492046F8F70AFA012517
:109FD800072286492046F8F704FA2B4675E6002A38
:109FE8003FF41BAE824B136001252B466DE60B68D0
:109FF800DFF82C827F4E591C022221601A702368D8
:10A0080006275A1C22601F7023680A22591C2160E7
:10A018001A70236801255A1922601D70B8F80010BB
:10A028002046F8F70CFAB8F802102046F8F707FAB5
:10A0380023685A1922601F70236850225919216019
:10A048001A7023680022591921601A703188204635
:10A05800F8F7F5F971882046F8F7F1F92B4634E658
:10A06800654B56E6654B1E780A3E16F0FF063FF430
:10A07800D4AD634B634F1E4403F101080A2314E077
:10A08800502B00F0A280002529462268501C206031
:10A0980020461370F8F7D3F929462046F8F7CFF988
:10A0A80046453FF4BAAD18F8013B0A2BE8D1564AA9
:10A0B8009568116805EB85054FF6FF726D009542AE
:10A0C800A8BF15469142A8BF114625EAE57521EAC1
:10A0D800E171ADB289B2D8E74C4B21681A78481CB7
:10A0E80020600A70002A3FF498AD013AD2B202EB20
:10A0F800420206EB42025578002D3FF48EAD013541
:10A108001D440133226813F8011F501C9D42206032
:10A118001170F7D181E53B687A689A4241F04C802A
:10A128003B4BFF221A704FF000093A4D0AF042FCEF
:10A1380049462022384885F8009023F022FE8DF801
:10A1480004909DF80430072B01F29B80DFF8D4803F
:10A15800314F4A469DF8043003EB430308EBC30331
:10A168005B7CE3B19DF8043003EB430308EBC303C6
:10A1780020215B699BB19DF8043003EB430308EB96
:10A18800C303586947F82200F7F701FA2B7857F804
:10A198002300F7F7BDFB2A780132D2B22A709DF866
:10A1A80004300133DBB28DF804309DF80430072BFE
:10A1B800D0D92368591C21601A70002E3FF42DADA8
:10A1C800164B336001252B467FE5BD68396871E77A
:10A1D800F8E20208356702083C3E0020F0590020EA
:10A1E800446C0020200503082C05030838050308E3
:10A1F800DDEF0008C8240020D42E0020DA3D00201E
:10A2080004E20208CC24002094240020D468002012
:10A21800BC220020FF4E0020FC58002035F1010828
:10A22800B435002060610020212D37D13346721CDF
:10A238003A60184D13F8022B6A703B6073782B70E4
:10A24800F31C3B60B378AB703846F8F7BAF83B6854
:10A258002881591C1A46396012F8021B69713A6044
:10A268005B78AB7101252B462FE5731C3B60337877
:10A278000A2B00F0C987502B40F0F5853846F8F7CF
:10A28800A0F8054E30803846F8F79BF80125708015
:10A298002B461AE54C6C0020C82400200B3DEF2DFE
:10A2A80000F2498201A151F825F000BF91B00008E1
:10A2B8003FA700083FA700083FA700083FA70008DE
:10A2C8003FA700083FA700083FA700083FA70008CE
:10A2D8003FA700083FA700083FA700083FA70008BE
:10A2E8003FA700083FA700083FA700083FA70008AE
:10A2F8003FA700083FA700083FA700083FA700089E
:10A308003FA700083FA700083FA70008FFAF0008C5
:10A318003FA7000887B100083FA7000865B10008FB
:10A328003FA700083FA700083FA700083DB1000865
:10A338003FA70008C7B000083FA70008CDAF000836
:10A348003FA70008A7AF00083FA7000895AF00087F
:10A358003FA7000841AF00083FA70008B5AE0008B6
:10A368003FA700083FA700083FA700083FA700082D
:10A37800239C00083FA7000899AE00083FA70008E3
:10A388003FA700087FAE00083FA7000825AE0008D9
:10A398003FA700083FA700083FA700083FA70008FD
:10A3A8003FA700083FA700083FA700083FA70008ED
:10A3B80001AF00083FA70008D7AD00083FA7000875
:10A3C8003FA7000899AD00083FA700083FA700086D
:10A3D8003FA700083FA700083FA700083FA70008BD
:10A3E8003FA70008CDAC00083FA7000817AC00083D
:10A3F8003FA700086DAB00083FA70008CBAA0008DC
:10A408003FA70008A3AA000885AA00083FA70008DC
:10A418003FA700083FA700083FA700083FA700087C
:10A428003FA700083FA700083FA700083FA700086C
:10A438003FA700083FA700083FA700083FA700085C
:10A448003FA700083FA700083FA700083FA700084C
:10A458003FA700083FA700083FA700083FA700083C
:10A468003FA700083FA700083FA700083FA700082C
:10A478003FA700083FA700083FA700083FA700081C
:10A488003FA700083FA700083FA700083FA700080C
:10A498003FA700083FA700083FA700083FA70008FC
:10A4A8003FA700083FA700083FA700083FA70008EC
:10A4B8003FA700083FA700083FA700083FA70008DC
:10A4C8003FA700083FA700083FA700083FA70008CC
:10A4D8003FA700083FA700083FA700083FA70008BC
:10A4E8003FA700083FA700083FA700083FA70008AC
:10A4F8003FA700083FA700083FA700083FA700089C
:10A508003FA700083FA700083FA700083FA700088B
:10A518003FA700083FA700083FA700083FA700087B
:10A528003FA700083FA700083FA700083FA700086B
:10A538003FA700083FA700083FA700083FA700085B
:10A548003FA700083FA700083FA700083FA700084B
:10A558003FA700083FA700083FA700085BAA00081C
:10A568003FA7000845AA00083FA700083FA7000822
:10A578003FA700083FA700083FA700083FA700081B
:10A588003FA700083FA700083FA700083FA700080B
:10A598003FA700083FA700083FA700083FA70008FB
:10A5A800E9A900083FA70008B1A900083FA70008CB
:10A5B800D5A80008BBA800089FA800083FA7000866
:10A5C80085A800083FA700085DA800083FA7000865
:10A5D80003A800083FA70008D5A700083FA7000860
:10A5E8003FA70008B3A7000885A7000871A70008BF
:10A5F80049A7000821A70008FFA600083FA70008F0
:10A608003FA700083FA700083FA700083FA700088A
:10A618003FA700083FA700083FA700083FA700087A
:10A628003FA700083FA700083FA700083FA700086A
:10A638003FA700083FA700083FA70008E5A60008B5
:10A648003FA700083FA700088DA600083FA70008FD
:10A658003FA700083FA700083FA700083FA700083A
:10A668003FA700083FA7000875A60008BE4B1B7847
:10A67800DB0760D4012505F0DFFC01F0CDFA2B469D
:10A68800FFF723BB731C3B6033780F2B53D8B21CE6
:10A698003A60C3EBC303B54A7178D154F11C3960F1
:10A6A8001344B2785A70321D3A60F2789A70721D6B
:10A6B8003A603279DA70B21D3A6072791A71F21D15
:10A6C8003A60B2795A7106F108023A60F2799A71E1
:10A6D800012515F00DFC2B46FFF7F7BA3846F7F7BA
:10A6E80070FEA34EF0813846F7F76BFE0125B08166
:10A6F8002B46FFF7EABA3846F7F763FE9D4E3082DD
:10A708003846F7F75EFE70823846F7F75AFE01259D
:10A71800B0822B46FFF7D9BA3346721C3A6013F859
:10A72800020B3B60F31C71783B60B2781BF09AF91E
:10A7380000287FF472AA4FF0FF352B46FFF7C5BA01
:10A748003346721C3A608C4A13F8021B11703B6046
:10A75800874A73789370F31C3B60884BB2789A7081
:10A7680001252B46FFF7B1BA854B864918684E225A
:10A77800012521F087F82B46FFF7A7BA3246731C4C
:10A788003B60814B12F8021B19703A6072785A705C
:10A79800F21C3A60B2789A703846F7F712FE7B4B93
:10A7A8000125D8802B46FFF790BA3846F7F709FEFF
:10A7B800764E30803846F7F704FE70803846F7F753
:10A7C80000FE0125B0802B46FFF77FBADFF8CC8169
:10A7D80098F80030002B3FF420AA6D4E002538462B
:10A7E800F7F7EFFD16F088FB98F80030A6EC010AA1
:10A7F80001359D42F3DBFFF710BA0D2B9BD1731C7B
:10A808003B603578072D96D8DFF8948138460C26BA
:10A81800F7F7D7FD06FB05F608EB0605A8803846CE
:10A82800F7F7CFFDE8803846F7F7CBFD3B6828817E
:10A838001A46591C396012F8021BA9723A605B78F3
:10A84800EB723846F7F7A6FD012548F806002B46B7
:10A85800FFF73BBA731C3B603078060600F11F8592
:10A86800414B1B78DD073FF5D8A9032828BF0020F6
:10A87800012505F0ABFB2B46FFF727BA3A4B1B78AF
:10A88800D8073FF5CAA9012505F0CAFB01F0C4F9AC
:10A898002B46FFF71ABA344B1B78DA073FF5BDA9E8
:10A8A8003C4A1378012543F0040313702B46FFF745
:10A8B8000CBA2D4B1B78D9073FF5AFA9364B4FF48F
:10A8C800C87201251A802B46FFF7FFB9092B7FF7BD
:10A8D80032AFDFF8D0803346721CD8F800503A60A7
:10A8E80013F8022B2A703B607378AB70F31C3B6043
:10A8F800B378642BA8BF6423321D6B713A60F37878
:10A90800642BA8BF6423721DAB713A603379EB7175
:10A91800B31D3B607379642BA8BF6423F21D2B72AF
:10A928003A60B379EB7006F108033B60F3792B7159
:10A938003846F7F746FD7A683B686881D11A0029DE
:10A948000CDD591CD8F800003960521A002A197811
:10A95800417203DD9A1C3A605B78437001250CF064
:10A96800FFFB2B46FFF7B1B95B5F002020510020A9
:10A97800C4350020206200200C550020D43500206A
:10A988009430002050FC0208BC350020CC54002034
:10A9980024540020943300205E300020DA3D00204B
:10A9A8002C50002040300020B94B1868F31C024698
:10A9B8002136991E396013F8031C1170591E39602D
:10A9C80013F8021C51703B6013F8011C917003339B
:10A9D800B34202F10302ECD116F05EF9FFF71DB99C
:10A9E800C3F34705122D3FF6A6AEBDB10AAB0DF174
:10A9F800020803EB45094646A9F126093846F7F748
:10AA0800E0FC26F8020FB145F8D1A24B38F8022F26
:10AA180023F8022F4645F9D1112D09D89E4A6B001B
:10AA2800023B13440021223223F8021F9A42FBD131
:10AA38009A4A01231D461370FFF747B9984E002321
:10AA480038463360F7F7A6FC012530602B46FFF740
:10AA58003CB93346721C3A6013F8025B3B60F31C46
:10AA680070783B60B178002D00F05A84012D7FF496
:10AA7800D4A807F0ADF82B46FFF727B9894B1B7808
:10AA880013F001017FF457AE731C3B603078012549
:10AA980006F0E0FF2B46FFF718B93346721C3A6000
:10AAA800814A13F8021BD1703B60804A7378537156
:10AAB800F31C3B607E4BB278DA7001252B46FFF71A
:10AAC80004B93846F7F77DFC3846F7F77AFC38467C
:10AAD800F7F777FC3846F7F77FFC3B686C4D19466B
:10AAE800581C2A68386011F8020B82F82C0039606B
:10AAF800597882F83610D91C39609B7882F837303B
:10AB08003846F7F769FC3846F7F766FC3846F7F732
:10AB180063FC38462E68F7F754FC708738462E6871
:10AB2800F7F74FFC3B687A683087D11A01290ADDAC
:10AB3800591C2A6839601B7882F82E303846F7F796
:10AB48004BFC3B687A68D31A032B09DD38462E681C
:10AB5800F7F737FC708638462E68F7F732FCB08670
:10AB6800286839E7731C3B60494DDFF85481337816
:10AB780088F8053038462E68F7F723FC30843846C5
:10AB88002E68F7F71EFC7A683B68F083D11A07290C
:10AB980015DD3846F7F715FCA8F80A003846F7F728
:10ABA80010FCA8F80C0038462E68F7F70AFC7084E9
:10ABB80038462E68F7F705FC3B687A68B084D11AE6
:10ABC80003290BDD3846F7F7FCFBA8F80E003846DA
:10ABD800F7F7F7FB3B687A68A8F81000D21A002A42
:10ABE80005DD591C2A6839601B7882F8263000F088
:10ABF80075FF17F0EBF92F4B1B68002B00F044830F
:10AC08002868012515F02CFD2B46FFF75EB8334662
:10AC1800721C3A60DFF8A88013F8022B88F802202B
:10AC28003B60254A73781370F31C3B60234DB3785F
:10AC38002B71331D3B60F378092BA8BF09233846D5
:10AC4800AB70F7F7BEFB3B687A682880D11A0129F8
:10AC580005DD3846F7F7B5FB3B687A68E8819A4224
:10AC680007D05A1C3A601B78003318BF012388F8B4
:10AC7800073000F033FF3B687A689A423EF4CDAF64
:10AC88005A1C3A601B78EB7001252B46FFF71DB85C
:10AC980094300020FE57002000580020245800203F
:10ACA800D42E00205B5F0020C4350020B45E002055
:10ACB800D4350020E8350020B83500202062002077
:10ACC8000C5500203846F7F77CFB05461FF0C2FA02
:10ACD800FF283EF4A2AF3F2D00F2EC820DF12808C8
:10ACE800002308F8243DEE0841460DF103008DF8D5
:10ACF800033001361FF0B2F99DF80330F6B205F0C3
:10AD08000705B34205F1010503D19DF80430AB42B4
:10AD180003D0294630461FF089FA3B687A68D21A70
:10AD2800012A7EF77AAF5A1C0AA83A6000221D78D9
:10AD380000F8252D1FF086F99DF80330AB420AD0A4
:10AD4800C14B1B683BB19A79AA4204D31B681B69A3
:10AD58000BB1284698473B685A1C3A604046002287
:10AD68001D788DF804201FF061F99DF80430AB427E
:10AD78003EF453AFB44B1B68002B3EF44EAF1B6838
:10AD88005B69002B3EF449AF28469847FEF745BF5C
:10AD9800AE4B1B78012B3EF640AF731C31463B602F
:10ADA800DFF8DC8211F8023B88F80230F31CD21A73
:10ADB8003960012A70783B6040F3B8823846F7F76B
:10ADC80000FB0125A8F800002B46FEF77EBF731C88
:10ADD8003B6096F80080B8F1110F3FF6ACACB31C9D
:10ADE8003B609B4D737805F818303846F7F7E9FA59
:10ADF80040F6CA039842A8BF184640F2EE2398428C
:10AE080005EB4801B8BF18460125A0F2EE222B46F3
:10AE1800192092FBF0F24A70FEF757BF731C3B6093
:10AE28008C4B3278DFF85C821A700023C8F8003047
:10AE38003846F7F7AFFA3A68D8F800308649874DB0
:10AE48000343501CC8F80030386013780B7238463A
:10AE5800F7F7B7FA28603846F7F7B3FA6860384664
:10AE6800F7F7AFFAA8603846F7F7ABFA3846F7F7BE
:10AE7800A8FAFEF7D2BE7A4B06F1080201363E6008
:10AE880016F8011C03F8011FB242F7D1FEF7C5BE40
:10AE98003346721C3A60734A13F8021B91703B6088
:10AEA8007378537001252B46FEF70FBF0722B3FBBB
:10AEB800F2F2C2EBC2015B1A7FF43DACD2B202F1EE
:10AEC800FF385FFA88F8002A3EF4A7AEDFF898B199
:10AED80008F101089946731C3B6096F90010624B13
:10AEE800002593F902208A4203F1080300F0A381A8
:10AEF8000135042DF5D11EE43346721C5B4D3A60D2
:10AF080013F8022B2A713B6073786B713846F7F798
:10AF180058FA3B6828805A1C3A601B78AB7138464F
:10AF2800F7F74FFA3B6868805A1C3A601B78EB7158
:10AF380001252B46FEF7C9BE731C3B6033780E2BE8
:10AF48003FF6F9ABB21C3A60707803283FF6F3ABD2
:10AF58004749062202FB03F28B18F51C58713D6025
:10AF6800B0788854321D3A60F2785A70721D3A608F
:10AF780032799A70B21D3A607279DA70F21D3A60CD
:10AF8800B2791A7101252B46FEF79FBE731C3B60F0
:10AF9800314B32785A7501252B46FEF796BE721C46
:10AFA8003A6035781F2D3FF6C6AB052B7FF4C3AB4F
:10AFB8003846F7F7EFF92F4B43F825001EF0A0FFAE
:10AFC800FEF72BBE2B4D05F140063846F7F7F9F989
:10AFD8003B68A5F88000591C1A46396012F8021B14
:10AFE80085F882103A605B7885F883300435AE4284
:10AFF800EBD1FEF712BE731C3B603578132D3FF67C
:10B008009AABB31C3B6070781BF06EFC00283FF4D1
:10B0180092AB194B027803F82520F21C3A6003EB37
:10B028008503B2785A70321D3A60F2789A70721DB0
:10B038003A6012493279DA70086801250CF01EF876
:10B048002B46FEF742BE00BFD86C0020DF3100203F
:10B05800C859002000360020404200207C2C0020E7
:10B068003F420020E0350020D06B0020E45400204F
:10B07800E02E0020BC5C0020083600209430002020
:10B08800E231002014320020AF49102B4FF00002AB
:10B0980028BF10230A604A608A60CA600A74002BBD
:10B0A8003EF4BBAD3A680139134401323A6012F8F4
:10B0B800010C01F8010F9342F7D1FEF7AEBD731CE6
:10B0C800A24D3B6033782B723846F7F77AF9A8839C
:10B0D8003846F7F776F928833846F7F772F93A6869
:10B0E8006883531C3B601278EA747A68D31A032B7E
:10B0F80000F3F7803B68D11A05290EDD5A1C3A6027
:10B108001B78EB723846F7F745F93B68E8605A1C3C
:10B118003A601B782B743B687A68D21A002A7EF74B
:10B128007CAD5A1C3A601B7885F8213001252B46E6
:10B13800FEF7CBBD731C3B60854930780870D21A86
:10B14800002A7EF76AADB31C3B607378003318BFE2
:10B15800012301254B702B46FEF7B7BD3846F7F79C
:10B1680030F97C4E30603846F7F72BF97060384676
:10B17800F7F727F90125B0602B46FEF7A6BD764EF6
:10B18800002333603846F7F705F933680125034390
:10B1980033602B46FEF799BD731C3B6033780A2B4E
:10B1A80038D03846F7F718F93846F7F715F938461A
:10B1B800F7F712F9FEF731BD5A1C19463A6067488D
:10B1C80011F8022B027039605B784370042A06D9A3
:10B1D800FF2A3EF4A8AF22680021FEF73EBD604971
:10B1E8000978994203D8022AF5D1FF2BF3D12368B5
:10B1F80001255A1922601D70002E3EF40EAD594BE0
:10B2080033602B46FEF761BD3846F7F7DAF8564E3D
:10B21800FFF738B8B31C3B60544B72781A70F21CB5
:10B228003A60B2785A70321D3A60F2789A70012505
:10B238002B46FEF74ABD0BEBC50A38468AF80210C2
:10B24800F7F7BFF83B682BF835001A46591C3960E8
:10B2580012F8021B8AF803103A605A788AF8042018
:10B26800DA1C3A609A788AF806201E1D3E6009F1B9
:10B278000109DB788AF80530C8457FF42CAEFEF763
:10B28800CCBC4A46FEF795BF39483A493A4A3B4B47
:10B29800036001250B6013602B46FEF716BD00F016
:10B2A8007F00032828BF0020012506F0ADFC2B46AF
:10B2B800FEF70BBD0DF1040840461EF0ABFEBDF8CD
:10B2C8000430AB423FF429AD2D4B1B68002B3FF4F3
:10B2D80024AD1B689B69002B3FF41FAD2846984797
:10B2E8001BE53846F7F76DF8A8843846F7F769F88C
:10B2F8003B687A68E884D11A03297FF7FCAE1A46BE
:10B30800591C396012F8021BA9773A605B7885F8F6
:10B3180020303846F7F755F83B687A686884EAE6DB
:10B32800012515F031FB2B46FEF7CFBC154BB17844
:10B338001A88012512FB00F22B4692FBF1F2A8F8BD
:10B348000020FEF7C2BC00BFA0350020404200200C
:10B35800003600207C2C002014320020BC22002063
:10B36800DA3D0020F5EF0008B43500207D300020DC
:10B37800E0520020345300209C530020430500086D
:10B38800D86C0020806D00200B4B002210B4027294
:10B3980003F1DC04012102E0072A09DC9979890715
:10B3A80002D51979815401329C4203F11403F3D177
:10B3B8005DF8044B704700BF600103081F2303704A
:10B3C800704700BF012310B41521142422224470B1
:10B3D8004171C2700370037183705DF8044B70474C
:10B3E8002DE9F0410B78057BDB43DFB200F1130256
:10B3F80000F11D0302F8015F9342FBD1DFF890E0F2
:10B4080000F12701002203F8012F9942FBD11421F2
:10B418000524002647FA04F303F00103002B1E4419
:10B4280014BF4FF019084FF00A0814F0010FF6B2D4
:10B4380014BFAC464FF0000C0023CA1810FA82F271
:10B448000133434582F814C0F7D15A1E92B2013233
:10B45800013C8B18621C9BB201D01946DAE716F042
:10B46800010F14BF19240A240022991810FA81F137
:10B478000132A2420D75F8D113449BB25A1C034401
:10B48800002192B21975AEF800200261BDE8F08182
:10B49800C02200202DE9F04FDFF890A0BAF8023062
:10B4A8000B3383B01FFA83F901F1060B4FF0010843
:10B4B8004FF0000C002711F801EB3E464C460122E4
:10B4C800A4F10B039BB2019105E001339BB2017B10
:10B4D80029759C4208D0C518002AF6D1C518013331
:10B4E8009BB29C422A75F6D103190136092F01999E
:10B4F80083F814C0F6B20CD0092E15D008FA07F359
:10B5080013EA0E0F14BF012200220C34A4B2013733
:10B51800D6E709F1780959451FFA89F9CAD1AAF875
:10B5280002C003B0BDE8F08F0022EEE7C022002081
:10B538002DE9F047DFF85C80B8F8043004331FFACF
:10B5480083FC01F109094FF0010E11F8017B6446F3
:10B558000026231F0EFA06F29BB23A40C2B1B0F899
:10B568000CA0C51801339BB29C4285F814A0F5D1F4
:10B5780001360434082EA4B2EBD10CF1200C494555
:10B588001FFA8CFCE1D10023A8F80430BDE8F0874D
:10B598009246E6E7C022002010B40268047B1168D6
:10B5A8000223A340194209D00649406800240C70C0
:10B5B80001684FF6FE742140016053605DF8044B4A
:10B5C800704700BFD3680020436A8269D154436A38
:10B5D8000169426B01338B4228BF00234362002A72
:10B5E8002FD0EFF31181502383F31288436B1A682D
:10B5F800D2072CD470B45E686EB9456A826A9542E7
:10B6080017D084691444DC600ED9AA1A5A6085627E
:10B61800002280F850201A6842F00102C9B21A606C
:10B6280081F3118870BC70470469A21A5A60866257
:10B63800EEE7012380F85030C9B281F3118870BC5D
:10B648007047C26C136843F0800313607047C9B237
:10B6580081F31188704700BF026B10B462B1036CAC
:10B66800C2684469D11A013B615C5DF8044B08BFAC
:10B6780013460364C8B27047016A4369C4685B5CD7
:10B688000131A14228BF114601625DF8044BD8B2CE
:10B69800704700BF436B13B190F850007047836A3E
:10B6A800406A181AB0FA80F040097047416A836A04
:10B6B80099420AD3CB1A416B026961B14968501E9D
:10B6C8000B4483420AD2C01A704702691144CB1A4C
:10B6D800416B0029F2D1501EC01A704700207047F4
:10B6E800036B43B1026C5B6893422FBF981AC06822
:10B6F8009B1AC0187047C269036A9A422FBFD01AB2
:10B70800C0688018C01A70472DE9F0470569C368FA
:10B718001D4028D00F4606464FF000484FF000095C
:10B72800B5FA85F328FA03F2D2431B3B3261154080
:10B73800042B16D8DFE803F03129211903007B6AAE
:10B74800002B32D003F1FF3A1FFA8AFAC7F8249087
:10B758003C6A34B123682046514698476468002CF7
:10B76800F8D1002DDCD1BDE8F0873868716B03682B
:10B7780089B29847002DD3D1F5E77868B16B036893
:10B7880089B29847002DCBD1EDE7B868F16B036813
:10B7980089B29847002DC3D1E5E7F868316C036892
:10B7A80089B29847002DBBD1DDE7F36A1FFA83FA07
:10B7B800CEE700BF2DE9F04F013085B0C3B2039347
:10B7C8008E4D8F4F8F4C904E0A230293DFF8409294
:10B7D80016F040F94FF4FA7A4FF0100C4FF47A70E3
:10B7E800D9F80430C3F30803002B40F0C880EFF306
:10B7F8001183002B40F0C3802968A26800BF2B6822
:10B808009942F9D1D7F800E000FB0EF39B1AB3FB7D
:10B81800FEF300FB01314FF0010E0191D9F804301D
:10B82800C3F30803002B40F08E80EFF31183002B45
:10B8380040F089802B68A16800BF2A689342F9D13B
:10B84800D7F800B000FB0BF2521AB2FBFBF200FB78
:10B858000323019A9B1AB3F57A7FDFD3BAF1010A61
:10B86800BED1039B002B40F0C4804FF47A7ADFF8F6
:10B87800A09150464FF0100CD9F80430C3F30803D8
:10B88800002B40F09980EFF31183002B40F0948057
:10B898002968A26800BF2B689942F9D1D7F800E05F
:10B8A80000FB0EF39B1AB3FBFEF300FB01314FF0D4
:10B8B800010E0191D9F80430C3F308033BBBEFF341
:10B8C800118323BB2B68A16800BF2A689342F9D172
:10B8D800D7F800B000FB0BF2521AB2FBFBF200FBE8
:10B8E8000323019A9B1AB3F57A7FE3D3BAF1010ACD
:10B8F800C2D1029B013B02937FF468AF4349444B9A
:10B908004448454A0860DA6005B0BDE8F08FEFF3B7
:10B9180011888CF31288A1682368DB0344BFC6F83A
:10B9280000E0A1682B6832685FFA88F888F311880C
:10B93800D7F800801A4400FB08F35B1AB3FBF8F34E
:10B9480000FB0233CDE7EFF311888CF31288A1686E
:10B958002368DB0344BFC6F800E0A1682B6832689F
:10B968005FFA88F888F31188D7F800801A4400FB3A
:10B9780008F35B1AB3FBF8F300FB023369E7EFF354
:10B9880011828CF31288D4F808E02368D90303D510
:10B9980001233360D4F808E02B683168D2B282F30F
:10B9A80011883A68194400FB02F3A3EB0E03B3FBBA
:10B9B800F2F300FB01312EE7EFF311828CF31288CA
:10B9C800D4F808E02368D90303D501233360D4F8F9
:10B9D80008E02B683168D2B282F311883A681944BA
:10B9E80000FB02F3A3EB0E03B3FBF2F300FB013100
:10B9F8005DE718461CF0E6FB37E700BF84650020CA
:10BA08008865002010E000E080650020FC9F002091
:10BA180000ED00E0EFBEADDE0400FA0530B50446E7
:10BA2800C06C61710368A26823F00103036087B0EA
:10BA3800A379009213F004023DD04FF4805213F022
:10BA48000203019244D102934FF4806300220393CE
:10BA580011F00103059237D1049308238D07694635
:10BA680048BF04931BF01CFD6079E36CA17900F0DA
:10BA78000202002A15BF4FF440324FF480324FF4CF
:10BA88000034002410F0010F586808BF2246CC0784
:10BA98004CBF024320EA02025A609A6809074CBF69
:10BAA80042F0080222F008029A601A6842F0010285
:10BAB8001A6007B030BD13F0020301920BD04FF4A7
:10BAC800005513460295C1E7042304930C23C5E7E8
:10BAD8004FF40053B7E70293B8E700BF38B5434BBC
:10BAE8005A899989914224BF00225A81198ADA8990
:10BAF800914224BF0022DA81DA788AB3072A2FD04C
:10BB08003B493C4D91F85700012400210A282C702C
:10BB18009C70D9713DD00C2865D0DFED377A8ABB8F
:10BB2800364C9FED370AA278002918BFF0EE407A0C
:10BB3800062A04D8334901EB820191ED000A2179E4
:10BB480059B3013A032A4DD8F7EE007A87EE800AF6
:10BB580020F00CF82388984228BF1846208038BD6A
:10BB6800D97921B198780428B8BF04209870204862
:10BB780090F857000A280CD00C28CED1DFED227A95
:10BB8800002ACDD0072ACBD00A282CD1DFED1F7A86
:10BB9800C6E70A20DFED1E7AC1E79B78154A07EE53
:10BBA800103A1178B8EEC77A27EE277A07EE901A7E
:10BBB800F8EEE77A67EE877AB4EEE70AF1EE10FA64
:10BBC80010DDC0EE077AFDEEE77A17EE903A102BFB
:10BBD800A8BF1023012BB8BF0123DBB28B4238BFAB
:10BBE8000B46137038BDDFED0B7A99E70C55002032
:10BBF800D8650020B83500206F1203392062002074
:10BC08006F12033808E202080AD7A3390F506E3AB8
:10BC18005304E9386F12833A2DE9F047B34FB44E15
:10BC28000FF0BAFFBE421ED2DFF84C83DFF84C9308
:10BC38004446258862197DB14A450DD2052D0BD998
:10BC480033886188C3F30B03994200F0FD801446E2
:10BC580025886219002DEFD1716830461436F6F741
:10BC680027F9BE42E4D3A34A1378A3F117010229A6
:10BC78000FD9A14911F83300002840F00781D800F6
:10BC88000144497829B19D4911F83330002B00F05F
:10BC980025819B4C6378022B84BF00236370237833
:10BCA800022B84BF00232370964B9A78042A00F055
:10BCB8000C8132B91A88B2F5F07F84BF4FF4F07264
:10BCC8001A80914D914A2B681A40002A00F0098188
:10BCD800D80700F1F580590400F1ED801A0700F14A
:10BCE800E5809B0400F1DB80894D2B685A8C998C88
:10BCF800914224BF00225A84FFF7F0FE11F012FF90
:10BD080010B9844804F046FA4020F6F707F9802075
:10BD1800F6F704F94FF40070F6F700F94FF4003025
:10BD2800F6F7FCF84FF48020F6F7F8F84FF00070BB
:10BD3800F6F7F4F84FF08060F6F7F0F84FF000608F
:10BD4800F6F7ECF86378022B06D8734A734903EBCD
:10BD5800430302EB83030B602378022B07D803EB22
:10BD680083016F4AC3EBC10302EB43032B600BF063
:10BD7800F7F9002130226B4822F003F8286814F004
:10BD88001FFE694B2E6803F1500102E0043399420B
:10BD98007AD01A78002AF9D19C78D8788442F5D2DA
:10BDA8006249634B91F804E06248634D5C6B634BF6
:10BDB8002860C827642111FB0E71DFF8C4E15960BF
:10BDC8005F4F30F8061C5F4DAEF8001000219960F7
:10BDD800D960196159619961D96183F8201083F894
:10BDE80021103A702E600CB10FF016FD564B9FEDE6
:10BDF800575A1B88564A9FED576A557B564C5749E8
:10BE08005748086006EE903AF8EEE66A1389C5EEE0
:10BE1800265A07EE103A5389127BC4ED005A07EEF2
:10BE2800903AB8EEC77A4F4BF8EEE77A1D725A721D
:10BE380027EE067A67EE867ABDE8F04783ED017A49
:10BE4800C3ED007A0FF090BE63799B077FF4FFAED5
:10BE5800716894F804A03046F6F72AF83388BAEBEC
:10BE6800133F04D01436BE42FFF4E2AEFBE67388FB
:10BE78007068AA1FC3F30B039A4204F10601A8BF16
:10BE88001A461FF0FFFCEDE7012289E7D8000C18DD
:10BE98006468002C7FF4F4AE17241470F0E632487E
:10BEA800F6F73CF84020F6F739F81DE72F48F6F783
:10BEB80035F82B6815E72E48F6F730F82B680DE7AC
:10BEC8002C48F6F72BF82B6805E79A8AB2F57A7FA3
:10BED800BFF4F7AE4FF47A729A82F2E61823137021
:10BEE800D7E643F001032B60F2E600BF2C390308C4
:10BEF8000835030800360020A8F70208E0FA02080F
:10BF080082300020206200201432002009600002E4
:10BF180094300020D06B0020AA310020403000204F
:10BF2800A23000208823002008360020E454002096
:10BF3800BC330020CA3500201C5F00205C6C002048
:10BF4800E0000020BC230020B8210020C0C9FB4825
:10BF5800C022002017B7D138BC210020C4520020CD
:10BF68003661023DA0520020094000020160000233
:10BF7800092000020860000202F00308000004081B
:10BF8800B83C002038B50C4C0C4DAC4206D2616868
:10BF980020461434F5F78CFFAC42F8D3084A094B15
:10BFA800094C1460002209491A705A700848086040
:10BFB800BDE838401DF0A4BF083503082C39030834
:10BFC8009430002082300020A23000204030002031
:10BFD800AA310020F0B50C292BD8DFE801F06F2A30
:10BFE8002A2A4C2A2A2A2B2A2A2A0700046AB2F863
:10BFF8000CE097881668674D24F480540462036A3D
:10C008004468C16923F4005343EA0E3321F4E6413E
:10C01800A84243EA073341EA062100F0B58005F556
:10C028000065A84200F0B08092684460C161026473
:10C038000362F0BD046A96899588D2F800E0554FEE
:10C0480024F480740462036A4468C16923F40073A9
:10C0580043EA062321F07301B84243EA052341EA83
:10C068000E017ED04C4DA8427BD092684460C161DD
:10C07800C2630362F0BD046A96899588D2F800E02D
:10C08800444F24F010040462036A4468816923F071
:10C09800200321F0807143EA061321F4E641B842F7
:10C0A80043EA051341EA0E2148D03B4DA84245D04A
:10C0B80092684460816182630362F0BD046A938977
:10C0C800B2F804E01768334E24F001040462056AEC
:10C0D8004468816943EA0E0321F4803125F00205A2
:10C0E8009BB221F07301B04243EA050341EA07011C
:10C0F80014D0294DA84211D005F54065A8420DD0AD
:10C1080005F58065A84209D005F58065A84205D0E7
:10C1180092684460816142630362F0BDD689158AE2
:10C12800578A23F0080333433D43D68824F44074E8
:10C1380023F00403ADB233432C43E9E7D589178ACA
:10C14800D68823F0800343EA051324F44064558A13
:10C1580023F0400344EA870443EA061344EA8504CB
:10C16800A6E7D589178AD68823F4006343EA05230E
:10C1780024F44054558A23F4806344EA071443EABC
:10C18800062344EA051470E7158A24F4804444EA37
:10C19800851449E7002C0140003401402DE9F04F97
:10C1A800C822002183B07848784CDFF80492784D93
:10C1B800784E794FDFF8FC8121F0E3FD7748784924
:10C1C800DFF8F4E1DFF8F4C100221359834200F0EC
:10C1D800C180B3F1804F00F0BF80AB4200F0C8804F
:10C1E800B34200F0C780BB4200F0C680734500F040
:10C1F800C580634500F0C480434500F0C380DFF884
:10C20800C0A153457ED00AF5806A534508BF09236B
:10C2180079D01432F02AD8D15C4C624D624E604F0E
:10C2280004F1F00802E01434A04568D0A379002B8B
:10C23800F9D023794FEA131909F1FF39B9F1050F3C
:10C2480003F00F03EFD835F8190040FA03F2D207CC
:10C25800E9D54FF0010A0AFA03F3013B18401FF031
:10C26800E7F916F809305149184411EBC002DAD041
:10C2780051F83000DFF84CE1217A00F138439B0A8D
:10C288001EF8033003F01F0E5B09022B0AFA0EFAA0
:10C2980069D0032B62D0012B03D17B694AEA0303DF
:10C2A8007B6193880093B3FA83F3C3F11F039BB2B6
:10C2B800DA0800EB820203F00703D2F820E09B00C3
:10C2C8004FF00F0C0CFA03FC2EEA0C0EC2F820E01B
:10C2D800D2F820E001FA03F343EA0E031362694639
:10C2E8000023022214348DF804208DF805308DF8CF
:10C2F80006308DF807301BF02FF9A04596D103B012
:10C30800BDE8F08F082309EBC3034FF0010B93F846
:10C3180020A00AF01F034FEA5A1ABAF1020F0BFACB
:10C3280003F30BD0BAF1030F0ED0DA457FF471AFE7
:10C33800D1F814A043EA0A034B616AE7D1F818A0C0
:10C3480043EA0A038B6164E7D1F81CA043EA0A03B5
:10C35800CB615EE70023D6E70123D4E7FB694AEA0D
:10C368000303FB619DE7BB694AEA0303BB6198E7E6
:10C378000223C8E70323C6E70423C4E70523C2E76B
:10C388000623C0E70723BEE7DC2D00206001030871
:10C39800000400400008004000100040002C01404C
:10C3A8000010024014010308200103083060002037
:10C3B80008E2020800400140001400400034014037
:10C3C800004401402801030801490248FFF79CB9CD
:10C3D8007C2E00200040014001490248FFF794B933
:10C3E800542E00200034014001490248FFF78CB95F
:10C3F800542E00200034014001490248FFF784B957
:10C408002C2E00200004004002494FF08040FFF726
:10C418007BB900BF042E002001490248FFF774B918
:10C42800DC2D0020002C014001490248FFF76CB9BF
:10C43800DC2D0020002C01402DE9F04104684A4D14
:10C44800A30AAB4272D009D8B3F5801F6AD04A3D1F
:10C45800AB425AD14FF0700E022608E0434DAB4272
:10C4680068D00335AB4252D14FF0C00E042647794D
:10C478004FEA970C002961D0B0006346851902275E
:10C48800D4F80C809F400CEB4503BFB2384D03F144
:10C49800040C47EA080745F8231045F82C20E76004
:10C4A800EFF31181502282F31288821905EBC20240
:10C4B800136973B313620433821905EBC202576917
:10C4C80017B11F6053690433821905EBC2029769DB
:10C4D80017B11F6093690433821905EBC202D7694B
:10C4E80017B11F60D36904330027CAB21F6082F3F3
:10C4F8001188304405EBC000036A6BB9E3684FF656
:10C50800FE721340E360BDE8F081BDE8F081BDE84C
:10C51800F08105EB0E03CFE7E36843F00103E36026
:10C52800BDE8F0814FF0480E0126A0E74FF0200E3D
:10C5380000269CE74FF0980E032698E7BF080223D1
:10C5480006FA03F0BB40DB43E768094D9BB23B406A
:10C5580087190CEB470CE3600CF1040345F82C1029
:10C5680045F823209CE700BF4B0010004D00100049
:10C57800DC2D002030B503685C4D18885C4CB4FB9A
:10C58800F2F20139013AAB4294B283B089B282B275
:10C5980066D05848834263D0B3F1804F60D0A0F58D
:10C5A800983083425CD000F58060834258D052486E
:10C5B80083425BD000F5806083427DD022F44072D4
:10C5C80000F58C3092B283421A80D9621C850ED055
:10C5D800484A93420BD002F54062934207D002F5D5
:10C5E8008062934203D002F58062934201D1002217
:10C5F8001A8601225A611A883C4992B242F0010215
:10C608008B421A8062D0B3F1804F61D03B4A93428B
:10C6180060D002F5806293425ED002F500629342D8
:10C628005CD002F5806293425AD002F59032934270
:10C6380058D002F54062934256D002F58062934288
:10C648001ED002F58062934208BF092219D002A8C1
:10C658004FF0012340F8043D1AF05EFC03B030BDF2
:10C66800254822F07002834292B2A3D101201A8099
:10C67800D9621C8558611A8892B202431A80C5E7AC
:10C6880008221F4B03EBC20301A893F821408DF841
:10C698000440012300228DF805308DF807308DF80D
:10C6A80006201AF039FC1B2CD8D1164B019301A88F
:10C6B8001AF032FC03B030BD01201A80D9621C8503
:10C6C80058611A8892B202431A809CE70022D8E780
:10C6D8000122D6E70222D4E70322D2E70422D0E7D8
:10C6E8000522CEE70622CCE70722CAE7002C014044
:10C6F80000A24A0400340140001000400004004039
:10C7080008E2020819010001204B98422DD0B0F12F
:10C71800804F2CD0A3F5943398422AD003F5806338
:10C72800984228D003F50063984226D003F5806329
:10C73800984224D003F59033984222D003F5406301
:10C74800984220D003F58063984207D003F58063B0
:10C75800984208BF092202D00020704708220C4BDB
:10C7680003EBC20393F8200070470022F7E7012289
:10C77800F5E70222F3E70322F1E70422EFE70522B7
:10C78800EDE70622EBE70722E9E700BF002C0140AE
:10C7980008E202082DE9F04F013085B0C3B20393D7
:10C7A8000B4602918B4C8C4E002B00F099808B4DE0
:10C7B8008B4FDFF8309215F04DF94FF4FA7A4FF0BD
:10C7C800100C4FF47A70D9F80430C3F30803002B27
:10C7D80040F0DE80EFF31183002B40F0D980296808
:10C7E800A26800BF2B689942F9D1D7F800E000FB96
:10C7F8000EF39B1AB3FBFEF300FB01314FF0010E61
:10C808000191D9F80430C3F30803002B40F0878066
:10C81800EFF31183002B40F082802B68A16800BFE2
:10C828002A689342F9D1D7F800B000FB0BF2521AEC
:10C83800B2FBFBF200FB0323019A9B1AB3F57A7F44
:10C84800DFD3BAF1010ABED1039B002B40F0BD80B3
:10C858004FF47A7ADFF88C9150464FF0100CD9F8E3
:10C868000430C3F30803002B75D1EFF31183002BB9
:10C8780071D12968A26800BF2B689942F9D1D7F80D
:10C8880000E000FB0EF39B1AB3FBFEF300FB013143
:10C898004FF0010E0191D9F80430C3F3080313BB1C
:10C8A800EFF31183FBB92B68A16800BF2A68934294
:10C8B800F9D1D7F800B000FB0BF2521AB2FBFBF229
:10C8C80000FB0323019A9B1AB3F57A7FE3D3BAF1ED
:10C8D800010AC4D1029B013B0293002B7FF467AF8E
:10C8E80005B0BDE8F08FEFF311888CF31288A168CA
:10C8F8002368DB0344BFC6F800E0A1682B683268F0
:10C908005FFA88F888F31188D7F800801A4400FB8A
:10C9180008F35B1AB3FBF8F300FB0233D2E7EFF33B
:10C9280011888CF31288A1682368DB0344BFC6F81A
:10C9380000E0A1682B6832685FFA88F888F31188EC
:10C94800D7F800801A4400FB08F35B1AB3FBF8F32E
:10C9580000FB023370E7EFF311828CF31288D4F8EE
:10C9680008E02368D90303D501233360D4F808E02D
:10C978002B683168D2B282F311883A68194400FBF7
:10C9880002F3A3EB0E03B3FBF2F300FB01317FE7E5
:10C99800EFF311828CF31288D4F808E02368D903E6
:10C9A80003D501233360D4F808E02B683168D2B28C
:10C9B80082F311883A68194400FB02F3A3EB0E03D3
:10C9C800B3FBF2F300FB013118E718461BF0FAFB42
:10C9D8003EE700BF10E000E080650020846500208D
:10C9E8008865002000ED00E0204B5B68C3F3080376
:10C9F80030B4BBB9EFF31183A3B91D4B1D4C1868B4
:10CA0800A16800BF1A689042F9D11B4B1C684FF40B
:10CA18007A7202FB04F3591AB1FBF4F130BC02FB41
:10CA280000107047EFF31182102383F31288114925
:10CA38008C680B6813F4803F104B02D001201860FB
:10CA48008C680B49D2B20D68186882F311880A4BBA
:10CA580019684FF47A72284402FB01F31B1B30BC9F
:10CA6800B3FBF1F302FB0030704700BF00ED00E0BC
:10CA78008465002010E000E08865002080650020C3
:10CA88002DE9F84F8046FFF7AFFF254E2549DFF81F
:10CA9800A0E0254A254D844610274FF47A740120DA
:10CAA800DEF80430C3F30803D3B9EFF31183BBB93D
:10CAB8000B68D2F808A000BFD1F800904B45F7D119
:10CAC800D6F800B004FB0BF9A9EB0A09B9FBFBF98E
:10CAD80004FB0393A3EB0C034345E1D3BDE8F88FB4
:10CAE800EFF3118A87F31288D2F808B01368DB03D2
:10CAF80044BF2860D2F808B00B68D5F800905FFAF8
:10CB08008AFA8AF31188D6F800A0994404FB0AF33C
:10CB1800A3EB0B03B3FBFAF304FB0933DAE700BF1B
:10CB2800886500208465002010E000E08065002012
:10CB380000ED00E02DE9F04FDFF830C1474A4849E1
:10CB4800484E494D8046102718F1FF38C0F08480C0
:10CB5800DCF80430C3F30803002B5CD1EFF3118336
:10CB6800002B58D10B68946800BF08688342F9D13C
:10CB7800D6F800904FF47A7000FB09FEAEEB040E75
:10CB8800BEFBF9FE00FB03EEDCF80430C3F3080338
:10CB98004FF47A740120FBB9EFF31183E3B90B6802
:10CBA800D2F808A000BFD1F800904B45F7D1D6F8CD
:10CBB80000B004FB0BF9A9EB0A09B9FBFBF904FB6C
:10CBC8000393A3EB0E03B3F57A7FBDD2DCF80430F0
:10CBD800C3F30803002BDFD0EFF3118A87F3128821
:10CBE800D2F808B01368DB0344BF2860D2F808B055
:10CBF8000B68D5F800905FFA8AFA8AF31188D6F89C
:10CC080000A0994404FB0AF3A3EB0B03B3FBFAF36C
:10CC180004FB0933D5E7EFF3118487F31288D2F8C0
:10CC280008901368D80303D501232B60D2F8089025
:10CC38000B682868E4B284F31188D6F800A04FF492
:10CC48007A7400EB030E04FB0AF3A3EB0903B3FBAE
:10CC5800FAF304FB0E3E97E7BDE8F08F10E000E022
:10CC680084650020886500208065002000ED00E0D4
:10CC780030B4EFF31183102282F312880649074C6F
:10CC88000A680748013200250A602560DBB202689D
:10CC980083F3118830BC70478465002080650020CC
:10CCA80010E000E00F4B1B88014643B90E4B0F4ABA
:10CCB8001B7810680BB981F00101F4F72EBE0C4BFC
:10CCC8005A691AB118B91A68106058747047094A35
:10CCD80018681188084A92FBF1F201210260597420
:10CCE800704700BF5C6500205E650020606500201D
:10CCF800646500207C65002020A107001D4B70B5ED
:10CD08009C68E36C226BDD69C2B1636B2BB12B07A6
:10CD180002D5E36C08221A6270BD2A06F7D5A26A0A
:10CD2800616A8A421FD0511CA069A162825C206995
:10CD3800E66C81423285EAD3A362E8E7A906E4D526
:10CD4800E26A1AB1988C80B29047DEE7E1699B8C61
:10CD58006069DBB24E1CE6614354E169E3689942BD
:10CD680028BFE261D1E7E26C136823F08003136007
:10CD7800CDE700BF582C00201D4B70B55C68E36CF4
:10CD8800226BDD69C2B1636B2BB12B0702D5E36C53
:10CD980008221A6270BD2A06F7D5A26A616A8A4219
:10CDA8001FD0511CA069A162825C2069E66C814297
:10CDB8003285EAD3A362E8E7A906E4D5E26A1AB1A4
:10CDC800988C80B29047DEE7E1699B8C6069DBB2A2
:10CDD8004E1CE6614354E169E368994228BFE26169
:10CDE800D1E7E26C136823F080031360CDE700BF3E
:10CDF800582C00201D4B70B51C68E36C226BDD6954
:10CE0800C2B1636B2BB12B0702D5E36C08221A62FF
:10CE180070BD2A06F7D5A26A616A8A421FD0511CE2
:10CE2800A069A162825C2069E66C81423285EAD3FE
:10CE3800A362E8E7A906E4D5E26A1AB1988C80B241
:10CE48009047DEE7E1699B8C6069DBB24E1CE661C6
:10CE58004354E169E368994228BFE261D1E7E26C93
:10CE6800136823F080031360CDE700BF582C00201F
:10CE780070B4EFF31186502383F31288436B1A685A
:10CE8800D20720D45D686DB9446A826A944217D08B
:10CE980081691144D9600ED9A21A5A6084620022AD
:10CEA80080F850201A6842F00102F1B21A6081F34A
:10CEB800118870BC704701698A1A5A608562EEE76A
:10CEC800012380F85030F1B281F3118870BC7047AB
:10CED8002DE9F04F2DED028B984B994A1C7893B0B1
:10CEE80000F59C412031814606911160002C00F02C
:10CEF8009086944A1268904240F28A80924A9349F6
:10CF08001768934DDFF888B20492013C02911C70B7
:10CF180007F48057002F40F08880029B5B7D002B30
:10CF280040F04186049B1B681E0401F11581894B62
:10CF380099459BF8023000F21385002B40F01485C8
:10CF4800854B0593049B1F6817F4805940F0CF85E3
:10CF5800029BB5F906605B8B9E42B4BF0026012692
:10CF68007E4B1B6813F0805369D0059A127812F033
:10CF780001026AD002987A49408C91ED037A0391B4
:10CF880007EE900AF8EEE77AB4EEE77AF1EE10FAD7
:10CF980081F28081002E60D1724C94F8A010002993
:10CFA8005BD171487149006890F82D0000240C602D
:10CFB8004C608C606E49002850D10870002A51D00E
:10CFC800F8064FD56B4A1278D1064BD4B9F1000F49
:10CFD80048D1002B46D17A0244D4674B1B78002BEA
:10CFE80001F0C486654B9B78002E41F03F873BB12A
:10CFF800634A644B12681B689B1A002BC1F2418775
:10D008001020584C1DF0D0FC012384F8A13029E0F1
:10D018004D4B4E4A1F68049307F4805702924C4DBB
:10D02800DFF86CB1002F3FF478AF00214B48F5F7DB
:10D03800EAFB00287FF471AF07F04EFE6DE77C0233
:10D0480093D4059A127802F00102464C002184F824
:10D05800A01043490391002EA3D045490120087030
:10D06800002AADD1484B1A78002A50D10299B5F957
:10D0780000E0488B898BB5F902407045B4BF802722
:10D08800002747F040037145D8BF3B469B0843F053
:10D098008007A042B8BF3B4643F04007A142C8BF43
:10D0A8003B469B08B5F90440B5F9067043F0800E7D
:10D0B800A042B8BF734643F0400EA142C8BF7346B2
:10D0C8009B0843F0800E274C8742C8BF734643F045
:10D0D800400E94F8A2C08F42B8BF73469C4501F039
:10D0E800C182A4F8A42084F8A620234984F8A23099
:10D0F8000F78002F01F053825F2B01F08D826F2B88
:10D1080001F02481059B1B78DE0741F1E880049B30
:10D118001B6803F00403002B40F088860DF14008DB
:10D128001A4C0022C8F8042004F15009109240F665
:10D13800330A192740F283362FE000BF2C3D002028
:10D14800E0380020283D00203055002040420020D3
:10D15800AC6C0020404B4C005B5F00208C330020FF
:10D16800543E0020D822002094300020A433002010
:10D178008822002094330020E0000020E0350020C1
:10D1880084650020A82E00202032002008360020C8
:10D198005C6C002004344C4520D0A278E3789A4295
:10D1A80017FB0260F6D26178043117FB036235F988
:10D1B80011305345A8BF5346B3F5617FB8BF4FF44C
:10D1C80061739842E6DA9A42E4DB21782429E1D8AF
:10D1D80040460434F5F708FB4C45DED1634A644BFE
:10D1E800177898E8030083E80300002F00F0808593
:10D1F800604B06935E480121F5F705FB002840F0D7
:10D20800AB829BF80330002B40F0A6825A4B079361
:10D218005A4C23881EB226F001061FFA86F84345A9
:10D22800A4F8008000F0F787554E4FF002090E2051
:10D2380014274FF0FF0A86F80090777086F802A04E
:10D248001DF0B2FB49464A48B4F80080F5F7DBFA0E
:10D25800002800F09E8228F0010292B24245228006
:10D2680009D00E2086F80090777086F802A01DF08D
:10D278009BFBB4F8008018F0020F01F08080414B4E
:10D28800414A19785068099318F0030F08BF81F0D4
:10D298000201C1F340010892F4F73FFB242134480E
:10D2A800F5F7B1FA30B9059A13785E0744BF23F051
:10D2B80004031370079B1B6813F00A0F1AD006218A
:10D2C8002B48F5F7A0FA002800F0B2872388580603
:10D2D80041F1C48007212648F5F795FA50B12B4B48
:10D2E8002B4AB3F904302B4982FB0302DB17C3EB4B
:10D2F800A2030B800C211E48F5F785FA2288002826
:10D3080000F05B8242F480739A42238009D01C4B60
:10D3180002201421FF2218700E2059709A701DF0F7
:10D3280043FB1D4B1B78082B00F053820E2B00F09B
:10D338005082049B1B68590561D5184B1B79002B3B
:10D3480000F0258114210A48F5F75DFA002840F01D
:10D35800238118F04DF8012003F0B2FE00284ED0CA
:10D36800DFF83C9000264FF0CC0A1EE0D66C002077
:10D378008C3300204030002004360020D46C00207C
:10D38800FC2F00204D65002050650020245000200F
:10D3980067666666A42E002000360020443E002002
:10D3A800244B0020DEB2022E29D80AFB06F8731C93
:10D3B80059F80870002FF5D1C378D04A90F90200C7
:10D3C80052F8233001970322009201213A4603F0D4
:10D3D80077FC034606EB460000EB0010079353B1B9
:10D3E800394609EB8000CC2220F0CBFC079B49F89A
:10D3F80008300136F6B21BF063FF0028D3D1059B35
:10D408001E7816F0010600F01482BD4B01221A7036
:10D41800069BB5F906101B68BA485A89012791423C
:10D42800077080F2EC81B84B4FF07E521A60B74A11
:10D43800029BB5F900E01F8B92F90430107892F83E
:10D4480001C0002BAEEB070314BF01224FF0FF32DF
:10D45800002BB8BF5B42B3F5FA7FA8BF4FF4FA734D
:10D46800984280F2C9811B1A07EE903AF8EEE77AE3
:10D47800039BBE45C3ED007A03DAF1EE677AC3ED8C
:10D48800007AB5F902E0AEEB0703002BB8BF5B42A8
:10D49800B3F5FA7FA8BF4FF4FA73984280F25D8221
:10D4A8001B1A07EE903AF8EEE77A039B7745C3ED2F
:10D4B800017A03DDF1EE677AC3ED017AB5F904006C
:10D4C800C31B002BB8BF5B42B3F5FA7FA8BF4FF46C
:10D4D800FA736345CCBFA3EB0C03002302FB03F3F1
:10D4E80007EE903A039A049BF8EEE77AB842C2ED49
:10D4F800027ABCBFF1EE677AC2ED027A1A6812F4BA
:10D50800805200F00782B1F5FA6F814BA8BF4FF443
:10D51800FA61B1F57A7F1878B8BF4FF47A71A1F53E
:10D528007A71002840F00F827A4D7B4885FB013ED6
:10D53800CB17C3EB6E1303F1010E6FF0630C30F9D8
:10D548001EE030F913000CFB0313AEEB000103FBE4
:10D5580001F385FB0315DB17C3EB651303441BB20B
:10D5680007EE903A039BB8EEE78A83ED038A002A18
:10D5780040F0918323885B0624D4002E40F0B080CD
:10D5880009F0CFFF13B0BDEC028BBDE8F08F059B0F
:10D598001B78DA077FF5DDAE3C2011F025F900286D
:10D5A8003FF42DAF03F074FB3C2011F085F8002800
:10D5B8003FF425AF03F06CFB3C2011F07DF8002808
:10D5C800F0D11CE7554B564AB3F904305549DFED05
:10D5D800566A09889FED557A82FB0302DB17C3EB75
:10D5E800A2035B1A1BB207EE903AF8EEE77A67EEF1
:10D5F800A67A77EE876ABDEEE66A16EE103A203311
:10D60800402B40F23787DFED4A6ABDEEE77A17EE26
:10D61800103A2033402B00F229879FED467AF4EE2A
:10D62800C77AF1EE10FA41F3AF82DFED435A9FED6E
:10D63800436A01E0F0EE477AF4EEC67AF1EE10FAAA
:10D6480037EEE57AF6DCDFED3E7AB4EEE77AF1EE16
:10D6580010FA41F19D82DFED385A9FED3A6A01E0F8
:10D66800B0EE677AB4EEC67AF1EE10FA77EE257A64
:10D67800F6D49FED2E7AF4EEC77AF1EE10FA00F3A5
:10D6880021869FED317AF4EEC77AF1EE10FA44BFA5
:10D698009FED2B7A77EE677A67EEA75A9FED2B5AA4
:10D6A8009FED2B6A9FED2B7AA5EE856A27EEA55A8A
:10D6B800A5EE867AE5EE077A039A92ED016AD2ED35
:10D6C800005A27EEC67A65EEA77AA5EEA67AE6EEA8
:10D6D800267A82ED007AC2ED017A002E3FF450AF2F
:10D6E800099B1978089B01F001011868F4F715F9EE
:10D6F80013B0BDEC028BBDE8F08F00BFECFE020852
:10D708005C5F0020C021002064220020BC3500207E
:10D71800082500201F85EB514430002024500020AC
:10D7280067666666A42E002035FA8E3CDB0FC93F7B
:10D7380000000000DB0F4940DB0FC940E4CB164175
:10D74800DB0F49C0E4CB16C1DB0FC9BF92E741B973
:10D758009730083C15A82ABEBF4B07931B689F0744
:10D768007FF556ADBD4CB4F8008018F0010F10D10C
:10D7780048F00103984523800BD0B94B02221421AD
:10D788001A700E20FF2259709A701DF00DF9B4F826
:10D79800008028F002039BB2434523803FF46FAD1D
:10D7A800AF4B1421FF2202260E201E7059709A706A
:10D7B8001DF0FAF8B4F8008061E522F480739BB29A
:10D7C8009A4223807FF4A3ADA64B1B78082B7FF4E5
:10D7D800ADAD228822F040039BB29A4223803FF4E9
:10D7E800A8AD9F4B02201421FF2218700E205970FB
:10D7F8009A701DF0D9F89CE5DFED9B7A38E6B1F513
:10D80800FA6F80F21984187A8B1A03FB00F3C2F5B9
:10D81800FA6293FBF2F3C3F1640307EE903AF8EE71
:10D82800E77A9FED927A924B67EE877AC3ED007A9A
:10D83800FDE5904B1B780793002B7FF4E9ADDFF8EB
:10D848006CA2DFF86C921AF8030C99F80080514624
:10D85800AAF1030709F0E2FB002800F0F483079B14
:10D86800B8F1000F53D107F10801787909F0D6FB18
:10D87800002841F00D828049B87A09F0CFFB0028D2
:10D8880000F0F583B8F1020F41F005827B49F87B7F
:10D8980009F0C4FB002841F001827949387D09F07C
:10D8A800BDFB002800F0F583B8F1040F41F0F981C1
:10D8B8007449787E09F0B2FB002841F0F58172497D
:10D8C800B87F09F0ABFB002800F0F583B8F1060F2C
:10D8D80041F0ED816D4997F8230009F09FFB00287E
:10D8E80040F059876A4997F8280009F097FB002803
:10D8F80000F0F583B8F1080F40F05E87654997F8A6
:10D908002D0009F08BFB00283FF482AD09231A464D
:10D9180000F043BF029B588B8142C0F28B83B1F564
:10D92800FA6FD4BFC0EB0101C0F5FA614FF47A7306
:10D9380003FB01F1584B1D78C0F5FA60B1FBF0F11B
:10D94800002D3FF4F1AD5B78544801FB03F380FBF5
:10D958000301DB17C3EB6111E6E5DFED437AA4E5CC
:10D9680013B901238BF802304D4B05931B201F7808
:10D978009BF8216009F07CFB012E07F00109824623
:10D9880000F0468607F0020303939BF82030DFF887
:10D998002481444C052B00F29D80DFE813F08D00B4
:10D9A80050000600DE000201C000012E04BF05235E
:10D9B8008BF82030B9F1000F00F01681029B3A4F26
:10D9C800B3F91810B8F80030002261F30F0263F3BE
:10D9D8001F42002361F30F0361F31F436A60396834
:10D9E800DBF814202B608A42C0F03B84012E41F002
:10D9F800568203229BF820300392CBE709F064FBA0
:10DA0800012808D1284FB8F802303A68642101FB90
:10DA18000323CBF81030BAF1000F04D098F8063081
:10DA2800002B40F09180012E54D01F4FDBF81020BE
:10DA38003B689A42C0F0678601238BF82030012E9C
:10DA48006DD098F80730012B00F0D88013F0E4FF70
:10DA58009BF820309EE700BF04360020D46C0020DD
:10DA6800FC2F002000360020000000000AD7233CCD
:10DA7800642200205C5F0020D42F0020D92F0020D2
:10DA8800DE2F0020E32F0020E82F0020ED2F0020BC
:10DA9800F22F0020F72F0020082500201F85EB51CA
:10DAA8005B5F0020806C002084650020CA2F002066
:10DAB80080000020E4540020B9F1000F9ED14FF4FB
:10DAC8008060BAF1000F00F0B0831CF0CBFF002398
:10DAD800CBF81030039B002B3FF434AA03981CF0BA
:10DAE80063FF049B1F6817F480593FF431AA1D2176
:10DAF800BB48F4F788FE00287FF42AAAB94A029B9B
:10DB0800D2881B8BB5F90660991A8E4240F3F085CE
:10DB180013449E42B4BF00260126FFF721BAB24F34
:10DB28003A68B8F80230642101FB03234FF480609F
:10DB38000022CBF810308BF820208BF803201CF043
:10DB480079FF9BF8203025E713F066FF03224FF496
:10DB58007A738BF82020CBF81C30A34F238843F02E
:10DB68000203238007F0B8F83A68DBF81C30134446
:10DB78000422CBF818308BF82020012E40F0BB850A
:10DB88003B68DBF818209A42A4D2984B187818B949
:10DB980009F06EFA00289DD1238823F00203238020
:10DBA800BEE7914FE9E7029A013BD27D35F9133080
:10DBB800002A40F05183A3F57A73B3F57A7FA8BFA2
:10DBC8004FF47A7323EAE37307EE903A9FED887A6D
:10DBD800F8EEE77A67EE877A864AFCEEE77A17EE80
:10DBE800903A1380FFF7A3B97F4F3B6847F2305252
:10DBF8000323CBF81C208BF82030AFE713F00CFF81
:10DC0800032240F6B8338BF82020CBF81C30764F2F
:10DC1800A4E7794F3B78002B00F0DC87774BDFF8DF
:10DC2800F881DFF8F8B1DFF8F8A1029345465E46BF
:10DC3800039099460EE019F804109847032C28DC45
:10DC480088B93B782AF8020F01349C4205F1040593
:10DC580080F21081072CE1B23046DBF80430EADDAF
:10DC6800984700B2EDE738F824206B88801A4FF403
:10DC78007A719B1A01FB00F040F6CA0290FBF3F0A0
:10DC88000844904240F2EE23A8BF10469842B8BF1D
:10DC9800184600B2D5E71D215148F4F7B4FD002815
:10DCA8003FF468AC9BF80330002B7FF463ACDFEDE6
:10DCB800547A544938EE678AC7F5FA63FDEEC87A94
:10DCC8001BB2CDED027ABDF90820120381FB0201D7
:10DCD800D217C2EBA11203FB02F343F30F333B4409
:10DCE80007EE903A039BF8EEE77AC3ED037A41E436
:10DCF800DFF830A1DFF83081434C0AF15A064FF0C3
:10DD0800010951461AF8010C09F088F9F8B19AF896
:10DD180004009AF802309AF803E000EB400104EBA3
:10DD28008101013BD1F8B42003EB43034344934200
:10DD38000DD094F8E02081F8B0E009FA00F022EA6A
:10DD48000000C1F8B430C1F8B87084F8E0000AF1F6
:10DD5800060AB245D5D12D4B06931946224A2C4BBB
:10DD68002C4C09681B78D2F8009008910793A4F10D
:10DD7800B00A002663685BB31F784FB3A268A9EBAB
:10DD88000202002A0ADB9AF8E0200121B14022EAC7
:10DD9800010209F5FA718AF8E020A160079ABAB180
:10DDA800227859780432D2B2002940F07982029957
:10DDB80035F91220098B01F1C800824240F36A84C8
:10DDC8009AF8E0109A7841FA06F3D90740F1DE8410
:10DDD8000136042E04F10C04CCD1FFF70BBA00BFB6
:10DDE8008C330020CC54002084650020E000002003
:10DDF800AAF1823F446C00207C5900204042002058
:10DE080000007A44D34D6210D82200204030002010
:10DE18003D6C00208823002094590020D43800202D
:10DE2800D6220020E12E002074E20208B24C94F8B9
:10DE3800AA3053B1059B1B78D80706D5029BB5F9C4
:10DE480006205B8B9A4200F376841121AB48F4F7E5
:10DE5800DAFC002800F00C8294F8AE302BB994F864
:10DE6800A83013B93223A4F8AC30012384F8AE30BB
:10DE7800FFF754B9DDF80C90A14A04921146A14A63
:10DE8800096842F2010AA2FB092B11EA0A0A4FEAC1
:10DE98009B1B00F0E9819C4D9C489D4C9D4A95F840
:10DEA80000E0007884F800E01070BEF1000F04D0A4
:10DEB800984A92F800E08EF0010E8F4C0F2084F8FB
:10DEC8002400002B00F04B83934B0B931B780A9391
:10DED8001E463B78029F914AB7F824C0DFF870824B
:10DEE80009903D46FF8C08973746A2FB0662520808
:10DEF8002D8B0E9502EB420294F825500C95BA1A18
:10DF0800D2B201F48051079204F128060BF59672FB
:10DF18006746834DCDF80CE0A4465446DDF830A0A2
:10DF28000F9100200592CDF834909E46039B002B5C
:10DF380000F039823CF910101FFA81F9B9454FEA0F
:10DF4800400203D3089B994540F26F8258F820108D
:10DF58008B4580F03182A95E002C40F0458201306B
:10DF68007045A95206F10606E0DB09986D4ADDF80E
:10DF780034908CF824000F28644651460CBF0121C8
:10DF88000021734684F825A0117000F0EE82DFF8B6
:10DF9800C4B1654E654F34883868DBF80810DBF883
:10DFA8000420CBF80C0044F00404401A9042574F68
:10DFB8003480584C4FF0010188BF0022397021701D
:10DFC80088BF8BF82120002B00F0E482049A029984
:10DFD8001768574EB1F824C0B1F818E0504817F444
:10DFE8008057344640F0F68239460EE0627802EBFC
:10DFF800820202EB820202F2EE2292B201318B42DD
:10E0080020F8022B04F102040ED016F81120002A81
:10E0180000F00F82022AE9D00131028820F8022B91
:10E028008B4204F10204F0D10B9A13780133137078
:10E03800FEF770BF11467DE41B7AC3F1640307EE57
:10E04800903AFFF7ECBB0AF10501787908F0E6FF92
:10E0580000283FF410ACB8F1010F40F0198607F121
:10E068000D01B87A08F0DAFF002840F0148631492B
:10E07800F87B08F0D3FF00283FF40FACB8F1030F8A
:10E0880040F00C862C49387D08F0C8FF002840F085
:10E0980008862A49787E08F0C1FF00283FF40FACB3
:10E0A800B8F1050F40F000862549B87F08F0B6FFA3
:10E0B800002840F0FC85234997F8230008F0AEFFBC
:10E0C80000283FF40FACB8F1070F40F064831E49F5
:10E0D80097F8280008F0A2FF002840F06D831B493C
:10E0E80097F82D0008F09AFF00283FF491A9B8F19D
:10E0F800090F3FF48DA909E4D82200208C330020B1
:10E1080030550020D34D6210B03800204807002059
:10E118003D6C00204907002029590020ABAAAAAA73
:10E12800AC6C002095330020806C002084650020B2
:10E13800C8590020D92F0020DE2F0020E32F00200F
:10E14800E82F0020ED2F0020F22F0020F72F0020CD
:10E158002C5900205C6C0020CC4CD4F88830A9EBFA
:10E168000303002BFEF6E3AEC94A94F88C30517CC9
:10E17800069AC4F888200133C64A029E32F8112054
:10E18800B17D03F00F0384F88C30234492B292FBE4
:10E19800F1F283F8902094F8901094F8912094F874
:10E1A800923094F89C000A4494F89310134494F81D
:10E1B8009420194494F895300A4494F8961013441E
:10E1C80094F89720194494F898300A4494F89910D0
:10E1D800134494F89A20194494F89B300A44134441
:10E1E80094F89D1094F89F20184494F89E300144A8
:10E1F8000B441A4442F30B12642AF17DA8BF64222F
:10E2080013B209B1C2F1640307EE903A9FEDA27A06
:10E21800F8EEE77ADEE40221A048F4F7F4FA0028E1
:10E228003FF4B7AA2680FFF726B81CF003FC4EE49B
:10E23800228822F040039BB29A4223803FF44AA8E6
:10E24800974B02201421FF2218700E2059709A70E3
:10E258001CF0AAFBFFF73EB8C3F53B6308331BB2BB
:10E26800A9E403230393C1E48E4A92F800E01CE674
:10E2780094F8A830002B3EF451AF059B1B7813F09F
:10E2880001037EF44BAF012284F8A83084F8A9205A
:10E29800FEF744BF7D4C012184F8A010FEF7DDBED7
:10E2A800012900F034849AF8E0200123B3400136B4
:10E2B8001343042E8AF8E03004F10C047FF45AADBD
:10E2C800FEF798BF9FED837A77EE677AFFF7E4B998
:10E2D800059B754A1B781060DB0700F13A8294F8B9
:10E2E800A60000287EF413AFB4F9A430322B7EF7D1
:10E2F8000EAF94F8A2200121572A84F8A61000F046
:10E30800B384049B1B6813F0040302D05A2A00F05C
:10E3180067855D2A00F005855B2A00F017855E2A6F
:10E3280000F02085562A00F07285972A00F04E8565
:10E33800A72A40F0C7845D49049B0A781B6842F00D
:10E3480004020A7003F00403FEF7E5BEB2F5FA7F93
:10E35800FEF6DDAE94F8A620002A7EF4D8AE059B22
:10E368001B780121DF0784F8A61000F1A38405F0CB
:10E3780061FE049B1B6803F00403FEF7CCBE48F063
:10E388000203434523803EF47AAF454B0222142111
:10E398001A700E20FF2259709A701CF005FBB4F811
:10E3A8000080FEF76CBF002F3DD058F820108B4539
:10E3B8004FEA4002FFF4CFAD3D4B995C03EB0209F5
:10E3C800002900F0F980022946D199F8011001EBE3
:10E3D800810101EB810101F2EE2189B2032832DDCE
:10E3E80009B2002C3FF4BBAD079B26F81310BAF115
:10E3F800000F03D10A9B022B7FF6B1ADB6F800A03F
:10E408007188B6F804902B4B514489440FFA89F966
:10E4180083FB0931284BA1EBE97123F8029009B27B
:10E428004FF0010A9BE539464200059B48F8203029
:10E4380092E5CAB2022A04D9032A7FF4EDAD6246F6
:10E44800DCE57246DAE5012303FA00F9099B23EAC1
:10E45800090309B209937FE5A95ABFE743F04002CF
:10E46800934222807FF4ECAEFEF734BFDFED137ADF
:10E47800FFF722B9F4EEC77AF1EE10FA40F3A7835A
:10E48800DFED115A9FED0E6A2EE000BFD822002062
:10E49800B4650020D065002014AE23418C330020E1
:10E4A800FC2F00203D6C0020AC2E0020943300206F
:10E4B800C859002056555555482300200000000033
:10E4C800E4CB1641DB0F49C0DB0FC940E4CB16C1D2
:10E4D800DB0FC93FDB0F494092E741B99730083C51
:10E4E80015A82ABEF0EE476AF4EEC66AF1EE10FAF5
:10E4F80036EEE57AF6DC5FED0D6AB4EEE67AF1EE1B
:10E5080010FA40F16B835FED105A1FED106A01E0BD
:10E51800B0EE667AB4EEC67AF1EE10FA77EE256AB6
:10E52800F6D41FED157AF4EEC76AF1EE10FA40F34F
:10E538008D801FED187A77EE666A66EEA65A1FED93
:10E548001A5A1FED1A6A1FED1A7AA5EE856A26EE89
:10E55800A55AA5EE867AE5EE076AFFF756B8BA49D6
:10E56800BA4A0B91BA4D012111701B21B948039386
:10E57800F4F749F9039B00287FF409ADDFF8F4B2FA
:10E58800B54FDBF80C203B68CBF808309B1AC82B3A
:10E5980000F22783049B1F6807F4805744E5394637
:10E5A800AC48F4F730F900283FF492AE84F8A7702D
:10E5B80005F040FDFEF7A6BDC1B2022940F2A582D2
:10E5C80003297FF449AF0E9B19460F9B002B08BF08
:10E5D800394603E700210FE0627802EB820202EB82
:10E5E800820202F2EE2292B20131994220F8022B05
:10E5F80004F102043FF418AD16F811201AB1022AEA
:10E60800EAD00288F0E7CAB2032AFAD87246EBE7E2
:10E6180000230393FFF7B9B9B2F5FA7FFEF677AD99
:10E6280094F8A630002B7EF472AD059B1B7801216F
:10E6380013EA010084F8A61000F0E18206F04CFB12
:10E64800049B1B6803F00403FEF765BD9FED837A06
:10E65800F4EEC76AF1EE10FA44BF9FED817A77EEC7
:10E66800666A6AE77F4A80491068B4F9A420C769D6
:10E6780081FB07018911FF17781A00F5FF407F30E9
:10E6880082423EF732ADC91B0A4412B2A4F8A42054
:10E69800FEF72BBDC8398A4240DA9AF8E0109A781A
:10E6A80041FA06F3DB073FF593AB5242012009928A
:10E6B80002F000FE7B1E099A162B00F21B81DFE890
:10E6C80013F0A401BA018B01E301D001F70176012F
:10E6D80061014A0133011C011901E3010901F70134
:10E6E80076016101F300DD00AC000C0294007E00AD
:10E6F8000126FEF735BC3A68DBF81C301344CBF82A
:10E708001830FFF7E7B913F087F9032240F6B8335A
:10E718008BF82020CBF81C30FFF720BA9AF8E030AD
:10E728000122B24023EA020309F5FA728AF8E030BE
:10E73800A260FFF74DBB00214648F4F764F80028B3
:10E748007FF483AB322384F8AA00A4F8AC30FFF737
:10E758007CBB464B1B78002B3EF4D9AC9BF80330AE
:10E76800002B7EF4D4AC94F8A7300133DBB2032B32
:10E7780084F8A7307EF6CBAC3D4B5B7813B9002EFE
:10E788007EF4C5AC06F0A8FAFEF7BCBC002A0CBFA4
:10E79800012002208BE707231A4602EB8202174466
:10E7A80089F80030B97878781BF040FD059B1E7811
:10E7B80006F00106FEF72CBE08231A46EDE7DAF844
:10E7C800E400DFF8B48090F8361098F8023011446D
:10E7D8006429A8BF642121EAE17180F83610002B72
:10E7E80040F09C8312F058FA5DE5DAF8E400DFF8AF
:10E7F800888090F8371098F802301144FE29A8BF95
:10E80800FE2121EAE17180F83710002BEAD01620AA
:10E8180008F08CFCDAF8E400E4E7DAF8E400DFF862
:10E82800588081781144C829A8BFC82121EAE1711C
:10E83800817098F80230002BD4D0142008F076FCB0
:10E84800DAF8E400CEE700BF29590020953300200C
:10E85800AC6C00208C33002084650020DB0FC9BF1E
:10E86800DB0F49C0C85E0020D34D62103D6C00200C
:10E87800E03500205C6C0020E2310020DAF8E4008A
:10E88800DFF8888641781144C829A8BFC82121EA41
:10E89800E171417098F80230002BA3D0132008F0E2
:10E8A80045FCDAF8E4009DE7DAF8E400DFF85C8676
:10E8B80001781144C829A8BFC82121EAE171017073
:10E8C80098F80230002B8DD0122008F02FFCDAF8CF
:10E8D800E40087E7DFF83486089898F80230417931
:10E8E80011446429A8BF642121EAE1714171002B18
:10E8F80040F03883DAF8E40074E7DAF8E400DFF887
:10E908000C86017A98F802301144C829A8BFC8219A
:10E9180021EAE1710172002B3FF464AF0B2008F08B
:10E9280005FCDAF8E4005DE7DAF8E400DFF8DC85F6
:10E93800C17998F802301144C829A8BFC82121EA32
:10E94800E171C171002B3FF44DAF0A2008F0EEFBD6
:10E95800DAF8E40046E7DAF8E400DFF8B085817910
:10E9680098F802301144C829A8BFC82121EAE171EA
:10E978008171002B3FF436AF092008F0D7FBDAF895
:10E98800E4002FE7DAF8E400DFF88085417998F8A9
:10E9980002301144C829A8BFC82121EAE171417198
:10E9A800002B40F08082112F7FF43BAF1AE7DAF892
:10E9B800E400DFF85885017998F802301144C82935
:10E9C800A8BFC82121EAE1710171002B40F0D08273
:10E9D800102F7FF457AF05E70899DFF830850F79D6
:10E9E8001744642FA8BF642727EAE7770F7108F058
:10E9F800B7FB98F80230002B3FF47CAF0320394670
:10EA080008F094FBDAF8E400ECE60898DFF8FC84F8
:10EA180001781144FA29A8BFFA2121EAE1710170AD
:10EA280098F80230002B3FF465AF012008F07EFB18
:10EA3800DAF8E400D6E60898DFF8D0848178114443
:10EA48006429A8BF642121EAE171817098F8023035
:10EA5800002B3FF44FAF022008F068FBDAF8E4001F
:10EA6800C0E60898DFF8A484C17998F80230114408
:10EA780081F30801C171002B3FF43CAF052008F079
:10EA880055FBDAF8E400ADE6089BDFF88084997955
:10EA980098F8020011446429A8BF642121EAE171B1
:10EAA8009971002840F034820D2F7FF415AF21E7CB
:10EAB800DAF8E400DFF85484C17898F80230114499
:10EAC800C829A8BFC82121EAE171C170002B40F014
:10EAD80029820F2F7FF4ECAE84E60898DFF82C84A7
:10EAE80041781144B1F5967FA8BF4FF4967121EA99
:10EAF800E171417098F80230002B3FF4FBAE15200D
:10EB080008F014FBDAF8E4006CE60E9966E435F9CF
:10EB180012209978B2F5617F4FF4966393FBF1F375
:10EB28003ADB40F633019142A8BF11460C2FA1F5FC
:10EB3800617191FBF3F100F00D81182F7FF4B3ABF5
:10EB4800C9B2C8290B46A8BFC823DAF8E400C27DB9
:10EB5800DFB297423FF4A7AB9A1ADFF8B083C775C4
:10EB680048BF0732D71098F802300137FFB23BB9D7
:10EB7800002F3FF498AB384602F09CFBFFF793BB9D
:10EB8800182008F0D3FAF3E7B0EE677AFEF75BBD1A
:10EB9800F0EE477AFEF76DBD0C2F40F0D1800027CC
:10EBA8003946C54B09915B78BB423FF47CABDFF833
:10EBB8005C83384603F028F898F8023009991BB1AD
:10EBC800C9B20C2008F0B2FA0137FFB2D0E7B0EEB4
:10EBD800667A90E4B94A0292FFF74EB9F0EE476AB6
:10EBE8009FE4B74A049B1F68138823F0040313802B
:10EBF800012307F480578BF82130FFF715BAB14B82
:10EC08001B6813F4003340F0A7801846AE490E5C29
:10EC18000F2E00F10C000ED00133152BF7D1049BF9
:10EC28001B68FA3A0021A4F8A42003F0040384F82E
:10EC3800A610FEF770BAA54FD7F800E05800BEF14D
:10EC4800000F07D0C61801EB86069EF801E076781B
:10EC58007645E4D218449E4E9E4B01EB800100207D
:10EC6800396030801860DAE79B4B9C491A684FF48A
:10EC78007A73B3FBF2F3C3EB431203EB8202049BF8
:10EC88001B68D200A1F8B42003F00403FEF743BACE
:10EC980001231A4681E502231A467EE503231A4614
:10ECA8007BE504231A4678E505231A4675E506230D
:10ECB8001A4672E5049B8A491B680A6003F004033C
:10ECC800FEF729BA0021BB2A10917CD0B72A76D04A
:10ECD800BE2A72D0BD2A59D09E2A00F0C1809D2A32
:10ECE80000F0B780AE2A00F0AD80AD2A00F0A38016
:10ECF800EF2A00F03181FD2A00F02881FB2A00F07C
:10ED08001F81FE2A00F01681F72A00F0C2807B2AB4
:10ED18007EF4FDA94FF4FA61022002F09BFEFEF793
:10ED2800F6B9704B002201206F49634C0B602270CA
:10ED380002F0C0FA049B1B6803F00403FEF7EBB96A
:10ED4800182F7FF4B0AA00210B46FEE6674B01227C
:10ED58000220E9E7CFB224E7654B1B78032B65D087
:10ED6800034653E7634B02220320DDE7002E3EF4FF
:10ED780047A9614C94F8A130002B3EF473A91BF00D
:10ED8800F7FD002384F8A130FEF76CB94FF6FE7347
:10ED98005A4AD0899689014433449381D1810CF031
:10EDA800FBFEF3F7F9F80CF0DFFEFCF735FF012066
:10EDB80002F080FAB4F8A42031E70223E8E70B4612
:10EDC8004FF6FE71E4E70B460221E1E7049B4C4A4B
:10EDD8001B684FF4C871118003F00403FEF79BB958
:10EDE80094F8A820002A40F0D48094F8AA3083F040
:10EDF800010384F8AA30002B40F0C2800C201BF0DD
:10EE0800D3FD049B1B6803F00403FEF784B90CF0E0
:10EE1800C3FEF3F7C1F80CF0A7FEFCF7FDFE0120D6
:10EE280002F048FA94F8A220FFF77FBA1BF0A0FD81
:10EE3800B4F9A420F3E6FF2100201CF0D9FC94F8D3
:10EE4800A22055E7012100201CF0D2FC94F8A22052
:10EE58004BE70021FF201CF0CBFC94F8A22041E7EF
:10EE680001201CF0C5FC94F8A22038E7002B80D0C4
:10EE78002449254A09684FF47A7000FB031313608C
:10EE880077E71D4C05F028FF002384F8A130FEF732
:10EE9800E9B80021042002F0DDFDFEF738B90323AC
:10EEA8000393FEF71BBE1120099208F03FF9DAF828
:10EEB800E400099A77E500BF823000204042002034
:10EEC800806C0020D42E0020B8F102085C220020BB
:10EED800B0220020B422002020550020D865002050
:10EEE800AC2E0020A230002094300020F03000200A
:10EEF800476C00203E310020D8220020C435002075
:10EF08005E30002084650020A82E0020E231002019
:10EF18000D20099208F00AF9099AC5E5172008F0AA
:10EF280005F9E7E40F20099208F000F9DAF8E4009F
:10EF3800099ACEE50021032002F08CFDFEF7E7B820
:10EF48000021022002F086FDFEF7E1B80021012031
:10EF580002F080FDFEF7DBB80021084602F07AFDDA
:10EF6800FEF7D5B80E2008F0E1F8DAF8E40039E445
:10EF78001020099208F0DAF8DAF8E400099A27E58F
:10EF88000B201BF011FD049B1B6803F00403FEF724
:10EF9800C2B884F8A80084F8A910FEF7BCB800BF6E
:10EFA80038B50B4C23688BB15A68821A002A05467B
:10EFB80004DA0CE05A68AA1A002A07DB9A68226069
:10EFC80018461A6890472368002BF3D138BD38BD1E
:10EFD800FC38002008B512F011F8024B024ADA603A
:10EFE800FEE700BF00ED00E00400FA05024A034B0B
:10EFF800127819780EF016B9BC220020BD22002024
:10F008002DE9F04F2DED028BA0F10A0389B00C46D3
:10F01800E72B00F24B86DFE813F01C01490649068E
:10F028004906490649064906490649064906490660
:10F038004906490649064906490649064906490650
:10F048004906490649064906490667054906490623
:10F0580049062B0549064906490642064906B405EC
:10F0680049069B0549068F054906860549061C067B
:10F07800490608064906490649060106F9054906EA
:10F088003703490649063003490608034906490675
:10F098004906F6024906490649064906D7024906BD
:10F0A800FC00490631046E0149064906490649062D
:10F0B8004906490649062D01490603044906CF03B6
:10F0C80049065803490644034906490649064906BC
:10F0D8000805CD04C6049504E800490649065B0204
:10F0E80036024906FF01E301490649064906490671
:10F0F800D80149064906B701490649064906A80143
:10F108009101C3028102490649064906720249066D
:10F118004906750449064906490649064906490645
:10F12800490649064906490649064906490649065F
:10F138004906080549064906490649064906490691
:10F14800490649064906490649064906490649063F
:10F15800490649064906490649064906490649062F
:10F16800490649064906490649064906490649061F
:10F17800490649064906490649064906490649060F
:10F1880049064906490649064906490649064906FF
:10F1980049064906490649064906490649064906EF
:10F1A80049064906490649064906490649064906DF
:10F1B80049064906490649064906490649064906CF
:10F1C80049064906490649064906490649064906BF
:10F1D80049064906490649064906490649064906AF
:10F1E8004906490649066A044004AC4E337853B1CF
:10F1F800AB4F002537F8021F2046F3F720F9337884
:10F208000135AB42F6DC012009B0BDEC028BBDE84C
:10F21800F08FA24E3378002BF5D0A24F0025B846C8
:10F22800236817F81520591C21601A7098F80110E6
:10F2380001EB810101EB810101F2EE2189B2204647
:10F24800F3F7FDF833780135AB4208F10208E7DC43
:10F25800D9E7954D28461BF041FD0028D3DD2B4604
:10F268000544226813F8011B501C9D422060117050
:10F27800F7D1C8E71AF0EEFFFF28064600F002862D
:10F2880008A9002501F8125D0DF10D008DF80D504B
:10F298001AF0E4FE08A800F8115D1AF0D3FE08A8D9
:10F2A80000F8105D1AF0C2FE08A820F8085D1AF0F0
:10F2B800B1FE23685A1C22601E7023689DF80D2039
:10F2C800591C21601A7023689DF80E20591C216072
:10F2D8001A7023689DF80F20591C21601A70236842
:10F2E8009DF81020591C21601A702046BDF818108E
:10F2F800F3F7A5F887E70B686C4E01255A1C0A60DE
:10F308001D700B68B278591921601A701BF0E6FA63
:10F318002368674A67495F1927601870B1F90010B8
:10F32800B2F90000F3F704FA23685A19226018703A
:10F3380031882046F3F783F8284665E70A685E4B6C
:10F348005E491878551C2560107022685878551C3D
:10F358002560107022689B78501C2060137020462E
:10F36800C988F3F76CF801204EE7544D0846298800
:10F37800F3F765F869882046F3F761F82046A9880D
:10F38800F3F75DF801203FE74D4D05F16006A988C8
:10F398002046F3F754F8E9882046F3F750F829890E
:10F3A8002046F3F74CF82368AA7A591C21601A7092
:10F3B8002368EA7A591C21601A7055F80C1B2046FC
:10F3C800F3F726F8B542E2D11DE73E4952232268F9
:10F3D800501C2060137011F8013F002BF7D112E781
:10F3E800394800232268056803EB4301561C6D5C0D
:10F3F80026601570026825680A446E1C52782660DB
:10F408002A70026825680A4401339278691C0A2B1D
:10F4180021602A70E6D1F6E62C4D0B682A68591C43
:10F42800127821601A702B6822689978531C23601F
:10F43800002311702A6821681A4401335279481C44
:10F44800032B20600A70F5D123682A68591C127AA8
:10F4580021601A7023682A68591CD27821601A70B2
:10F4680023682A68591C127921601A702B68204673
:10F478005989F2F7E4FF2A682368527A591C2160F7
:10F488001A702A6806E100212046F2F7C1FF2046DB
:10F498000021F2F7D4FF0120B6E600BFD4380020DF
:10F4A800AA6C0020C8590020A0350020E2310020B5
:10F4B800806D0020826D0020BC350020CC540020D7
:10F4C8002C500020BCE2020894300020403000207C
:10F4D800A84D08462988F2F7B2FF69882046F2F756
:10F4E800AEFFB5F90430A44AD91782FB0323C1EB58
:10F4F800A301204689B2F2F7A2FF012084E69F4DBE
:10F508000846298AF2F79BFF698A2046F2F797FF97
:10F518002046A98AF2F793FF012075E6DFF894E206
:10F528000027FEB2714600232268501C2060167026
:10F538002268501C20601370226811F8010F0133F3
:10F54800551C062B25601070EED10137062F0EF1E1
:10F55800060EE6D18A4900232268501C20601770E5
:10F568002268501C20601370226811F8010F0133C3
:10F57800551C0B2B25601070EED12368814A581C4E
:10F5880007212060197023680021581C2060197019
:10F59800236892F8F020591C216001201A7033E684
:10F5A8000B68794A79491078794A5D1C256018708A
:10F5B80023688978581C2060197023689278591C30
:10F5C800216001201A701FE60B68724D591C2A79B8
:10F5D80021601A7023686A79591C21601A70298879
:10F5E8002046F2F72CFF2368AA79591C21601A706B
:10F5F80069882046F2F723FF2368EA79591C2160BD
:10F6080001201A7000E60B6800255A1C0A60204683
:10F6180029461D70F2F7FCFE29462046F2F7F8FE4F
:10F6280029462046F2F7F4FEEDE50B685A4A5B4D91
:10F6380011785B4A581C2060197011682046F2F74F
:10F64800E7FE2368574A591C127A21601A702988E4
:10F658002046F2F7F4FEA9882046F2F7F0FE298941
:10F668002046F2F7ECFE00212046F2F7E8FE20469D
:10F678000021F2F7E4FE0120C6E5084608224949C0
:10F68800F2F7AFFE0120BFE50B68474A581C917896
:10F698002060197023685278591C216001201A7063
:10F6A800B2E50B68394A4149D078394A5D1C256072
:10F6B800187023684979581C206019702368D2781B
:10F6C800591C216001201A709EE500212046F2F79E
:10F6D800B6FE00212046F2F7B2FE00212046F2F7DE
:10F6E800AEFE2368324D00265A1C22601E70236825
:10F6F8002A68591C92F82C2021601A7023682A68FD
:10F70800591C92F8362021601A7023682A68591CFF
:10F7180092F8372021601A7023685A1C22601E70E4
:10F7280023685A1C22601E7023685A1C22601E70AF
:10F738002B682046598FF2F782FE2B682046198FD6
:10F74800F2F77DFE23682A68591C92F82E20216062
:10F758001A7023685A1C22601E702B682046598E26
:10F76800F2F76DFE2B682046998EF2F768FE0120AD
:10F778004AE500BF245000206766666620620020C4
:10F788009F5D0020BC5C00200C550020C435002083
:10F79800D4350020E4540020003600207C2C0020C2
:10F7A8001432002040420020E0350020B45E0020E2
:10F7B800943000207B5D0020B54E0B687279B54D02
:10F7C800591C21601A702B682046198CF2F737FEF5
:10F7D8002B682046D98BF2F732FE71892046F2F762
:10F7E8002EFEB1892046F2F72AFE2B682046598C56
:10F7F800F2F725FE2B682046998CF2F720FEF18956
:10F808002046F2F71CFE318A2046F2F718FE2A68D5
:10F81800236892F82620591C216001201A70F3E40D
:10F828009B4EF378002B00F01F830B680822591CAD
:10F8380021601A7023680122991821601A702368C0
:10F84800954D591C2A7921601A702368AA78591C89
:10F8580021601A7029882046F2F7F1FDE9892046CF
:10F86800F2F7EDFD2368F279591C21601A702368BC
:10F87800EA78591C216001201A70C5E40B6800253C
:10F888005A1C0A601D700B685A1C0A601D700B68B0
:10F898005A1C0A6029461D70BFE6804B03F17005AB
:10F8A80022681978501C2060117022685978501C01
:10F8B8002060117022689978501C206011702268AD
:10F8C800D978501C2060117022681979501C20606A
:10F8D800117022685979501C20601170226899793A
:10F8E8000733501C9D4220601170D9D18BE46C4DB8
:10F8F8000846E989F2F7A3FD2046A989F2F79FFD9A
:10F90800012081E40B68674F591C3A7821601A700E
:10F918003B78002B3FF477AC0025EEB230460CF074
:10F928009BFF23684278591C216030461A700CF0FE
:10F9380093FF01892046F2F782FD3B780135AB42FF
:10F94800EBDC60E4584D594E9FED598ADFF88C8105
:10F95800DFED588A05F120070EE0FCEEE77ACDEDE1
:10F96800017ABDF8041020460435F2F768FDAF426D
:10F9780006F118063FF447AC717C0029F3D04E4BD2
:10F98800D5ED007A1B78012BE7D14C4B1B68DB04C3
:10F9980040F16282F5EE407AF1EE10FA40F08B8287
:10F9A80040F2DC51DFE7084610224549F2F719FD1D
:10F9B800012029E4434B9B8AB3F5006F00F2608273
:10F9C800B3F5806F00F27582B3F5007F34BF01276D
:10F9D80002273D4D05F10C0655F8041B91FBF7F184
:10F9E800204689B2F2F72BFDAE42F5D1374D384F9C
:10F9F80005F10C06B5EC010AD7ED087A80EE270A66
:10FA08001CF0B4F881B22046F2F719FDB542F1D1E5
:10FA1800304D05F10C0655F8041B204689B2F2F763
:10FA28000EFDAE42F7D1FFF7EEBB00258146DFF8A9
:10FA3800B080DFF8B0B005950495069507950121CB
:10FA48004FF6FF7A05E001350B2D00F04F8118F9CC
:10FA5800011F4F1C4AFA05F3F5D0DE07F3D5BBF8B2
:10FA680000302B41D807EED506A8F2F7BDFEEAE72D
:10FA7800194D08462988F2F7E2FCA9882046F2F7D2
:10FA8800DEFC20462989F2F7DAFC0120FFF7BCBB2F
:10FA98000C550020943000202062002020510020C6
:10FAA800C4350020DA3D00201434002060610020B5
:10FAB8000000404200E082444462002030550020AB
:10FAC80004340020BC330020F433002024550020E7
:10FAD800D8650020FC5400207C2C0020DB9B914141
:10FAE800ECE20208D46C00209F4D05F150062878FE
:10FAF80016F014FF2368027A591C21601A702368D3
:10FB08006A78591C21601A702368AA78591C2160E8
:10FB18001A702368EA780435591CAE4221601A70BD
:10FB2800E5D1FFF770BB0B68904A591C527D2160E4
:10FB380001201A70FFF768BB8D4D05F1800655F856
:10FB4800041F2046F2F764FCAE42F8D1FFF75BBB16
:10FB5800884D05F14006B5F880102046F2F76FFC95
:10FB6800236895F88220591C21601A70236895F83B
:10FB780083200435591CAE4221601A70EBD1FFF77F
:10FB880042BB7A4D0B682A7A591C21601A70A98BDE
:10FB98002046F2F754FC298B2046F2F750FC698B7B
:10FBA8002046F2F74CFC2368EA7C591C21601A7045
:10FBB800A98C2046F2F743FCE98C2046F2F73FFC7B
:10FBC8002368AA7F591C21601A70236895F82020A1
:10FBD800591C21601A70698C2046F2F730FC2368A2
:10FBE800EA7A591C21601A70E9682046F2F710FC7D
:10FBF80023682A7C591C21601A70236895F82120F3
:10FC0800591C216001201A70FFF7FEBA0B68012207
:10FC18009918216010461A70FFF7F6BA08460021B5
:10FC2800F2F7F6FB0120FFF7EFBA534D534E05F1FB
:10FC3800200795F90210524B93F906208A4203F1E6
:10FC4800080336D09E42F7D10835BD42F1D1FFF7FF
:10FC5800DABA4C4B03F15A0522685979501C2060D6
:10FC6800117022681978501C206011702268597828
:10FC7800501C2060117022689978501C2060117007
:10FC88002268D978501C20601170226819790633CF
:10FC9800501C9D4220601170DED1FFF7B4BA0B688A
:10FCA800394A581C117820601970F3E40020FFF7D6
:10FCB800ABBA23685A1C2260197029882046F2F7CB
:10FCC800BEFB2368EA78591C21601A7023682A79D8
:10FCD800591C21601A702368AA79591C21601A706E
:10FCE80023686A79591C21601A70ADE7DFF8A4A06F
:10FCF80000254FF008080135C5F1200208FA02F284
:10FD0800A5F120032AFA05F6164328FA03F31E4341
:10FD1800252D06F001024FF000030BD01343EAD063
:10FD2800E8B207F0A5F90028E5D0294606A8F2F7B9
:10FD38005BFDE0E7154B1B78DA0700F1AA80002588
:10FD4800134E2F4602E00135252D25D02946304691
:10FD5800F2F759FD0028F6D0294606A8F2F753FD18
:10FD6800002874D10137EEE7083600204042002011
:10FD7800B85C0020BC5C0020D06B002090560020AE
:10FD880070560020E02E0020003600205B5F002027
:10FD9800445F002090E33FF4654B664DB3F8501084
:10FDA8002046F2F74CFB00212046F2F748FB624B55
:10FDB80019684B0103F02002C1F340031343C1F358
:10FDC800800243EA4203C1F3C00243EA8203C1F35B
:10FDD800401243EAC20301F0100119432046F2F72A
:10FDE8002EFB04A904222046F2F7FBFA236829789F
:10FDF800524A581C2060197011886429A8BF6421D0
:10FE08002046F2F71CFBB9F1960F47D00021204697
:10FE1800F2F715FB2168B7F1190348BFA7F11203E0
:10FE2800A3F3C4034A1C226020461A460B7005A996
:10FE3800F2F7D7FA2368424A581C1021206019703B
:10FE480020461188F2F7E4FA0120FFF7DDB93946B8
:10FE580004A8F2F7C9FC85E7F4EEC87AF1EE10FAC7
:10FE680045DA4FF47A717EE50B68B178354A581C4B
:10FE78002060197023681278591C21601A70DEE41A
:10FE88000827A6E523685A1C226001201E70FFF788
:10FE9800BBB9069B43F00103069350E7236803228E
:10FEA800591C21601A7023686A78591C21601A70DD
:10FEB800B0E704278DE5F4EEC87AF1EE10FA3FF5C5
:10FEC8006FADF4EEE87AFDEEE77AF1EE10FA17EE90
:10FED800901A1ED86FF4F973303903FB01F140F220
:10FEE800E73391FBF3F101F2DB5189B23BE5FDEE1B
:10FEF800E77A40F2E73217EE903A303B02FB03F321
:10FF080088FB0312D917C1EB622101F2E93189B2EA
:10FF180029E540F2F313A1F5836103FB01F140F2F7
:10FF2800E73391FBF3F101F2DD5189B21BE500BF24
:10FF3800200800208230002004360020B22E002045
:10FF4800806C0020B83500201C4C08B50121022027
:10FF5800F1F7EDFC237803F00502052A2AD003F017
:10FF68000903092B08D000210120F1F7E0FC00214A
:10FF78000846F1F7DCFCFEE7114A124B11681A68D3
:10FF88000B68114C4FF6FE7003400B601388206815
:10FF980023F001031B041B0C138018B12922002332
:10FFA8008271C37102224E21F1F720F92068F1F71E
:10FFB800AAFCD8E711F0B4F82378D0E7542C002035
:10FFC800D0230020D42300203C240020022828BF6E
:10FFD800022010B4084C094B207000EB8002C0EBE3
:10FFE800C20207495DF8044B013003EB4203C0B27B
:08FFF8000B6001F05FB900BFCE
:020000040801F1
:1000000082300020A23000209430002008B50BF090
:10001000C7FDF1F7C5FF0BF0ABFDFBF701FE0120BB
:10002000BDE8084001F04AB908B5FBF7AFFF0BF097
:10003000B7FDF1F7B5FFBDE808400BF099BD00BF73
:1000400008B50BF0ADFDF1F7ABFFBDE808400BF0D4
:100050008FBD00BF084B196861B130B45D68074CB3
:10006000642202FB05F2B2FBF1F2228030BC0020D8
:1000700018605860704700BFC0230020B22E0020D7
:100080002A4B1B7813B12A4B1B7803B970472DE913
:10009000F04328490B7803F0FF0E002B43D1264C88
:1000A000A368C31A002B3EDB244B254A1D78E66863
:1000B000DFF89880013D6F0007EB050C02EB4C0C5C
:1000C0003D4402EB0609BCF8043099F814C002EB79
:1000D0004502A8FB038352880D78DB08013603FB39
:1000E0000CF310440E2E0344E660A36088BFC4F8EE
:1000F0000CE035B1134803680A780133002AFBD1BC
:100100000360114B226960691C8A012500230D7070
:100110005460436203889BB22B43038013682B43D4
:100120001360BDE8F083BDE8F08300BF982C002089
:10013000992C0020D3680020C0230020D468002020
:10014000F8E20208C86B0020E0680020CDCCCCCCDF
:1001500070B40F4C0F4E054607CC0023AA603446FE
:1001600028606960012200E0A27912F0200F04F1FA
:10017000140404D101330C2BF6D170BC704703EB8F
:10018000830306EB83031B79EB7270BC704700BFDF
:100190001CE3020860010308704700BF70B5242209
:1001A000044600211DF0F1FD0B4BC4F8033014226E
:1001B0005220002602256421A27084F82200012228
:1001C000C4F80B30C4F81330C4F81B30A672A576FF
:1001D0002184A274228070BD050405002DE9F0433E
:1001E0002E4DAB6983B013B12B7F022B02D003B02D
:1001F000BDE8F0834FF020084046294C05F1200966
:100200000126552706F038FFA0B199F800300BB948
:10021000217891B908F101085FFA88F8B8F1230F45
:1002200004F1010409F10109E1D0404606F024FF80
:100230000028EAD189F80000ECE7A86950B30DF175
:10024000080EAA220EF8052D8DF802108DF8007008
:100250008DF801608DF8043069465522534008221C
:1002600013F0800F02F1FF324FEA430318BF83F00F
:10027000310312F0FF02DBB2F2D1714502D011F866
:10028000012FEBE7AA2269468DF803308DF8042090
:100290000EF034F989F80060BCE700BFC0230020ED
:1002A00028E302082DE9F04F764D81B0FCF7A0FB62
:1002B000AC6A00226A62002C00F0A180237D052B2D
:1002C000074617D9216A23690B44C31A9342B8BF62
:1002D00005F128010ADBD1E0137D052B0AD9136A49
:1002E00012691344FB1A002B80F2C88051F8042FC6
:1002F000002AF1D14FF0010B0023B9461E466B6274
:1003000098469A46274620E07A6A39693B7DA9EBF0
:100310000204B4FBF1F40134A4B213FB04F301337F
:1003200001369BB2B6B23C83FB82984506D2BBF144
:10033000000F01D1012C5CD99846BA466B6A013393
:1003400005EB83026B62976A47B3BB68C3B1FC8A53
:10035000002CD9D1396A4846A9EB01019847D0B1A0
:1003600095F87430002B52D13B7DC7F824900136AC
:1003700001334FF00102B6B23A83FB820124D4E785
:100380003B6A3A69A9EB0304B4FBF2F4A4B23C83E0
:1003900034BBFB8AC9E73C83FB8AC6E72B686A68E3
:1003A0003949013316443C4685E848004F46C1F8B8
:1003B00000A0BAF1000F27D0DAF8203095F87420A9
:1003C000AAF81640FB1ACAF81C30CAF82090002A76
:1003D00035D1DAF80C30484601B0BDE8F04F184787
:1003E0003B7D13FB04F3013301369BB2B6B2FB82B3
:1003F0009BE73A7D062A04BF9846BA469EE72B68DB
:10040000214A01332B60146001B0BDE8F08FFCF786
:10041000EFFA1E4B1E4A1F4C11681A68A0EB090028
:1004200002EB000E2268C3F800E09042A1EB5111EC
:10043000014438BF1046164A2060116094E7FCF76B
:10044000D7FADAF80C3004469847FCF7D1FADAF814
:100450002C20DAF82830DAF83010001B9042A3EB99
:1004600053130344014438BF1046CAF82830CAF871
:100470003010CAF82C0001B0BDE8F08F4FF0000B2F
:100480003AE700BFC0230020C85E0020B82E00203D
:10049000BC2E0020C02E0020F0B43423174F184A81
:1004A00003FB00F3966FFC58FD18002E6B684B6041
:1004B0000C600CDD936A9D421DD02832002303E0BE
:1004C00052F8044FA54216D00133B342F8D10022AE
:1004D000342303FB00700A720369CB60037D4B7207
:1004E000836AC56A046BC2690A615B094D618C61EC
:1004F000CB61F0BC70470122EAE700BF2008002072
:10050000C02300202DE9F041434EB46F112C67DC6D
:10051000002C7FDDB36A984262D0012C4DD0F36A83
:1005200098425DD0022C48D0336B984258D0032CAF
:1005300043D0736B984253D0042C3ED0B36B984297
:100540004ED0052C39D0F36B984249D0062C34D0CC
:10055000336C984244D0072C2FD0736C98423FD014
:10056000082C2AD0B36C98423AD0092C25D0F36CD1
:10057000984235D00A2C20D0336D984230D00B2CC5
:100580001BD0736D98422BD00C2C16D0B36D9842B3
:1005900026D00D2C11D0F36D984221D00E2C0CD00A
:1005A000336E98421CD00F2C07D0736E984217D030
:1005B000112C02D1B36E984212D0B56A45B32B7D8F
:1005C000017D8B420FD3154F00253A4605E052F8C6
:1005D000043F53B11B7D8B4207D30135AC42F6DAA1
:1005E0000020BDE8F0810D4F00256B1C9B00191FFA
:1005F000621B06EB850580463944F81892000134E9
:100600001DF0A9FBC5F82880B4670120BDE8F08182
:10061000024FEAE7D1D0E3E7C0230020E82300201F
:1006200013282DD0112807D8174B342202FB003095
:1006300019B1C3680BB165E7704770B5134DAC6F66
:10064000002C0EDDAB6A98420CD005F1280633462B
:10065000002203E053F8041F884206D00132A24270
:10066000F8D170BD002205F128069000011DA21AE4
:10067000920031443044013C1DF06DFBAC6770BD0D
:10068000034B1868D4E700BF20080020C0230020D7
:10069000C85E0020F0B50D4685B006460068F0F74C
:1006A00019F995E81800E41A0023039324238DF820
:1006B00008304D238DF80930B5F90A30FF2C224659
:1006C000A8BFFF2201333DD02B7B002B0CBF3E2364
:1006D0003C238DF80A30FE2C2B898DF80B208DF8E9
:1006E0000C3031DD23128DF80D408DF80E300727C8
:1006F0003A4602A93068F0F7F2F802ABDA190DF1C8
:100700000B0100238A4221D1002C8DF807300CDD2B
:10071000224629683068F0F7E2F82B689DF8072038
:100720001919994216D18DF8072001220DF1070100
:100730003068F0F7D4F83068F0F7C7F804F1090032
:1007400005B0F0BD2123C4E70527D1E711F8010B5F
:100750004340D7E713F8010B4240E2E7F0B5834B83
:10076000DD7A95B045B11B78022B0AD0032B00F03F
:10077000E580012B00F0CF807D4B00221A7015B070
:10078000F0BD7C4C7C4BC4F8E43200264FF41B7364
:1007900018224AF29E37626004F1140031461A466C
:1007A000A760267023611DF0F0FA284618F0BAF809
:1007B000724FC36802687A610646002B00F0A5807C
:1007C0002846F0F754FCF86718B1292200238271FB
:1007D000C371327A4E21F0F70DFD00222921307CC1
:1007E000F2F722F90023C0226549307CF2F7F8F8CD
:1007F0007869FBF78DFF17F085FEA188614A624B8F
:10080000786902FB01F29A4240F3A880002314A900
:10081000002521F84C3D5C4AADF80C500133B2FB89
:10082000F3F3A268B3FBF2F3C3F34E029BB2A281CF
:100830000293ADF80650ADF80E5018F021F8ADF85F
:1008400016500695ADF81C50ADF81E50ADF820506E
:10085000ADF82250F379ADF81450602204925A0793
:1008600078D401214FF48072ADF81410ADF8202037
:10087000002503F00203ADF81C30069504AA717937
:100880007869FBF7ABFB7179786917F0D9FF7A6962
:10089000F068536C386143F40043536403684FF6C7
:1008A000FE721340036016F093FA09A816F062FA7C
:1008B0007B6972792169ADF8301034331344334ABF
:1008C000099309A94FF400534FF0100E0A923869AA
:1008D00013954FF4807280240D95109511950F9209
:1008E0001293CDF82CE00E9416F052FA72797B69CF
:1008F0000C2A9CBF264931F81250D9683A690D4339
:10090000DD60136843F002031360194B01221A7073
:1009100018F0BEFC33E7174C1E4923701E4EC4F876
:10092000E4124FF43473182704F114001A4600211E
:100930006760A66023611DF028FA36E70D4C174B5F
:10094000C4F8E432C823122749F2704604F11400B7
:100950001A46ECE70422ADF8162089E703EB5203B0
:10096000B3FBF2F3013B9BB251E700BFD468002018
:10097000982C0020E06800202CE30208C02300200F
:10098000A1B5000840420F0000A24A04F46800200C
:100990004001030830E30208CE07070034E30208F1
:1009A00008B50E4B1978012913D00DD3022902D1B5
:1009B0000020EFF7CBFFFCF71BF8094B00F5F42004
:1009C00000F59070186008BD00210846F0F7B3FFED
:1009D000F1E70020F0F7AFFFEDE700BF6030002047
:1009E000643000202DE9F041054682B00D2006F06C
:1009F00043FB68BB404E34681CB1404F3B68AB4280
:100A000002D902B0BDE8F08110F020FF38B93C4AAD
:100A1000137A013B042B02D823780A2B55D0394A8C
:100A2000DFF8F08013786168B3B1B8F800300024C3
:100A30001470CA5C002A3AD1002242F210710133CC
:100A400001FB0255A8F800303D6002B0BDE8F0811E
:100A50000A2019F0ADFFCDE7B8F800300120107082
:100A6000CA5C002AE8D02378254A013B126800FAC4
:100A700003F3134226D0244B01221A70FFF790FF94
:100A8000B8F80030326853B911780539012906D811
:100A9000FBF7AEFF1D4B32681860B8F800305268A3
:100AA000D25CFE2A21D10023A8F80030A9E7204615
:100AB000FCF7FCF8144B1C70FFF772FF3268B8F8B3
:100AC0000030ECE7FCF7F2F8D5E7019203F076FF8F
:100AD0000120FCF733F80E4B019A1878117A0DF0CB
:100AE00013FF04F0EDF8346899E7FF2AA5D102B0AE
:100AF000BDE8F04119F040BF5C220020B422002084
:100B0000D42E0020826C0020603000208835002028
:100B1000DA3D0020B02200202DE9F04F83B0484C90
:100B2000484F0190019803685B699847002840F09E
:100B30008380DFF818914448D9F80430DFF810E1D9
:100B4000C3F308034FF00A0A4FF0100C4FF47A7504
:100B5000002B3BD1EFF31183002B37D10168A26842
:100B600000BF03689942F9D1DEF8006005FB06F387
:100B70009B1AB3FBF6F305FB013101260091D9F86E
:100B80000430C3F30803002B3BD1EFF31183002B98
:100B900037D10368A16800BF02689342F9D1DEF83B
:100BA00000B005FB0BF2521AB2FBFBF205FB03236C
:100BB000009A9B1AB3F57A7FE1D3BAF1010AB1D05A
:100BC000D9F80430C3F30803002BC3D0EFF311822C
:100BD0008CF31288A6682368D90302D501233B60F1
:100BE000A66803683968D2B282F31188DEF8002063
:100BF000194405FB02F39B1BB3FBF2F305FB013128
:100C0000BBE7EFF311888CF31288A1682368DB033C
:100C100044BF3E60A16803683A685FFA88F888F3C9
:100C20001188DEF800801A4405FB08F35B1AB3FB59
:100C3000F8F305FB0233BBE703B0BDE8F08F00BF5C
:100C400010E000E0806500208465002000ED00E0F9
:100C5000886500200F4B1A68904209D09A6890422C
:100C600012D01A69904211D09A69904210D0704700
:100C7000002110B403EBC1040022A28043F831200C
:100C8000C2625DF8044B70470121F2E70221F0E7F0
:100C90000321EEE770560020F8B50A4E0546002401
:100CA000A359AB4204EB060707D12846FFF7D2FF52
:100CB000CC22002138461DF068F8CC34B4F5197FF9
:100CC000EED1F8BD244B00202DE9F04F624D95F98F
:100CD000066091B086429DF868909DF86CA004462D
:100CE00012D095F90E00A04200F0C48195F91600CB
:100CF000A04200F0C28195F91E00A04200F0C08120
:100D0000002011B0BDE8F08F4FF0000B4FEACB068A
:100D1000A8198788002FF3D1002CF1DB022C029355
:100D20000392019140F3B680142CE9D1DFF858A169
:100D30004A48DAF81830DFF8549143F00103CAF852
:100D400018301121F0F727FC4448F0F7E0FDC820E7
:100D5000FBF7F4FE4148F0F7DFFDDAF8143043F416
:100D60000033CAF8143003234FF4C05205A94FF0E2
:100D700090408DF819304FF0020305928DF818302D
:100D80008DF81A708DF81B7016F0EAFB4FF0904347
:100D90003348596A21F470415962596A41F46041FB
:100DA0005962596A21F470215962596A4FF48022BC
:100DB00041F4602159624FF00108026012230821BA
:100DC00009F1C800C9F8C83089F8CD1089F8CE807B
:100DD00017F056FE234924480F60DAF81C30DFF87C
:100DE000B0E0224A224943F40003CAF81C300368E9
:100DF000CEF800004FF0020E1E4881F808E01160A6
:100E00001D49016098471D491D48C8604FF0020305
:100E100005A88DF815308DF817808DF814408DF8E1
:100E2000167016F07DF805A82A228DF815808DF829
:100E300016708DF8142016F097F84846114B40F8BC
:100E4000803F2E44BDF804300471B38045F83B0068
:100E500011B0BDE8F08F00BF7056002090600020F8
:100E600014040140D8004242D4070020BC560020A0
:100E7000C8560020EC5700208400002000ED00E060
:100E80000005FA0538E3020800100240C0230020E4
:100E9000F0570020E4B21946204653464A46F1F77F
:100EA000D7FD804600283FF42BAFC06C88F8059032
:100EB00088F806A00268029BC8F82070C8F81C7069
:100EC000C8F82870C8F8247022F001020121039F9D
:100ED000C8F82C70C8F8083088F8501002601AF072
:100EE0000402059300F0BA804FF4805206921AF083
:100EF000020240F0D48007924FF48062002119F082
:100F0000010A08920A9140F0B180CDF824A008228D
:100F100019F0020705A918BF099216F0C5FA98F84A
:100F2000052098F8060002F00201002915BF4FF4D1
:100F300040314FF480314FF4003E4FF0000E12F07C
:100F4000010FD8F84C20536808BF714610F0010F0C
:100F500014BF194323EA01015160916803074CBF94
:100F600041F0080121F008019160116841F0010190
:100F70001160BAF1000F37D0D8F83010002900F016
:100F8000828005A815F0F6FED8F84820D8F80C1095
:100F9000D8F81430D8F8300005924FF480520E92F1
:100FA000002206930F92802309920B920C920792D3
:100FB00020220D92ADF820100A9315F009FF05A923
:100FC000D8F8300015F0E4FED8F83010D8F84C20EE
:100FD000086840F001000860906840F040009060B0
:100FE000496889B2C8F84010002F31D0D8F83410C1
:100FF00000294FD005A815F0BDFED8F84410D8F848
:10100000102005914FF480510027D8F834000E913C
:10101000ADF820208021102207920A910F9709979E
:101020000B970C970D9715F0D3FE05A9D8F834004F
:1010300015F0AEFED8F83410D8F84C20086840F00F
:10104000020008604F604F60916841F0800191603C
:10105000116841F0010140461160F2E61AF0020AFF
:10106000069222D04FF40051079147E704220992DB
:101070000C224DE74FF0010B48E64FF0020B45E61E
:101080004FF0030B42E620211162116841F020016C
:101090001160A9E7116841F080011160D8E74FF4B1
:1010A000005207924FF4806228E7CDF81CA0524608
:1010B00024E700BF38B1038813EA010003D08B4254
:1010C0000CBF012002207047124B13491A881042AE
:1010D0000BD11A89104211D11A8A104214D11A8BDD
:1010E000104014D104230B707047012210B4002467
:1010F0000A7003EBC4005DF8044B70470222012024
:101100000A7003EBC000704703220220F8E70422B4
:101110000320F5E7D06B0020CC6B00202DE9F347CE
:101120000120FFF7D1FF174EDFF85CA00024CC2789
:1011300008B1022C02D902B0BDE8F08707FB04F821
:1011400056F8085015B10134E4B2F1E7C37890F9CC
:1011500002005AF8233001950322009201212A4609
:10116000FFF7B2FD814648B104FB0760CC22294657
:101170001CF00BFE013446F80890E4B218F0A4F815
:10118000D6E700BF244B0020ECFE020810B54FF458
:10119000804082B0FFF798FFF0B10022032390F95E
:1011A0000200009301924FF4E1334FF48041FFF7C6
:1011B0008BFD0B4B986168B101240222112021465E
:1011C00083F8204083F8214083F822401A77FFF704
:1011D00027FA204602B010BD014B9869EBE700BF2B
:1011E000C023002080B3B0F5165F2ED0B0F5964F27
:1011F0002DD0B0F5164F2CD0B0F5614F2BD0B0F5F7
:10120000E13F2AD0B0F5613F29D01D4B984228D04C
:101210001C4B984227D0B0F5E12F26D01A4B9842AC
:1012200025D0B0F5612F24D0184B984223D0184B0D
:10123000984222D0174B984205D0174B98420CBFCA
:101240000F20002070470E207047012070470220B9
:101250007047032070470420704705207047062020
:1012600070470720704708207047092070470A2000
:1012700070470B2070470C2070470D20704700BF4F
:1012800090D00300801A060020A1070040420F0002
:1012900060E3160080841E0070B02500142809D871
:1012A00000EB4000044B13F820301BB1013B012040
:1012B0009840704700207047B8F10208400040286D
:1012C000094A30B4A8BF4020002302251424D55475
:1012D0000233D118984201F8014CF8D8FF21D154BB
:1012E0000E2030BC19F064BBFC2F0020704700BFFB
:1012F00030B4034600F12405064C07CC0C3343F808
:101300000C0C43F8081C43F8042CAB42F4D130BC5D
:10131000704700BF60E30208034B33F80C2F0280D4
:101320009B788370704700BF60E3020870B5164E6B
:101330000546582404FB05641AF01CFC636813B3CB
:10134000DB6803B31149237B114A01EA40011943C9
:1013500089B20B1283EA11134B4003F00F0305EB24
:10136000850043EA011105EB400000251368257351
:1013700089B206EBC00098476368DB6858601A685A
:1013800042F001021A6070BD48620020FEFF0100B9
:101390003C620020094B00EB4000C0001A1892ED9F
:1013A000027AD2ED037AE7EE007A10B5B0EE670A62
:1013B0001C581AF0DFFB206010BD00BF60610020E8
:1013C00010B51120EFF753FE044618B11122002387
:1013D0008271C37120212046F0F7DDF80A20FBF767
:1013E00053FB2046F0F7C2FA034B00280CBF012242
:1013F00002221A7010BD00BF68520020614B1B789A
:10140000002B39D02DE9F0415F4B604D9B792C6862
:101410002860013B82B0041B032B00F28280DFE8CE
:1014200003F03002282805F053FE002800F08180E8
:10143000574B58491B786A8FD1ED037A6A64DB07F2
:1014400000F1838002FB04F007EE900ADFED526AA0
:10145000524BB8EEE77AD5ED107A5A60E7EE267A6D
:101460001A60BDEEE77AC5ED107A85ED0F7A83ED4F
:10147000027A02B0BDE8F081484A1360536093607D
:101480007047474A474BD279DFF82C8133F8122056
:10149000B8F902304448B8F9001092B207EE902A29
:1014A00040F6E44707FB02F6C3EB1633B8EE670AD3
:1014B0004FF47A7606FB03F393FBF1F32B61EEF71F
:1014C000E9FFD5F810E0D5ED027ADFED336AB8F91F
:1014D0000220324BB8F900C0C3F804E00EFB04F060
:1014E00007EE100AB8EEC77ABCEEC06AE7EE267ABD
:1014F0008DED016ABDF80410C5ED027ABDEEE77A04
:1015000007FB01F7C2EB173706FB07F683ED027AFC
:1015100096FBFCF685ED017AEE601E6002B0BDE838
:10152000F0811E4B00221A605A609A6002B0BDE83A
:10153000F0811E4B1B68DE067FF57AAF144B6A8F75
:101540001B786A64D9070FD47CE7FDEEE77A184E62
:1015500017EE900AA0F57A7101FB01F386FB0306F2
:10156000D817C0EB26100844B5F93810114B00FB12
:1015700001F083FB0013C017C0EBA31002446A64A0
:1015800060E700BF523E00204C6C002090240020F9
:101590005B5F0020543E00202FE33E31F0590020D5
:1015A000B4650020D0650020A42400203055002020
:1015B0001F85EB51D34D6210B4350020F0B5244B9C
:1015C0005B79012B83B00ED0224900230B804B8026
:1015D000214B1B78022B04D1204B48880A881880A5
:1015E0005A8003B0F0BD1E4A1E4B92781E4D33F850
:1015F0001240A4B207EE904A05F14C00B8EE670A1B
:10160000EEF748FF194A1349107896785378FCEEA4
:10161000C07A00EB4010CDED017ABDF8042044F60D
:10162000FB77C3EB033300FB027200FB0474B2FBD5
:10163000F3F2B4FBF3F3B2FBF6F2B3FBF6F392B2C0
:101640009BB2A5F84820A5F84A300A804B80BFE736
:101650004C6C00203C3E00202C3E0020303E002000
:10166000B4650020D0650020902400207D3000204B
:10167000F8B5254D25496879254C264B264E042280
:1016800064270A7001284FF0000184F8702084F864
:101690007970A4F87210A4F8741084F87810E167D7
:1016A00031701980598020D0A9791C4A0023012962
:1016B000136084F880305360936007D0022904D10E
:1016C000174AE36353609360F8BDF8BD154A636041
:1016D00053609360D3609FED140A02F110004CF246
:1016E0005031BDE8F840F1F735B8282204F1480040
:1016F0001CF04BFB4CF250319FED0C0A04F14C00F6
:10170000F1F728F8D0E700BF4C6C0020476C0020B0
:10171000902400203C3E0020523E0020F059002042
:10172000CC24002094240020CDCCCC3ECDCCCC3D8C
:101730002DE9F04F0C68DFF800E32588BB4EB6FBBF
:10174000F2F285B0013B013A74459EB2ADB292B25D
:10175000BDF838709DF83CC062D0B54B9C425FD05C
:10176000B4F1804F5CD0A3F598339C4258D003F578
:1017700080639C4254D0AF4B9C4257D003F58063AA
:101780009C4253D025F4407503F58C33ADB29C4296
:101790002580E66222850FD003F500639C420BD0C2
:1017A00003F540639C4207D003F580639C4203D05D
:1017B00003F580639C4201D10023238601236361EA
:1017C0004A79CB79BCF1000F01D083F0020313F00A
:1017D00004052FD0002113F0020F4FF040060CBF7C
:1017E0004FF0080888468C46039189468E460B4682
:1017F00001914FF4806502964FF0040A0C2A00F222
:10180000DC80DFE812F0AA00DA00DA00DA008600F5
:10181000DA00DA00DA006100DA00DA00DA002A0021
:10182000844B25F070059C42ADB2A7D12580E662BD
:101830002285C3E74FF480660396012603F0020376
:101840000295AA46A8464FF480414FF4805C4FF0C1
:1018500010094FF4807E0196D0E7256ADFF8D8E1C1
:1018600025F480552562256A6668D4F81C8025F425
:10187000005545EA0C0C744528F4E6454CEA033360
:1018800045F4C04500F0E6800EF5006E744500F0AA
:10189000E1806660E56127642362E36943F40063E5
:1018A000E361636C43F400436364238821469BB285
:1018B00043F0010321F8343B00238D184460056098
:1018C0008B5005B0BDE8F08F216ADFF86C9121F4F0
:1018D00080712162216A6668D4F81CA021F400712D
:1018E00041EA0E0E2AF0730A4C454EEA03234AF0F1
:1018F000600100F0A380DFF838E1744500F09E80BD
:101900006660E161E7632362E36943F00803E36132
:10191000C7E7216A484E21F010012162216A6568FB
:10192000D4F818C021F0200E2CF080714EEA09097D
:1019300021F4E641B44249EA031341F4C04168D0BE
:1019400006F50066B44264D06560A161A7632362B6
:10195000A36943F40063A361A3E7216A019EDFF852
:10196000D8C021F001012162D4F820906568A169F6
:1019700021F48031334321F0730129F002066445DC
:1019800043EA060341F0600138D0294EB44235D015
:1019900006F54066B44231D006F58066B4422DD0DB
:1019A00006F58066B44229D06560A1616763236251
:1019B000A36943F00803A36173E70C2A3FF671AFF4
:1019C00001A353F822F000BFB1190108A3180108C0
:1019D000A3180108A318010851190108A318010848
:1019E000A3180108A318010809190108A318010880
:1019F000A3180108A31801089B18010823F00C0381
:101A000043EA080325F4407543EA0A0345EA0E0554
:101A1000CAE723F08003029E43EA081323F0400341
:101A20003343039E25F4406535438DE700A24A0405
:101A30000034014000100040002C014023F40063FA
:101A400043EA082323F4806326F440562B434CEAF0
:101A5000060655E726F480460E431AE7F8B5494CCA
:101A600094F884305BB3042829D8474AB4F89A30F4
:101A70009FED467ADFED466A94F8985002EB8000BD
:101A800007EE903A0269B4F89E300E46F8EEE77A17
:101A9000642106EE102A01FB032367EE877AB8EE75
:101AA000C66A07EE103A67EE867AB8EEC77A87EE16
:101AB000870A20EE260A002D4FD0012D00D0F8BD58
:101AC000D4F8947007EE907AF8EE677A27EE800AE1
:101AD0001AF050F870B9D4F88800EFF718FFB4F88E
:101AE0009C003044FBF72AF8D4F88800BDE8F840A1
:101AF000EFF712BF2749284A48620023CF6253629A
:101B0000D762EFF31183502080F312880D80DBB28F
:101B1000158083F31188214BCD60D5601A68B4F825
:101B20009C10114431441A689142FCD819491A4A50
:101B30000B88D4F8880023F001031B041B0C0B80D6
:101B4000138823F001031B0400241B0C1380CC60BA
:101B5000D460BDE8F840EFF7DFBED4ED257AD4F8C5
:101B60008C50F8EE677A27EE800A1AF003F80B4BD8
:101B700028601B68B4F89C1019443144C4F8A410C0
:101B8000F8BD00BF9024002060E302080AD7233C80
:101B9000CA269B3E001000400014004084650020CF
:101BA00008B5044BD3F88800EFF7B1FE024B0022D2
:101BB0001A6108BD902400200014004008B5044BB1
:101BC000D3F88800EFF7A8FE024B00221A6108BD87
:101BD0009024002000100040012800D970470129FE
:101BE000FCD88842FAD030B4084B01EB410103EB3A
:101BF000810100EB400080000D684C688968C55089
